:020000022000DC
:1070000000000420619E0900A19E09002DAE090028
:10701000A59E0900A79E0900A99E09000000000086
:10702000000000000000000000000000059D0900B5
:10703000AD9E090000000000259D0900B19E0900D9
:107040008DA00900B39E0900F57A0900DD9B0700B9
:10705000B39E0900B39E0900097D0900B39E090093
:10706000B39E0900B39E0900B39E0900B39E0900B8
:10707000B39E0900B39E0900B39E0900B39E0900A8
:10708000B39E0900959A0900B39E0900B39E0900BA
:10709000B39E0900B39E090089600900B39E0900F0
:1070A000B39E0900B39E0900B39E0900B39E090078
:1070B000B39E0900B39E090000000000000000001C
:1070C000B39E0900B39E0900B39E090031A50900D3
:1070D000B39E0900B39E0900B39E0900897B02009C
:1070E000017B0900B39E0900B39E09000000000067
:1070F00000000000B39E09000000000061A5090027
:10710000000000000000000000000000000000007F
:10711000000000000000000000000000000000006F
:10712000000000000000000000000000000000005F
:10713000000000000000000000000000000000004F
:10714000000000000000000000000000000000003F
:10715000000000000000000000000000000000002F
:10716000000000000000000000000000000000001F
:10717000000000000000000000000000000000000F
:1071800000000000000000000000000000000000FF
:1071900000000000000000000000000000000000EF
:1071A00000000000000000000000000000000000DF
:1071B00000000000000000000000000000000000CF
:1071C00000000000000000000000000000000000BF
:1071D00000000000000000000000000000000000AF
:1071E000000000000000000000000000000000009F
:1071F000000000000000000000000000000000008F
:1072000010B5054C237833B9044B13B10448AFF3E0
:1072100000800123237010BD586C00200000000086
:10722000646D0D0008B5034B1BB103490348AFF370
:10723000008008BD000000005C6C0020646D0D0043
:10724000A3F5803A704700BF174B002B08BF134BC4
:107250009D46FFF7F5FF00218B460F461348144A61
:10726000121A88F01BFF0E4B002B00D098470D4BD5
:10727000002B00D098470020002104000D000D488D
:10728000002802D00C48AFF3008088F0C7FD200032
:10729000290072F027FE88F0D9FA00BF000008002C
:1072A000000000000000000000000420586C0020D6
:1072B00034EF0120000000000000000001460148FA
:1072C00000F07ABA906C002038B5054B1D78002488
:1072D000E0B2854203D900F02DFD0134F8E738BD56
:1072E0008C6C00202DE9F047074692B09846154671
:1072F000002A00F090804B4B93F81C6193F81D110D
:1073000093F81EA1B21C83F81C214C1C8A1C83F824
:107310001D2164F07F040AF1010241F08009E4B20A
:1073200083F81E214222002101A888F0B7FE002D1B
:107330006DD0B8F1410F73D940F20220ADF80800CA
:1073400040F20940ADF80C0040F20120ADF8100009
:1073500024208DF8160034480690731C0120DBB2FF
:107360008DF806608DF80E608DF81C008DF8266093
:107370002E48397D8DF81E30032640F608320890DD
:107380008DF8273040F224608DF82B608DF8313075
:1073900008260A230427ADF804208DF814100222D1
:1073A0000521ADF824008DF82C6040F207508DF8CF
:1073B00034304FF4116640238DF807208DF81220E9
:1073C0008DF81510ADF828008DF83320ADF8380091
:1073D0008DF83B208DF81F708DF82A90ADF82E6047
:1073E0008DF830708DF83AA08DF83C3007238DF879
:1073F0003F308DF8401044F2020342220DEB0701AA
:1074000028468DF84140ADF8423088F01FFE4220FA
:1074100012B0BDE8F087924614469146164681E7C1
:107420000020F5E7906C00202001052424020205CD
:10743000A0F11000FFF756BF07B503688DF80710DD
:107440005B6801220DF10701984703B05DF804FB6A
:1074500010B5407DFF2807D000F03CFC044608B979
:1074600073F0FEF9204610BD0020FCE707B5407D13
:10747000FF2804D14FF0FF3003B05DF804FB0DF19D
:10748000070100F04DFC0028F4D09DF80700F3E759
:1074900007B5407DFF280AD001220DF1070100F059
:1074A00025FC20B19DF8070003B05DF804FB4FF008
:1074B000FF30F9E7407DFF2801D000F03BBC70476A
:1074C000407DFF2801D000F095BC00207047F8B542
:1074D000437DFF2B06460F46144612D015465DB17C
:1074E000707D00F0D3FB38B12A463946707D00F03C
:1074F00061FC2D1A074401D1601BF8BD73F0B0F98F
:10750000EDE70020F9E7000000214FF47A72C0E9AE
:107510000112054A02F10801303202614FF47F4244
:1075200001608282704700BFE0580B0010B5437DB8
:10753000FF2B11D1094A137873B900F1100401210E
:10754000117043750649204600F0D2F921460548DE
:10755000BDE8104000F012B910BD00BF8C6C0020D7
:10756000D0580B00906C0020FFF7E0BF10B5044628
:10757000044800F0B1F8044B00221A70FF23637531
:1075800010BD00BF906C00208C6C002010B5407DB9
:10759000FF2807D000F07AFB044608B973F060F9C1
:1075A000204610BD0024FBE707B549B940B969463C
:1075B00000F082FB009BB3F5966F01D100F0FAFA60
:1075C00003B05DF804FB00000148FFF79DBF00BF5A
:1075D000746C0020F0B50546002004462B5D2E1982
:1075E000002B68D003F14002D2B2012A3DD9F42B1E
:1075F0003BD81A061BD40122A3F55846B6F5006FF6
:1076000033D3B3F5803F14444FD31E2853DCA3F586
:10761000803342009E0A0A44C3F30903A6F52056AC
:10762000A3F5105321F8106002305380D6E703F021
:10763000E002C02A1BD103F01F03022206F1010C55
:1076400016441CF8017B07F0C00EBEF1800F0CD170
:1076500007F03F07664547EA8313F2D1022A16D1A5
:10766000A3F18006B6F5F06FC6D30134B6E703F098
:10767000F002E02A03D103F00F030322DEE703F058
:10768000F802F02AF1D103F007030422D6E7032A17
:1076900004D1A3F50066B6F5784FE5E7A3F580328F
:1076A000B2F5801FE1D20422A6E7202803D021F8FA
:1076B0001030013092E7F0BD034690F850010B28DE
:1076C00008D839B1421C83F8502100F1480243F830
:1076D0002210704700207047F0B5234B89B003AAF1
:1076E000044603F11007154618685968164603C684
:1076F0000833BB423246F7D11B8833800FCD264674
:107700000FC61A4A2B681068516833806B4603C352
:107710006B4603CB137A84F82030154BC4F818312C
:107720004FF48073A4F81C3104F118050123A06103
:10773000E16184F81E3165612022002104F5987012
:1077400088F0ACFC40F20943C4F82031094BC4F87E
:107750002431094BC4F828310023C4F82C31042308
:1077600084F8503109B0F0BD3C590B004E590B0064
:107770000900000114590B0021590B0038B50446CB
:107780000846B4F81821B4F81A31616905689B1AE3
:107790002D680A449BB294F81C11A84758B1B4F85C
:1077A0001831626903449BB2A4F81831538094F8ED
:1077B0001C311371012038BD70B504460D460126F9
:1077C000FFF78AFF40F2EF23A3804FF4E131044832
:1077D000A671FFF7ABFE284600F0DAF9304670BD1F
:1077E000746C00202DE9F041D0F82C5188B08C1C2D
:1077F000002D3BD1684600F0DFF9224603462C46B7
:10780000E1B28B4202F104022BD91B4D04AF05F10A
:1078100010083E46C64628686968BC46ACE80300C6
:10782000083545456746F6D11DF80470124D07F03E
:107830000F0108A8014411F8101C22F8021C286846
:107840006968B446ACE80300083575456646F6D16C
:1078500008A901EB1717013417F8101C22F8041CB3
:10786000CEE75800C0B208B0BDE8F08121462846F6
:10787000FFF7B0FEF6E700BF2B590B0010B504462A
:1078800079B103291BD090F850318B421CD901F1FA
:10789000480300F5AA7150F82300FFF79BFEC0B221
:1078A00004E0D0F82031A0F854310120013040002C
:1078B00040F44070A4F8520104F5A97010BD00F521
:1078C000A971FFF78FFFF1E70020F7E70048704745
:1078D000906C0020014B5869704700BF906C0020ED
:1078E0000A4601460148FFF7C9BF00BF906C00205F
:1078F00010B504460248FFF7DFFE207110BD00BF3F
:10790000906C0020024B53F8200000B1C068704713
:10791000246E002030B40546084C54F82540084633
:1079200011461A46BDF8083024B1246914B1A446A2
:1079300030BC6047002030BC704700BF246E002080
:1079400030B40546074C54F82540084611461A46FF
:10795000BDF8083024B1646914B1A44630BC604756
:1079600030BC7047246E002000207047024B18681E
:1079700008B190F8600070472C6E00202DE9F843A4
:107980001F461F4B0446186889469046002834D08D
:107990002C2303FB04001B4B066A456A846A002EF5
:1079A00008BF1E46184B002D08BF1D46174B30461A
:1079B000002C08BF1C4689F08BFE08280246314681
:1079C00028BF0822484688F041FB284689F080FEFF
:1079D00010280246294628BF1022404688F036FB70
:1079E000204689F075FE042802462146384628BF05
:1079F0000422BDE8F84388F029BBBDE8F88300BF46
:107A00002C6E002057590B0060590B00BC980B00DE
:107A100070B50D4E34680546A4B12C2303FB004419
:107A2000636913B1984784F8320032682C2303FB52
:107A3000052393F832402CB923463A2202212846E6
:107A400000F048FF204670BD2C6E0020054B1B68DF
:107A500010B533B12C2404FB0030C36A0B60038ED5
:107A6000138010BD2C6E002008B5202200230521B4
:107A700000F030FF4FF0FF3008BD000030B4044686
:107A8000084611461A46064B1B6833B12C2505FBE8
:107A90000434E3690BB130BC1847012030BC704797
:107AA0002C6E002030B4044608461946074B029A53
:107AB0001B6833B12C2505FB0434A3680BB130BC23
:107AC00018474FF0FF3030BC704700BF2C6E0020CD
:107AD00030B4044608461946074B029A1B6833B176
:107AE0002C2505FB0434E3680BB130BC18474FF07C
:107AF000FF3030BC704700BF2C6E0020044B1B6869
:107B00002BB12C2202FB0030036903B118477047E8
:107B10002C6E0020054B1B682BB12C2202FB003081
:107B2000836903B118470120704700BF2C6E002005
:107B300004F0C2B807B5124B402283F82723002077
:107B400002F072FC4FF080430024D3F838548DF8D3
:107B50000040684672F032FA0A4B019301A872F0B5
:107B60008BFA72F053FAEB0702D5204604F0A4F822
:107B700000214FF0FF3002F0B1FEFFF7A5FBF7E761
:107B800000E100E0317B0200002003F095BE000020
:107B900007B500230322CDE9002304490448C82285
:107BA00071F050F903B05DF804FB00BF6D590B0094
:107BB000357B020073F008BA4FF08052536E1BBA47
:107BC0000360136E1BBA436008207047004870477B
:107BD00072590B0070B51A4E33680D4611466BB3DF
:107BE000012D01D0012070BD1478C4F34114012C83
:107BF00013D0022C22D15278012A07D0022AF1D1C7
:107C00008B88072B1AD10F4A138902E09A69AAB10F
:107C10001378BDE8704003F049BA5278222AE1D1C6
:107C20004A88003A18BF01225A7503F027FA3268D1
:107C3000D369002BD6D0507D9847D3E70020D2E7F8
:107C4000306E00200460002070B500F1100504467D
:107C5000284602F005FB3F2815D9E178002002F004
:107C6000A1FD80B1284602F0FBFA3F28E17807D950
:107C700004F536724023BDE87040002002F0B2BD2A
:107C8000002002F09FFD002070BD000010B50446EA
:107C900002F0B2FB08B9002010BD02F0B5FB0028CD
:107CA000F9D104484FF4567303FB0404207900F023
:107CB0000100F1E7346E0020054B4FF4567202FBD1
:107CC0000033986808609A899B7B8B718A80704723
:107CD000346E002008B5044B4FF4567202FB00309E
:107CE000103002F0A5FA08BD346E00204FF4567330
:107CF00058430A4B70B54FF6FE764FF6FF741D18C9
:107D0000B24288BF2246103092B2184402F0BAFA4A
:107D100004462846FFF798FF204670BD346E0020C9
:107D2000034B4FF4567202FB0030103002F0ADBA34
:107D3000346E00202DE9F041044602F05DFB10B9DD
:107D40000020BDE8F08102F05FFB06460028F7D175
:107D50004FF45671154D4C4304F12408A844404695
:107D600002F066FA0028EBD02F193046B97802F0FD
:107D700019FD0028E4D004F5467425442946402224
:107D8000404602F07FFAB978044658B103462A46C5
:107D9000304602F027FD38B9054B1B68DB07CFD50D
:107DA00000BECEE702F00EFD2046CAE7346E00208A
:107DB000F0ED00E00E4B70B54FF4567404FB003448
:107DC00005464FF6FF734FF6FE70824288BF1A4693
:107DD000243492B2204602F073FA0646204602F09E
:107DE00027FA3F2802D92846FFF7A4FF304670BD86
:107DF000346E002008B5044B4FF4567202FB00307D
:107E0000243002F02DFA08BD346E002073B51A4CF0
:107E10004FF456720021204688F040F9FF23637129
:107E20004FF4E1330025A36008230126A37304F176
:107E30003801009501234FF4807204F11000A581F0
:107E400002F0C5F933464FF4807204F59C71009638
:107E500004F1240002F0BBF904F50E71304670F015
:107E6000A3FC04F52271C4E90750304670F09CFC75
:107E7000C4E90C0502B070BD346E002010B5094C89
:107E800000232360237104F11000243402F01EFA51
:107E9000204602F01BFA20460121BDE8104002F006
:107EA00035BA00BF346E0020F7B54B79022B074678
:107EB00003D00025284603B0F0BD8B79022BF8D102
:107EC0001F4EB3787BBB8B7833700C7809250C443C
:107ED00003E023781D44ADB21C446378242B1BD1EE
:107EE0009542F6D96378042B12D163790A2B0FD10E
:107EF000144B267801930133009302231A46A119EB
:107F0000384602F01BFC70B10E3516FA85F5ADB29D
:107F10000B48FFF799FECDE7052BE3D12146384604
:107F200002F0E8FB28B9084B1B68DB07C1D500BE8F
:107F3000BFE7A378737023781D44ADB21C44D1E72A
:107F4000346E0020366E0020F0ED00E038B50B46B0
:107F50001146127802F06002202A47D1244A8C8808
:107F60001578A54242D14C78203C032C3ED8DFE85E
:107F700004F002141731012B05D11E4A072303F028
:107F800095F8012038BD032BFBD11B4B002BF8D0FB
:107F900018490020AFF30080F3E7012BF1D1ECE7A3
:107FA000012B02D103F06AF8EBE7032BE9D14C88EF
:107FB0001248147104F0010585F0010102F0A6F9E0
:107FC0000F4B002BDDD0C4F3400229460020FFF701
:107FD000EBFAD6E7012BE5D0032BD2D1094B002BCE
:107FE000CFD049880020AFF30080CAE70020C9E75E
:107FF000346E00203C6E002000000000586E00200F
:10800000A9750200000000002DE9F3471C46374B1C
:10801000DA788A4207460E461D4607D09B788B4287
:1080200058D1AB78B34232D001245AE003F536710F
:1080300003F11000A2B202F043F92D4B2BB92D4BE6
:10804000EBB92A48FFF700FEEBE76B79FF2BF6D080
:1080500005F536794FF0000805F1100AA045EED07D
:1080600019F8013B6A799A4206D1504602F0F0F8BD
:1080700010B96979AFF3008008F10108EEE71E48F6
:1080800002F0E6F80028DCD1AFF30080D9E71B4B03
:1080900013B10020AFF300800020FFF74BFE002853
:1080A000C2D1174802F0C4F80028BDD1002CBBD0C3
:1080B00014F03F03B8D1A9780193384602F072FB5F
:1080C000019B04460028AFD0A9781A46384602F032
:1080D00089FB06E00B4B1C6814F0010401D000BEC4
:1080E0000024204602B0BDE8F08700BF346E0020B7
:1080F0000000000000000000446E002000000000AE
:10810000586E0020F0ED00E002484FF48C72002120
:1081100087F0C4BF8C7100200020FFF7F5BF00007E
:108120002DE9F34713464A79032A81460D4604D0C8
:108130000024204602B0BDE8F0870A79C2EBC204F1
:108140001234A4B29C4223D8284B59781F4629B137
:1081500093F88D30E3B94FF0010800E088462B78A2
:10816000E9184878212813D18C2606FB08F607EB7E
:10817000060ACAF88810E85C731C3B440193B31CE0
:108180003B44009301440323484602F0D7FA28B940
:10819000174B1B68DA07CBD500BEC9E7AB79012BBB
:1081A00004BFEB798AF803308C2303FB08F807EB54
:1081B000080301221A71AA7807F80820D3F888204A
:1081C0009978B2F80720DA800029B2D006F1480287
:1081D00040233A44484602F005FB0028A9D1044B4D
:1081E0001B68DB07A5D500BEA3E700BF8C7100208C
:1081F000F0ED00E013782DE9F74303F01F06012EA0
:1082000007460C46154601D0002480E091887D4A3F
:108210001078C9B2884291460AD092F88C208A42DE
:10822000F2D113F060032AD1012C03D001246EE0B7
:108230000026F6E76B78062BE6D16B881B0A212B0C
:108240000ED18C2202FB0696D6F88820002ADBD0BD
:1082500013782946384603B0BDE8F04302F026BF44
:10826000222BD1D13046FFF74DFB8C2303FB069622
:108270000246F3882946384602F018FF47E0202BD3
:10828000C2D16B78013B0A2BBED801A252F823F071
:10829000BD820200B7830200C98302000982020086
:1082A000098202000982020009820200098202009A
:1082B0002B83020089830200DB830200012CB5D1ED
:1082C00008234FF08C0C1CFB063CEB886988402B84
:1082D0004FEA1122184628BF402011F0FF0109EB98
:1082E0000C0818D0012B16D9013809F80C1008F128
:1082F000010380B200903046FFF70CFB0444A4B2A7
:1083000064B9414B1B68DB077FF57EAF00BE20469A
:1083100003B0BDE8F08343460024EBE72346424622
:108320002946384602F0C2FE80E7012C08D1EB88CE
:10833000402B3FF669AF8C2202FB0692483299E748
:10834000032C7FF473AF6988ED884823402D4FF0EC
:108350008C044FEA112214FB0634284628BF402023
:1083600011F0FF0109EB040309D0012D07D919F819
:1083700004408C4202BF00F1FF30013380B2009014
:108380003046FFF7DDFA51E7012C7FF44FAF6988E3
:108390001E4B8C2202FB0699090A89F805102BB1A5
:1083A0003046AFF3008000283FF42EAF2946384610
:1083B00002F064FE3AE7012C7FF438AF8C2202FB16
:1083C00006922346053255E7012C7FF42FAF8C220D
:1083D00002FB0692234604324CE7012CE6D0032C24
:1083E0007FF424AF69880A4B8C2202FB0699C9B23C
:1083F00089F80410002B3FF419AF3046AFF300802A
:1084000014E700BF8C710020F0ED00E000000000D8
:108410000000000073B5224C0546A07862788842BF
:1084200012D08A4210D094F88E0094F88D208842A1
:1084300012D0914210D01B4B1B68DA0702D40020E7
:1084400002B070BD00BEFAE7002062788A420CD10B
:10845000154A22B90120F3E78C340120F5E79AB2DE
:1084600004F10801AFF30080F4E7A2788A42F1D169
:10847000002204F148069BB2114600933346FFF7F1
:108480005FFAA17840233246284602F0ABF9002873
:10849000E0D1044B1B68DB07D1D500BED0E700BF9D
:1084A0008C710020F0ED00E00000000070B500F1DC
:1084B00010050446284601F0D3FE3F2817D9A178BD
:1084C000002002F06FF990B1284601F0C9FE3F2864
:1084D000A17807D904F5EC724023BDE87040002074
:1084E00002F080B9BDE87040002002F06BB970BDA9
:1084F00070B500F124040546204601F099FE08B944
:10850000002070BD6978002002F04CF90028F7D0F7
:1085100005F5067631462046402201F0B3FE697823
:10852000044658B103463246002002F05BF938B9E0
:10853000044B1B68DB07E3D500BEE2E702F042F91B
:108540002046DEE7F0ED00E037B5154C00254FF48E
:1085500016720021204687F0A1FD04F13801009534
:108560000123802204F1100001F031FE012380225A
:1085700004F1B801009504F1240001F028FE04F58F
:108580009C71012070F010F904F5C471C4E9075022
:10859000012070F009F9C4E90C0503B030BD00BF3B
:1085A000E8EB012010B5084C10220021204687F08E
:1085B00075FD04F1100001F089FE04F12400BDE80E
:1085C000104001F083BE00BFE8EB01202DE9F04729
:1085D0004B79012B8046924603D000252846BDE802
:1085E000F0878B79012BF8D1CB79002BF5D10C7862
:1085F00023460C446278242A06D15345EDD82278CC
:1086000013449BB21444F5E7042AE6D16279012AA7
:10861000E3D1A279032AE0D1E579002DDDD11E4A0C
:10862000577891780F43914630D1A27889F800208D
:1086300026789D19ADB2264410E0B378DA0914BF4C
:1086400089F8013089F80230337801371D44ADB222
:108650001E44FFB233781D44ADB21E442379BB42A1
:1086600003D80D48FFF722FFB8E75545F9D87378CE
:10867000052BEFD13146404602F03CF80028DCD112
:10868000064B1B68DA07A8D500BEA6E7034B1B689C
:10869000DB07A2D500BEA1E7E8EB0120F0ED00E08A
:1086A0000020704773B51F4D1C46AB788B420646C1
:1086B0001DD06B788B422BD12846FFF719FF28BBC2
:1086C00005F1240001F0B4FD00BBFCB114F03F0340
:1086D0001CD169780193304602F064F8019B04468E
:1086E000A0B169781A46304602F07CF817E0A2B2D1
:1086F00005F5EC7105F1100001F0E2FD0A4B13B134
:108700000020AFF300800748FFF7D0FE012406E009
:10871000064B1C6814F0010401D000BE0024204662
:1087200002B070BDE8EB012000000000F0ED00E0B9
:10873000034B43F602229A87002283F83E207047BB
:10874000A474002030B4104B02249A6B83F82C10D0
:10875000996883F8304093F83C408A1A9A6224B9A9
:1087600042F205059D8783F83E4051B14AB11A7B1C
:10877000D20930BC14BF93F82E1093F82F1002F0DA
:1087800071B830BC704700BFA474002038B5144BDA
:10879000144C054673B1607BFFF7BCF950B942F247
:1087A000077384F83E00A38728460121BDE83840BE
:1087B000FFF7C8BFA26BA36894F82F109B1AB3F5FC
:1087C000007F28BF4FF40073074A9BB2284602F08F
:1087D00009F820B9054B1B68DB0700D500BE38BD82
:1087E000157B0200A4740020A4720020F0ED00E0CC
:1087F00070B5254CE28AA36852BA92B286B005469B
:1088000012B1B3FBF2F292B2A06BD4F81110B0FB2C
:10881000F2F61B1AB3F5007F28BF4FF4007309BAB4
:10882000009302FB1602194B607B3144FFF73AF9C3
:10883000031E07DAFFF77CFF01212846FFF782FFBE
:1088400006B070BD94F82E1010D1CDE90333072285
:108850008DF8101003A819468DF80C508DF80D20D6
:1088600005938DF8113001F05BFEE9E7074A9BB2F2
:10887000284601F0B7FF0028E2D1054B1B68DB0753
:10888000DED500BEDCE700BFA4740020A472002087
:10889000F0ED00E0C28A836852BA92B223B9002A8E
:1088A0000CBF002002207047C17B282904D1017B26
:1088B000C90906D1022070472A2902D1017BC909C2
:1088C000F8D122B1934234BF02200020704701202A
:1088D00070470000044880F83C1080F83D2080F884
:1088E0003E300120704700BFA4740020024840229F
:1088F000002187F0D3BB00BFA474002002484022AF
:10890000002187F0CBBB00BFA474002073B54B7966
:10891000082B054602D0002002B070BD8B79062BD3
:10892000F9D1CB79502BF6D1162A05D8174B1B68F5
:10893000D907F0D500BEEEE7154C8B7884F82D30C2
:1089400004F12E030E78019304F12F030093022308
:108950001A46314401F0F2FE28B90C4B1B68DA07C5
:10896000D9D500BED8E7002384F8303094F82F1012
:108970001F232246284601F035FF20B9034B1B6810
:10898000DB0700D500BE1720C6E700BFF0ED00E012
:10899000A4740020F0B5012985B00646154615D10E
:1089A000137803F07F02022A46D16C78012C43D160
:1089B0006A88002A40D13C4AAB8892F83070042F74
:1089C000DBB2154604D1194601F04CFF012017E037
:1089D00092F82E10994215D1022FF7D19368946B1B
:1089E0001B1B9362032382F830300D23203201F0E9
:1089F000F9FE0028EAD12D4B1B68DB0752D500BEDB
:108A000005B0F0BD92F82F109942DFD1002FDDD1D3
:108A1000019101F019FF01990028D7D1304602F0E9
:108A2000BFFA0028D2D1002385F830301E4A95F8CD
:108A30002F101F233046DAE703F06003202B31D1DB
:108A40006B78FE2B13D0FF2B2CD16B8853BBE9889E
:108A50008AB23ABB144B304699872946C3E90D22A6
:108A600083F8302083F83E2002F008FBAEE76B88E5
:108A7000C3B9EB88012B15D18DF80F300C4B1BB10E
:108A8000FEF774FF8DF80F009DF80F3053B1013BD6
:108A90008DF80F300DF10F0201232946304602F008
:108AA00005FB93E70020ABE7A4740020F0ED00E0A5
:108AB0006D7902002DE9F041AB4C94F83070012F34
:108AC0008EB005461E4600F09F81032F00F00D82F8
:108AD000002F42D194F82F308B4201D0012013E0B7
:108AE0001F2E03D12268A14B9A4210D094F82E1069
:108AF0000423284684F8303001F0B4FE94F82F1097
:108B0000284601F0AFFE00200EB0BDE8F081984B82
:108B100023626368E67BD4F8088084F82C70C4E98B
:108B20000937012384F8303006F0FD03282BC4E90F
:108B30000D872CD12046FFF7ADFE014618B128461F
:108B4000FFF700FE09E0B8F1000F00F05781282E72
:108B500040F0AA812846FFF74BFE94F83030022BF4
:108B6000BCD194F82E10284602F01AFA0028B5D18C
:108B7000A368A26B94F82E10934240F2DF81207B11
:108B8000C00900F0DB81284601F06CFEA6E7B8F1D1
:108B9000000F15D0237BDB0912D1B8F5007F01D976
:108BA0000121CCE7734A1FFA88F3284601F01AFE28
:108BB0000028D2D1704B1B68D907A4D500BEA3E70B
:108BC000252E94F80D8008D8192E14D8032E00F005
:108BD000DD80122E00F08C8066B394F83C30002BC0
:108BE000DED1A38E634A6549607BFEF73DFF002816
:108BF00080F2FD80D4E71A3E0B2EEED801A353F885
:108C000026F000BF338D02004F8C0200DB8B020088
:108C1000DB8B0200DB8B0200DB8B0200DB8B0200B4
:108C2000DB8B0200DB8B0200A98C0200DB8B0200D5
:108C30006B8C02004046FEF7EBFE002840F0DA8025
:108C400094F83C30002BC8D1FFF772FDC5E74C4BC0
:108C5000002B00F0CF80E17C4046C1F3400301F0DF
:108C600001020909FEF70AFFE7E704AA05A9404641
:108C7000FEF7ECFE059B002BE2D0BDF81020002A89
:108C8000DED03C49013B1BBA12BAC1E900320820D0
:108C9000A368002B84D0834228BF03466363354A10
:108CA00094F82E109BB280E700230DF10E0205AE62
:108CB00004A94046C6E901330593FEF7C7FE049AAE
:108CC000002ABDD0BDF80E30002BB9D012BA5BBA65
:108CD000082106920222ADF81E308DF817108DF88B
:108CE0001C2096E80700234B83E807000C20CFE701
:108CF000244B204F0022CDE905324FF020361F23B0
:108D00001022202109A8CDE907668DF8183087F0D8
:108D1000C5F90D960DAB09AA07A9404605AEFEF7A9
:108D20002DFE0FCE0FC70FCE0FC733683B60242038
:108D3000AEE7059B03F4000343F003030593124BD6
:108D40007BB14046FEF7E6FE9DF8163080F001004C
:108D500060F3C7138DF81630064B059A1A6004208D
:108D600096E70120F0E700BFA4740020555342436A
:108D700055534253A4720020F0ED00E0B37400207C
:108D80007D7A020000800202157B0200122200217F
:108D900005A887F083F994F83C0094F83D1094F806
:108DA0003E208DF82010F0238DF814304FF0000392
:108DB00060F303038DF816300A238DF81B308DF80D
:108DC000212005AE0FCE644F0FC733683B80634B45
:108DD000C3B14FF40072A7F110014046AFF3008019
:108DE00000239842A38784F83E30FFF6F6AE0028B1
:108DF0007FF44EAFA368002B7FF4D2AE022384F839
:108E00003030AAE61220EBE7E37BA26B282B05D1DA
:108E1000636B32449A42A263F0D29BE62A2B47D17D
:108E2000E08A40BA80B218B1A368B3FBF0F080B218
:108E3000D4F81110484FB2FBF0FC09BA00FB1C2219
:108E40000096607B3B466144FEF742FE002805DA4F
:108E5000A36B3344A363FFF76BFCA1E686421DD9E5
:108E6000361A40B1A16B11FA80F1A163324639186C
:108E7000384687F0F9F8002194F82F30079607223A
:108E800005A8CDE905118DF814508DF815208DF841
:108E900018308DF8191001F043FB5EE6A36B1E44F9
:108EA000636BA6639E42A9D22846FFF76FFC54E687
:108EB000237B3244DB09A2630CD1A38E264A607B5C
:108EC00004F10F01FEF7D0FD002803DA39462846E9
:108ED000FFF738FCD4E90D329A428FD2204B1B6841
:108EE000DB077FF53AAE00BE37E694F82E308B42B2
:108EF0007FF433AE0D2E7FF430AEE37B282B09D008
:108F00002A2B14D0174B53B1607B04F10F01AFF340
:108F1000008004E0144B13B1607BAFF300800023AA
:108F200084F83030114A94F82F101F233DE6104B7F
:108F3000002BF4D0607BFEF7E1FDF0E79B1AA36203
:108F4000032384F830300B4A0D23284601F04AFCF5
:108F500000287FF4C3AD2DE6A472002000000000BD
:108F6000F0ED00E00000000000000000A47400200C
:108F7000FD7A0200C474002010B5044681780020F8
:108F800001F010FC90B1201D01F06AF93F28A17892
:108F900007D904F5A6724023BDE81040002001F077
:108FA00021BCBDE81040002001F00CBC10BD000049
:108FB0002DE9F041044601F01FFA10B90020BDE888
:108FC000F08101F021FA06460028F7D14FF4E6714E
:108FD000154D4C4304F11808A844404601F028F907
:108FE0000028EBD02F193046797801F0DBFB002800
:108FF000E4D004F5C674254429464022404601F0D9
:1090000041F97978044658B103462A46304601F0C2
:10901000E9FB38B9054B1B68DB07CFD500BECEE7AF
:1090200001F0D0FB2046CAE7E4740020F0ED00E038
:1090300037B5144C00254FF4E6720021204687F026
:109040002DF804F12C01009501234022201D01F090
:10905000BEF80123402204F16C01009504F11800D0
:1090600001F0B5F804F1AC0101206FF09DFB04F1B3
:10907000FC01C4E9045001206FF096FBC4E9090526
:1090800003B030BDE474002010B5064C2046002328
:1090900040F8043B01F01AF904F11800BDE8104053
:1090A00001F014B9E4740020F7B513464A79FF2A99
:1090B0000D4602D0002003B0F0BD1A4E7178B27890
:1090C0000A43F7D1AA782C7832702A792C442AB333
:1090D000234403E09C4204D221780C4461780529A2
:1090E000F8D1114F01977B1C00932146022301F018
:1090F00025FB28B90D4B1B68DB07DBD500BEDAE783
:109100002B79C3EBC3031C44B37813B1781EFFF76C
:1091100033FF737813B10020FFF74AFF601B80B262
:10912000C9E700BFE4740020E5740020F0ED00E022
:1091300008B5114882788A4204D042788A4211D018
:10914000002008BD9AB200F5A671043001F0B8F80D
:109150000A4B13B10020AFF300800748FFF70CFF64
:109160000120EEE7064A1AB199B20020AFF3008061
:109170000020FFF71DFFF3E7E4740020000000006B
:1091800000000000C3883BB1027804490B2000FBBB
:10919000021210681844704718467047B0760020D5
:1091A000884202D24378934200D170470378184432
:1091B000F6E7000038B50B4D1446884201D3084647
:1091C00038BD8378112B06D825FA03F3DB0702D5C7
:1091D000C378A342F4D0037824221844FFF7E0FFB9
:1091E000EBE700BF5010020010B51446884201D3CF
:1091F000084610BD837803F0FD02052A01D0112B2B
:1092000002D1C378A342F4D0037824221844FFF794
:10921000C7FFEBE72DE9F0410C46FFF7B3FF18B1AC
:10922000A278037B9A4207D9484B1B68DB0700D51D
:1092300000BE0020BDE8F0812AB9012B01D9012030
:10924000F8E70122A2706FF03F03A3766FF00303EB
:10925000E3766FF064032377032300254FF00108C2
:10926000A377082384F808806572A572E57284F8F4
:109270000E80E5732574657484F81D8084F81F8062
:1092800084F8208084F8218084F8225084F82330E8
:109290000378B0F80D10194401441844FFF78AFF11
:1092A00088420646C0D08778042F3BD0062FC0D115
:1092B000E27833799A42B7D81AB9012BBFD8012284
:1092C000E27030783044FFF78FFF8842ACD0D4F89A
:1092D00012302BB9042F29D0062F30D0C4F8123009
:1092E000626852B9417E0129A9D8D0F81A2019B96B
:1092F000D0F81E109142A2D1626042F20F718A42F0
:1093000092D9013B42F21071B2FBF1F21344B3FB6C
:10931000F2F30233B3F5807F28BF4FF48073C4F8B3
:1093200016308CE784F80C806573C1E7B0F807301D
:10933000B0F805205A43737D5343DB08CEE7B0F8FD
:109340000520B0F8073053431B01F6E7F0ED00E0CD
:109350002DE9F0410446416990F850002369A7695E
:10936000461A1E44BE42354628BF3D46854209D2B4
:109370000F4B1D6815F0010501D000BE00252846E1
:10938000BDE8F081E368A5EB00085030194442467F
:10939000204486F05BFE6369BE42434463619EBF26
:1093A00094F8513043F0020384F85130E7E700BFEE
:1093B000F0ED00E038B514461D46884201D308465A
:1093C00038BD8378A34202D1C378AB42F8D003788A
:1093D00004221844FFF7E4FEEFE78278884202D2C5
:1093E0008378934200D07047037818448142F5D9BE
:1093F0004378042BF2D00B2BF6D1EFE72DE9F041A7
:109400000F680E46898813463944BA788046384634
:10941000FFF7D0FF8142044602D80020BDE8F0816A
:10942000037D012B05D9134B1B68DA07F5D500BE68
:10943000F3E70379CBB1012BEFD10378C5891D4444
:109440000544407A1844294605222044FFF7A8FE27
:10945000A8420146E1D2404601F04CF928B9054B3B
:109460001B68DB07D9D500BED8E7E41BF4800120D8
:10947000D4E700BFF0ED00E02DE9F84F17460B7878
:10948000424A0C460B2101FB03238246D3F800809D
:1094900023896BB143440025997801F08FFD6389DE
:1094A00025812BB143445046997801F087FD6581B1
:1094B00000266088B4F804906661C4E903664044FD
:1094C000C14482783B464946FFF774FF8145054613
:1094D00002D80020BDE8F88F90F804B0BBF1020F6D
:1094E00005D92B4B1B68DA07F3D500BEF1E7A0EBDB
:1094F0000803E38067B1297804F108060D4406EB00
:109500004B0BB3451ED10FB1022363770120E1E776
:10951000637F012BEFD004F11E0339466777A76103
:109520003022184686F0BAFD01462046FFF772FE4B
:109530000028E0D1CDE76B78052B06D0042BD0D0E6
:109540002B781D44A945F6D8CBE7EB7803F003034D
:1095500097B1012B05D1AA88A369C2F30A029A42E6
:10956000B7D32946504601F0C5F840B9084B1B68EF
:10957000DB07AED500BEADE7022BF2D0A9E7A5EB25
:10958000080326F8023B2B781D44BAE7B07600208A
:10959000F0ED00E0044B0548002159601960C3F864
:1095A0000710502286F07ABDB0760020BC760020ED
:1095B000044B0548002159601960C3F80710502278
:1095C00086F06CBDB0760020BC7600202DE9F04F0F
:1095D0002DED028B4B790E2B08EE100A85B00C4650
:1095E000174605D0002005B0BDEC028BBDE8F08F1A
:1095F0008B79012BF6D1CB79012BF3D1314ED6F8F3
:109600000080B8F1000F57D13160B2803146424638
:10961000FFF7F4FE0028E5D0F2883368DFF8AC905D
:10962000134427443946204693F814B0FFF7D5FE7B
:1096300006F10803054601935FFA88FAD34503D87B
:109640002C1BA0B2B480CEE7B9F80220A2BB019BCC
:1096500089F8002003F8012B3946019328462B1B7B
:109660000392A9F80230029389F801A0FFF7B5FE32
:10967000039A029B89F81D20011B0546A9F80410D6
:10968000BAF1000F02D008F10108D5E7BBF1010FD4
:10969000F9D114FA83F014FA81F182785B46FFF76E
:1096A00089FE8142EFD118EE100A52464946FFF773
:1096B000E3FE0028E7D195E7034B1B68DB0791D554
:1096C00000BE8FE7B0760020F0ED00E0BC76002011
:1096D0002DE9F0478846117801F01F03012B8EB069
:1096E0000746154648D1A94E938832685FFA83FC35
:1096F000B146002A00F0E6809478644540F0E280AC
:10970000C1F3411A11F0600F544603D0012C67D009
:1097100007230BE06B780A2B0AD00B2B24D09C4B31
:10972000186810F001004FF0070356D1737223E060
:10973000B8F1010F04D0002389F8093001240FE0AB
:10974000EB88012B15D1F1880A442946D2788DF88F
:10975000082002AA01F0AAFC044650B186F809A02C
:1097600020460EB0BDE8F087B8F1010FE3D1EB88D9
:1097700023B1FF2389F809300024F1E7B9F8061076
:1097800053181879A8B1525C587AD98910441144F9
:10979000194405221844FFF703FD814205D87C4B8C
:1097A0001B68D807E5D500BEE3E78178384601F0AD
:1097B00005FC002689F8066089F807606A88734905
:1097C0003846FFF71BFE04460028D2D0294638460B
:1097D00001F054FC89F80960C2E700BE7372BFE76C
:1097E0001C0A57D16B881A0A012A0AD0022A3ED0D5
:1097F000674B186810F001004FF00703BAD000BEA5
:10980000B8E76B78812B24D0862B27D0012BEFD1A2
:10981000B8F1010F0BD1EB88012BAAD15D4A0123CE
:109820002946384601F042FC002884D1A1E7B8F16E
:10983000020F80D1584B002B3FF47DAF99F80A10EE
:109840000020AFF3008089F80900B0FA80F46409C1
:1098500086E7B8F1010F7FF46EAFDCE7B8F1010FD6
:109860007FF469AFEB88012B83D14C4AD8E76B7842
:10987000812B08D0862BBBD1B8F1010F7FF45BAFF1
:10988000474A4346CCE7B8F1010F7FF454AF454A4D
:109890000123C5E7B9F80630D018D15CC389194453
:1098A000014481427FF647AF8378023B052B03D802
:1098B000C378A3423FF43FAF037824221844FFF754
:1098C0006FFCEEE7DFF8E0A0BAF802005646002889
:1098D0003FF452AF9AF800200B2101FB0299D9F80E
:1098E00000402044827862457FF446AF2A78C2F374
:1098F000411912F0600F484603D0012856D00723C3
:1099000041E06B780A2B0BD00B2B29D0204B1C6825
:1099100014F001044FF0070334D18AF81C301FE71C
:10992000B8F1010F02D00023337707E7EB88012B52
:1099300040F021825046FFF725FC002800F01B82F2
:10994000C3788DF8083002AA43462946384601F00C
:10995000ADFB0446002800F00E828AF81C90FFE65A
:10996000B8F1010F40F0A3806A8851463846FFF7EE
:1099700083FD0446002800F0FE812946384601F0A8
:109980007DFBEAE700BE8AF81C30F5E6B0760020E1
:10999000F0ED00E0BA76002000000000AC590B00AA
:1099A000AB590B00B9760020BC7600201C0A2CD1E4
:1099B0006A88130A022B00F07581062B1BD0012B3D
:1099C0001ED1737F03B1747795F80190B9F1010F3F
:1099D00034D009F17F03DBB2062B11D8A9F1810342
:1099E000062B0DD8DFE813F067014000400040006F
:1099F000B001530140006B78812B08D0862B16D024
:109A0000B74B1B68DB0700F1B48107230DE0B8F109
:109A1000010F88D1434606F11C022946384601F061
:109A200045FB00287FF47FAFFF233377A4E6B8F12E
:109A3000010F7FF478AFAB4A0123EEE7B8F1010FD5
:109A400002D1A94A3023E8E7B8F1020F7FF46BAFE7
:109A5000A549A1F11E00FFF7DDFB044600287FF4B5
:109A600062AF082333777BE6B8F1010F7FF45BAF79
:109A7000EB88002B00F07F819B4B02AA03F1300E94
:109A80001446186859689446ACE8030008337345D7
:109A90006246F6D19DF80A20B2BBB9F1830F08D017
:109AA000B9F1870F2ED0B9F1820F2BD00820307773
:109AB000CBE68E48FFF766FB10B1037B8DF80A30CA
:109AC0004FF001130121CDE904130023ADF8183044
:109AD0004FF6C043ADF8223040F29B13ADF824306E
:109AE00040F20313ADF82630814B0A93224630230F
:109AF0002946384601F0DAFA0446002800F03B8196
:109B00000023AFE70123D9E79DF80BA00192BAF13A
:109B1000000F48D17548FFF735FB019A28B9704B03
:109B20001B68DA07C2D500BEC0E70378B0F80D1095
:109B3000194401441844FFF73DFBB9F1830F8046F7
:109B400007D0B9F1870F19D0B9F1820FAED1012238
:109B500000E002798DF80B2098F800004044FFF7F0
:109B600043FB98F80230042B11D0062B9ED1B0F89D
:109B70000520B0F8073053431B0110E08378042B15
:109B800003D0062B92D18279E4E7827DE2E7B0F838
:109B90000730B0F805205A4398F815305343DB08D6
:109BA000CDF81A30A2E7DDF80C80B8F1000F9DD196
:109BB0004E48FFF7E7FA019A0028B0D00378B0F8D2
:109BC0000D10194401441844FFF7F4FA0378524683
:109BD0001844A9F18209FFF707FBB9F1050F3FF619
:109BE00065AF01A353F829F0359C0200019C0200E7
:109BF0005D9C0200AD9A0200AD9A02004F9C0200EB
:109C0000437EA3B1053300EB8303D3F80280D0F881
:109C10001A3042F21072B3FBF2F3CDF80C80B8F1B7
:109C2000000F22D1ADF81E80ADF820805EE7D0F89D
:109C30001E80ECE7437E3BB1053300EB8303D3F892
:109C40000230D0F81A80E4E7D0F81E30F9E7D0F8F7
:109C5000158042F21073B8FBF3F3DEE7437E13B9CD
:109C6000D0F82280F5E70023D7E7DDF81A2043B9C2
:109C7000931CB3F5807F28BF4FF48073CDF81E305E
:109C800034E7013A1A44B2FBF3F30233F1E7B8F1D7
:109C9000010F7FF448AEEB88012B7FF4C5AE43463D
:109CA000144ABAE66B78852B4ED00DD8012B23D001
:109CB000812B7FF4A5AEB8F1010F7FF434AEEB88B1
:109CC000002B7FF4BEAEAFE6862B7FF499AEB8F1E1
:109CD000010F7FF428AEEB88012B7FF4A5AEDFE700
:109CE000F0ED00E0AB590B00DA760020BC760020E6
:109CF00001010008AC590B00B8F1010F3FF4A1AE0F
:109D0000B8F1020F7FF40FAE1C49A1F11E00FFF75E
:109D100081FA044600283FF4A4AE736BB361184B7C
:109D20003BB1164A71783078AFF3008000287FF499
:109D3000FAAD0023C6E9033373610223A6F850305D
:109D40004FF48073B3830BE5B8F1010F7FF4EBADF3
:109D5000EB88022B7FF468AE3022ADF8082029464C
:109D600002AA384601F0A2F9044600287FF4C8AEE2
:109D70005AE600BE49E6FF2099E600BFDA760020E9
:109D800000000000F8B51E4C2389054683B32778F0
:109D9000DFF878C00B2606FB07C6366833449E788A
:109DA0008E4225D1D4E904329A4215D200F0FAFC51
:109DB00018B32046FFF7CCFA04F1500283B23146C3
:109DC000284600F00FFD08B1012017E00D4B1B687D
:109DD000DA0712D500BE11E00023C4E90333636142
:109DE000094B002BF0D061783846AFF30080EBE7E9
:109DF000044B1B68DB0700D500BE0020F8BD00BF88
:109E0000BC760020F0ED00E000000000B0760020FD
:109E10000A4492B291424FEA400001D8824201DBEB
:109E2000121A92B21046704738B50546D41A084641
:109E3000A988A4B29A423CBF04EB4104A4B2B4B1D5
:109E4000A14205D2914294BF531A8B189BB26B81E9
:109E5000994209D9EA882968C2F30E0202FB03116C
:109E600086F0F4F8012038BD5B1A9BB2F0E720467B
:109E7000F9E7930813B501EB8303044699420BD12C
:109E800012F0030206D0002301A8019386F0DEF849
:109E9000019B236002B010BD51F8040B2060EDE778
:109EA0002DE9F04385B08588BDF830401E1BB6B261
:109EB000A3423CBF06EB4506B6B280460F4666B3EA
:109EC000B54206D29D4294BF5C1BEC18A4B24481FB
:109ED0002E46964228BF1646A54222D9B8F806005B
:109EE0009DF83430D8F80010A5EB0409751BC0F3B9
:109EF0000E0225441FFA89FC15FB02F519FB02F935
:109F0000012B1FFA89F9ADB202FB041116D0664588
:109F10000AD87243384686F099F8304605B0BDE855
:109F2000F083641BA4B2D7E74A46384686F08EF821
:109F3000D8F800102A4607EB0900ECE7664506D87A
:109F400016FB02F292B23846FFF793FFE5E729F0DD
:109F50000304A4B2224638460191FFF78AFF19F0A4
:109F6000030929D0C9F104039BB2AB42019928BF70
:109F70002B4600222144ED1A03A80392ADB201EB57
:109F800009040246A1420DD1D8F8001009F1FF39A9
:109F900091440B4499420AD1039B3B60002DBCD0F5
:109FA0002A46D0E711F801CB00F801CBEAE711F817
:109FB000012B09F8012FEDE7D8F80010EEE77FB587
:109FC000044600690D461E4628B14FF0FF3103924A
:109FD0006EF0D2FC039A2389618989B2CDE900161B
:109FE0009BB229462046FFF75BFF61890246054682
:109FF00089B2A088FFF70CFF6081206920B100239F
:10A000001A4619466EF04CFB284604B070BD13B5D5
:10A01000930800EB8303984209D112F0030204D0A5
:10A020000B68019301A986F011F802B010BD0C680D
:10A0300040F8044BEFE72DE9FF470646C0680F469E
:10A040001546984618B14FF0FF316EF095FCF37944
:10A05000B6F808907189B488DB091FFA89F989B2CA
:10A060001CD1894536BFC1EB4401A9EB010149442C
:10A0700089B2A14236BF611A002189B28D4228BF40
:10A080000D46002D55D1F06820B100231A4619461F
:10A090006EF006FB284604B0BDE8F087A5420BD35E
:10A0A000B8F1000F05D1F3882D1BC3F30E0303FB9A
:10A0B000057789462546E4E789454FEA440236BFDD
:10A0C000531AA9EB01034B449BB22B449342D8DBB8
:10A0D000621B92B22046FFF79BFE8146D1E7ACEBB4
:10A0E00004001FFA80FCA445F9D2F2883068A4EB82
:10A0F0000C0A2C1BC2F30E0364441FFA8AF114FBF2
:10A1000003F41AFB03FAB8F1010F1A461FFA8AFA90
:10A11000A4B203FB0C0017D08D420CD86A43394619
:10A1200085F094FFB0882A464946FFF771FE3081DA
:10A13000A9E7CC46D7E75246394685F087FF306815
:10A14000224607EB0A01EBE78D4206D815FB03F226
:10A1500092B23946FFF75BFFE4E72AF003081FFAE3
:10A1600088F8424639460190FFF751FF1AF0030A7A
:10A170002BD0CAF104039BB2A34201983A68039220
:10A1800028BF2346E41A08F1FF380DF10C0CA4B2E5
:10A190004044514662460139C9B2FF290BD13068AB
:10A1A00092440AEB0301421E514509D11844002C88
:10A1B000B8D02246CDE71CF801EB00F801EFEAE742
:10A1C0001AF801CB02F801CFEEE73068EFE7B2F5FD
:10A1D000004FF8B504460F4616461D4626D8C068FF
:10A1E00018B14FF0FF316EF0C7FB206918B14FF086
:10A1F000FF316EF0C1FB9DF81830E0682760C5F3B1
:10A200000E0545EAC33500236381A680E5802381DE
:10A2100018B11A4619466EF043FA206920B100239E
:10A220001A4619466EF03CFA012000E00020F8BD05
:10A230000389428981889BB292B2934236BFC2EBB6
:10A2400041029B1A9B1898B2884228BF0846704763
:10A250000289438992B29BB2D31A5842584170473F
:10A260008288038940899BB280B2834236BFC0EBAB
:10A270004200181AC01880B2824286BF101A80B2FB
:10A28000002070470023FFF79ABE38B504460069E6
:10A290000D4618B14FF0FF316EF06EFB22896389D5
:10A2A00029469BB292B22046FFF7BEFD05462069C3
:10A2B00020B100231A4619466EF0F2F9284638BD3F
:10A2C00012B10023FFF7B7BE1046704710B5044621
:10A2D000C06818B14FF0FF316EF04EFB206918B125
:10A2E0004FF0FF316EF048FBE0680023638123816B
:10A2F00018B11A4619466EF0D3F9206920B100232F
:10A300001A4619466EF0CCF9012010BD38B5044646
:10A31000C0680D4618B14FF0FF316EF02DFB20697B
:10A3200018B14FF0FF316EF027FBE379E06865F379
:10A33000C713E37120B100231A4619466EF0B0F935
:10A34000206920B100231A4619466EF0A9F90120B0
:10A3500038BD00002DE9F041184D194E194F8046C7
:10A3600000242978E3B24A1D9A4210DA38220021EB
:10A37000154885F093FE1022FF21144885F08EFECB
:10A38000BDE8F04112481222FF2185F087BE9942B4
:10A390004FF018020AD9396802FB03134BB90D4B71
:10A3A0001B68DB0700D500BEBDE8F0815B1A02FB2D
:10A3B00003635B68404698470134D2E71078002079
:10A3C000B8590B000C7800206478002068780020D1
:10A3D00078780020F0ED00E037B50C4605460868B7
:10A3E000019200F0A3FE2368019A0121284603B0E0
:10A3F000BDE8304018477047024B5878003818BF06
:10A400000120704764780020024B1878C0F3800068
:10A41000704700BF64780020024B1878FF3818BFDF
:10A4200001207047146100202DE9F743314E337845
:10A43000FF2B054644D1382200212F4885F02EFEFF
:10A440002E4901206EF0B0F92D4B186040B92D4B0C
:10A450001B6813F0010F4AD1002003B0BDE8F08360
:10A46000294F3B46002233F80C0B00927A6879881A
:10A470006EF0DAF8B96804466EF02CFB234B1C60D2
:10A480002CB9204B1B68DB07E6D500BEE4E7204B68
:10A4900023B12048AFF300801F4B18601D4FDFF839
:10A4A0007C80DFF8749000243A78E0B2531D834238
:10A4B00008DA2846357000F0C6FF284600F0C4FFD1
:10A4C0000120CAE782424FF0180309D9D9F80020C9
:10A4D00003FB002038B90B4A126812F0010FBAE7EB
:10A4E000801A03FB0080036898470134DCE700BE54
:10A4F000B3E700BF146100206478002014780020C6
:10A500009C780020F0ED00E0B8600020A0780020EA
:10A5100000000000107800200C780020B8590B00D3
:10A520002DE9FF414378023B04460D46042B13D826
:10A53000DFE803F00333222A88004F4B1A786FF3C9
:10A5400000021A701A7800216FF341021A705970D4
:10A550001A7861F382021A70484B1868002D77D17F
:10A560002B464FF0FF3221466EF09AF86178207842
:10A570002A46FFF740FF3CE03F4B1A78D00738D51A
:10A580001A7842F00402E6E73B4A1378D90730D53F
:10A5900013786FF382031370DEE7374A13785B0793
:10A5A0001DD513786FF38203137002780023CDE971
:10A5B00001338DF8042005228DF805202F4A0393DE
:10A5C0001068C9B90B464FF0FF3201A96EF068F868
:10A5D0009DF805109DF804002A46FFF70CFF284E51
:10A5E000284FDFF8A88000253178EBB24A1D9A4247
:10A5F00014DA04B0BDE8F0816A4601A900936EF058
:10A60000E8F8009B002BE3D01F4B4FF080525A60BC
:10A6100040BFBFF34F8FBFF36F8FD9E799424FF021
:10A6200018020BD9D8F8001002FB031323B15B69A1
:10A6300013B16168207898470135D5E75B1A02FBB2
:10A640000373F4E70C4AD3780133DBB2D37083E7AA
:10A65000002301AA214601936EF0BBF8019B002B59
:10A6600084D0094B4FF080525A6040BFBFF34F8FE8
:10A67000BFF36F8F7AE700BF64780020A0780020D6
:10A6800010780020B8590B0000ED00E00C78002095
:10A690001FB5CDE90201154908240023019308687C
:10A6A0008DF80540144672B9134601A94FF0FF32E8
:10A6B0006DF0F6FF9DF805109DF804002246FFF7A7
:10A6C0009AFE04B010BD6A4601A900936EF081F8AD
:10A6D000009B002BEED0064B4FF080525A6040BFDB
:10A6E000BFF34F8FBFF36F8FE4E700BFA078002068
:10A6F00000ED00E038B58B7803F07F03082B0C46A3
:10A7000006D90B4B1B68DB0700D500BE002038BD07
:10A71000084B1D78084B2046997801F023FC00284F
:10A72000EFD021462846BDE8384000F0A5BE00BF66
:10A73000F0ED00E014610020647800202DE9F0477E
:10A74000DDE9085681460C4690469A460027B845F2
:10A7500001DC01200CE06378052B04D1E37803F0E1
:10A760000303534508D00E4B1B68DA0702D40020C0
:10A77000BDE8F08700BEFAE721464846FFF7BAFF7A
:10A7800028B9074B1B68DB07F1D500BEF0E7A378BB
:10A79000DA0914BF33702B70237801371C44D6E7D5
:10A7A000F0ED00E0CB0901F07F00263303EB40031E
:10A7B000024A03481168184401F08CBB9C780020C1
:10A7C00064780020CB0901F07F00263303EB4003BF
:10A7D000024A03481168184401F0A5BB9C78002088
:10A7E00064780020154838B501F07F0500EB45007E
:10A7F00000EBD1142034A079C00707D5104B1B689B
:10A80000DA0701D4002038BD00BEFBE7A07940F094
:10A810000100A0710B48007800F060FF0028F2D121
:10A82000A37960F30003A371A37960F38203A3719A
:10A83000034B1B68DB07E5D500BEE4E76478002026
:10A84000F0ED00E014610020054B01F07F0203EB06
:10A85000420303EBD11191F8260000F0010070478C
:10A860006478002010B50C4B01F07F0203EB42032B
:10A8700003EBD1142034A3799B070BD4074B187832
:10A8800000F0A4FFA37943F00203A371A37943F07E
:10A890000103A37110BD00BF647800201461002083
:10A8A00010B50C4B01F07F0203EB420303EBD11414
:10A8B0002034A3799B070BD5074B187800F0AAFF2B
:10A8C000A3796FF34103A371A3796FF30003A3711D
:10A8D00010BD00BF64780020146100202DE9F04F06
:10A8E000A14B1B78FF2B8BB0834600F00A834FF4FB
:10A8F0007A72002380024FEA9B5184F0B1FD012857
:10A9000038BF01200490994BBBF1FF3F18681BD062
:10A91000049BBBF1000F14BF1A46002207A96DF07B
:10A92000B1FF002800F0ED829DF81D30013B072BA0
:10A9300000F21C83DFE813F00A001B001A03F80280
:10A9400007032700B60213035A46E7E79DF81C00E9
:10A95000FFF700FD00F0E2FB854B9DF820209A7088
:10A96000824B18686EF09EF80028CCD1C9E29DF8A1
:10A970001C00FFF7EFFC00F0D1FB7E4B002BEFD06B
:10A98000AFF30080ECE77A4CE378013BDBB2E37095
:10A99000E378A04603F0FF00002BE1D123789DF877
:10A9A0001C5043F00103237094F8263060F3000339
:10A9B00084F8263094F8263060F3820384F8263039
:10A9C00094F8273060F3000384F8273094F8273098
:10A9D00060F3820384F8273000F0A8FB9DF8202064
:10A9E00002F06003602B06D1634B1B68DC0740F16B
:10A9F0001B8200BE18E2402B0DD16048002800F0F9
:10AA0000138200F093FB08AA01212846FDF7E2F823
:10AA10000028A5D108E202F01F02012A00F08C8173
:10AA2000022A00F0BF81002ADED1202B22D19DF81E
:10AA300024300F2B00F2F8811C44514B21791B78F4
:10AA400099420DD24F4B1B6801EB410113EBC10141
:10AA500000F0EA8108AA0C312846FFF7BDFCD7E7D1
:10AA60005A1D8A42C0F2E081474AC91A182303FBE3
:10AA70000121EFE7002BB7D19DF82130092BB3D886
:10AA800001A252F823F000BF23AD020011AD020075
:10AA9000E9A90200FDAC0200E9A90200B1AA020086
:10AAA0006BAC0200E9A90200CBAA0200E1AA0200F5
:10AAB00008A800F041FB9DF82210284600F0CAFCCF
:10AAC000237843F0020323704AE763788DF81A3045
:10AAD00001230DF11A0208A9284600F0E7FA3FE722
:10AAE0009DF822300193019A63789A4234D06378BA
:10AAF0003BB1284600F04AFDA6782846FFF72AFC1D
:10AB0000A670019B002B00F0A980581EC0B2FCF774
:10AB1000E1FE10B14378022B06D0174B1B68DF070C
:10AB20007FF562AF00BE5FE7C379C3F38012C3F362
:10AB300040131B0143EA4213227822F030021343F0
:10AB400023704388C31800F109060393039BB342A3
:10AB50001ED80E4B002B7ED1019B637008A928469E
:10AB600000F08CFAFCE600BF14610020A078002001
:10AB70006478002000000000F0ED00E0D57B0200CA
:10AB8000107800200C780020B8590B00000000005D
:10AB900073780B2B03BF337896F80380F6184FF0C9
:10ABA00001087378042BB8D1039B9A1B92B200233F
:10ABB0000293B14B9DF808701B78591D8F42ACDC95
:10ABC000BB424FF0180933D9AC4B1B6809FB07395E
:10ABD000B9F1000FA1D0D9F80830059231462846C6
:10ABE00098470828059A824632D9824230D3B8F174
:10ABF000010F0BD1D9F80830A14A934208BF4FF09A
:10AC00000208A04A934208BF4FF002089E49002262
:10AC1000D0B2804511D83B4631469C48524601F09F
:10AC2000D1F9954B1B7805339F4256448EDD74E76E
:10AC30009749FB1A09FB0319CDE7B378034451FA8E
:10AC400083F301321879FF287FF467AF1F71DFE7C4
:10AC5000029B0133ACE7AFF300807DE78D4B002B07
:10AC60003FF47AAFAFF3008076E7BDF82200030A25
:10AC70005A1EC0B20E2A00F2D780DFE802F0081D8B
:10AC80002ED5D5381DD5D5D5D5D5D5D51100FCF7C0
:10AC90001DFE1223024608A9284600F007FAB7E66F
:10ACA0007D4B002B00F0C080FCF790FF024600288F
:10ACB0003FF49AAE4388EEE7022B07D1FCF70AFE79
:10ACC00000283FF491AE43880246E4E7734B002B23
:10ACD00000F0AA80AFF30080F2E7BDF82410FCF783
:10ACE000FFFD0246002800F09F800378D3E76C4BFD
:10ACF000002B00F09980AFF30080F2E7BDF822301E
:10AD0000012B40F09180237843F00803237025E75E
:10AD1000BDF82230012B40F0878023786FF3C30306
:10AD2000F4E72378C3F340129B0803F002031343B4
:10AD3000ADF81A300223CCE69DF824300F2B73D8DF
:10AD40001C444D4B21791B78994222D24B4B1B68F6
:10AD500001EB410113EBC10166D008AA0C31284672
:10AD6000FFF73AFB00287FF4FBAD9DF8203013F08D
:10AD7000600459D19DF821300A3B012B54D800F0D2
:10AD8000D5F99DF821300A2B7FF4E8AE8DF81A40F2
:10AD90009EE65A1D8A4247DB3D4AC91A182303FB27
:10ADA0000121DAE79DF8241001F07F06082E3FF616
:10ADB0001BAE720004EB4606DFF8BCC006EBD116F2
:10ADC0009CF800C0367D66454FEAD11018D206EBDC
:10ADD000460C2A4E366806EBCC061BBB9DF821308C
:10ADE00003F0FD0CBCF1010F29D0002B7FF4FCAD6A
:10ADF00008EB0207384490F82630C3F3400397E786
:10AE00000CF1050EB645C0F2B880214FA6EB0C063A
:10AE10004FF0180C0CFB0676002BDFD008AA06F1C9
:10AE20000C0119E6002EF9D19DF81C00002100F05C
:10AE3000CDFC9DF81C00802100F0C8FC90E5BDF819
:10AE4000222022B9012B284613D1FFF729FD002E1D
:10AE50003FF486AD06F10C0108AA2846FFF7BCFABC
:10AE6000002000F063F994F82730DE073FF578AD55
:10AE700074E6FFF7F7FCEAE7107800200C78002072
:10AE8000A97E0200CD850200647800207878002039
:10AE9000B8590B0000000000CD7B0200000000004C
:10AEA000000000009DF82010364B01F07F0403EBFA
:10AEB000440303EBD11393F826006FF3000083F8EB
:10AEC000260093F826006FF3820083F826003CB931
:10AED000099B9DF821209DF81C0000F03BF93FE5FF
:10AEE000294A1B7D127893420ED2284A126803EB3E
:10AEF000430312EBC3030FD1254B1B68D80700D5C2
:10AF000000BE0BB0BDE8F08F501D9842F4DB214825
:10AF10009B1A182202FB03031C699DF82120099B40
:10AF20009DF81C00A0471BE5164B1A78D1077FF54A
:10AF300017AD194A002A3FF413AD1878C0F3C000CA
:10AF4000AFF300800CE50F4B1B78DA077FF508ADF7
:10AF5000124B002B3FF404ADAFF3008000E5089BDB
:10AF6000002B3FF4FDAC09989847F9E4084B1B68A7
:10AF7000DB077FF5F5AC00BEF2E4002B7FF454AFA5
:10AF80001E462BE764780020107800200C78002003
:10AF9000F0ED00E0B8590B000000000000000000D8
:10AFA000054B01F07F0203EB420303EBD11191F853
:10AFB0002600C0F34000704764780020134B10B5A2
:10AFC0000C462BB9124B1B68DB0700D500BE10BD29
:10AFD000104B187800F024FB0F4B04F07F0103EBBB
:10AFE000410303EBD41191F826306FF3410381F84C
:10AFF000263091F826306FF3000381F8263091F85F
:10B0000026306FF3820381F82630E0E721B6020094
:10B01000F0ED00E0146100206478002037B5144999
:10B020000446CA89888991F90050831A9BB2402B43
:10B0300028BF4023002D10DA904214D01A468968A8
:10B040000C48019385F002F80A4A019B80212046B2
:10B0500003B0BDE83040FFF7C5BB90424FF00001A0
:10B0600003D10022F3E78021FBE7024AEFE700BFAC
:10B0700064790020787900207047000030B40A4CD1
:10B0800005460A4608684968234603C392F900202A
:10B0900000239A42C4E9023328461A4630BCACBFAA
:10B0A00080211946FFF79EBB64790020F8B5194E40
:10B0B0000C46054608684968B260374603C7002158
:10B0C000F181E1888B4228BF0B46B38179B143B14E
:10B0D0003AB9114B1B68DA0701D40020F8BD00BE55
:10B0E000FBE72846FFF79AFF68B10120F6E794F9DD
:10B0F0000030002B0A460B462846ACBF80210021B9
:10B10000FFF770FBF0E7044B1B68DB07E5D500BEDB
:10B11000E4E700BF64790020F0ED00E0024814226B
:10B12000002184F0BBBF00BF64790020014B18618F
:10B13000704700BF6479002010B50246044C0068D7
:10B140005168234603C30023C4E9023310BD00BF86
:10B1500064790020F8B52F4F1E463B78C909B1EB42
:10B16000D31F05463C4614D03EB12B4B1B68DA0773
:10B1700001D40020F8BD00BEFBE73946FFF77CFF95
:10B180003B690BB90120F5E73A4603212846984769
:10B19000F8E797F90030002B06DBB8680028E8D004
:10B1A0001E49324684F052FFA268E3893244334498
:10B1B000A260E2889BB29A42E38101D03F2E24D85C
:10B1C00023699BB994F90030002B4FF000031A4615
:10B1D000ACBF802119462846FFF704FB0028D1D1D7
:10B1E0000D4B1B68DB07C4D500BEC3E70221094A2B
:10B1F0002846984701460028E4D1284600F0E6FAA0
:10B200008021284600F0E2FABCE72846FFF706FF57
:10B21000E4E700BF64790020F0ED00E078790020D9
:10B22000064B1868043B1B68082B04D103288CBF0D
:10B230000020012070470020704700BF340100103B
:10B2400042DF704743DF704744DF704712DF7047CB
:10B2500043F2040307B51A68094B9A424FF0000005
:10B260000AD18DF807000DF10700FFF7EFFF9DF8F9
:10B270000700003818BF012003B05DF804FB00BFD1
:10B28000DBE5B15101230360BFF36F8FBFF34F8F35
:10B29000074B984202D0043B984207D1BFF35B8F23
:10B2A000044B002283F82021BFF35B8F704700BF5F
:10B2B00050700240B879002010B40E4BBFF35B8F82
:10B2C00001464FF00104D3E84F2FC3E84C4FBCF1C7
:10B2D000000FF8D1BFF35B8F12F0FF0F05D00648C7
:10B2E0005DF8044B0122FFF7D3B95DF8044BFFF77B
:10B2F000C9BF00BFD87A0020B9B202000D4B03EBE2
:10B300004013D98A9A8A521A198B92B28A4228BF5C
:10B310000A4619691423434303F1804303F51C33A0
:10B32000C3F80016C3F80426034B03EB8000FFF7B5
:10B33000C3BF00BFB879002004700240F0B42C4AAB
:10B34000BFF35B8F02F590734FF00104D3E84F1FFA
:10B35000C3E8454F002DF9D1BFF35B8F11F0FF0F0C
:10B3600014460BD0234B5A68C2F30802003A014638
:10B37000F0BC214818BF0122FFF78AB908281F49ED
:10B380001AD1D1F8C034D80308D5BFF35B8F00239E
:10B3900084F82031BFF35B8FF0BC704792F80B014B
:10B3A0000028F2D0D2F800211548C1F8A027C1F832
:10B3B000A437F0BCFFF766BF02EB401500F59473AD
:10B3C000460151F82340EF88AB88DB1B9BB2A4B247
:10B3D000A34228BF23469459142202FB0011C1F84E
:10B3E0000047C1F80437074B03EB8000E1E700BFDB
:10B3F000B879002000ED00E009B4020000700240BE
:10B400004870024028700240C0B2FFF797BF07B5EE
:10B41000FFF71EFF58B1002301A80193FFF714FFA7
:10B420000198003818BF012003B05DF804FB4FF00D
:10B430008043D3F80C24D3F80C0410F4803018BFE8
:10B4400002F00100F0E77047014B80225A6070471C
:10B4500000E100E0074BD3F80014D3F800240A43BE
:10B46000C3F800240022C3F858214FF48002C3F827
:10B47000042370470070024070B58A788E883F4C74
:10B48000C97802F07F03580000EBD21004EB0010E3
:10B4900001F00301C6F30A0601294FEAD21506811D
:10B4A00029D00120364900FA03F4D5B903F10C067E
:10B4B000B040C1F80403D1F8140503F59473204398
:10B4C000C1F8140541F823502D4BC3F8182542F458
:10B4D0008072C3F80C25BFF36F8FBFF34F8F01202D
:10B4E00012E002339840C1F80403D1F81035234329
:10B4F000C1F81035E8E7082B07D0224B186810F088
:10B50000010001D000BE002070BD1D4BDDB9B4F8B4
:10B51000182112B18022C3F81C250022C3F8502143
:10B52000D3F8002312F4001208BFC3F85421144BBF
:10B530004FF44012C3F80423D3F8142542F4807268
:10B54000C3F81425C7E70022C3F82C21B4F808215A
:10B5500012B18022C3F81C25094BD3F8002312F442
:10B56000001208BFC3F85421074AC3F80423D3F8D4
:10B57000102542F48072C3F81025ACE7B87900209A
:10B5800000700240F0ED00E0000820001F4B802218
:10B590002DE9F041C3F88420BFF34F8FBFF36F8FC5
:10B5A00001241B4DDFF87480274604F10C03A21C14
:10B5B00007FA02F207FA03F31343C5F80833A300AE
:10B5C00003F1804303F51C3300265E6008EB441052
:10B5D0009E6220223146013484F060FD082CE4D1C3
:10B5E0000C4BC5F808332022C5F81C6531466E6245
:10B5F0000948AE6484F052FDC5F81475C5F810759D
:10B60000024B80225A60BDE8F08100BF00E100E0FB
:10B610000070024000083000B87A0020B87900209D
:10B6200070B501F07F05082D2A4B2B4C4FEAD11144
:10B6300023D0012202FA05F0C043A1B905F10C069E
:10B64000B240C3F80823D3F814251040C3F81405FA
:10B6500001EB450104EB01110023CB72BFF36F8FA7
:10B66000BFF34F8F70BDAE1CB240C3F80823D3F8B0
:10B6700010251040C3F81005EAE704EB0112002082
:10B68000A2F80801D1B94FF48012C3F80823D3F807
:10B69000142522F48072C3F81425C3F850110D4B01
:10B6A000B4F808010022C3F81C25B4F81821C242DE
:10B6B00004BF4FF40012C3F80823C9E74FF4006237
:10B6C000C3F80823D3F8102522F48072C3F810259C
:10B6D000E5E700BF00700240B87900202DE9FF4186
:10B6E00001F07F00334F0E461C46430003EBD61398
:10B6F0004FEA031807EB0313C90993F80BC03D4643
:10B700000CF0FF0EBCF1000F0AD02B4B1B6813F09E
:10B71000010301D000BE0023184604B0BDE8F0814B
:10B7200047F808209C80A3F806E008BB04BB234B25
:10B73000D3F88034C3F3C0138B4219D02048FFF7ED
:10B74000BBFD204B59680394C1F3080100394FF445
:10B75000E06318BF012101A8CDE90144ADF8043030
:10B760008DF808608DF80940FEF7DAFE0123D3E773
:10B770000124D9B905EB4012D47220B91248FFF761
:10B780009BFD2346C8E7BFF36F8FBFF34F8F957ABA
:10B7900005F0FF03002DF4D0D47A04F0FF05002C4F
:10B7A000BAD09172FFF7CAFD2B46B5E7FFF7A6FDA9
:10B7B000E7E700BFB8790020F0ED00E0007002403C
:10B7C0005070024000ED00E04C70024011F07F002C
:10B7D00008B507D10D4B01225A65BFF36F8FBFF338
:10B7E0004F8F08BD0828F8D0084B41F48072C90972
:10B7F000C3F81825F1D1064B03EB40139A7A002ABF
:10B80000EBD09972FFF79AFDE7E700BF00700240A6
:10B81000B879002011F0770F12D00A4B41F48072F2
:10B82000C3F80C15C3F80C25CA09C3F8181504BFD2
:10B8300001F5947143F82120BFF36F8FBFF34F8F51
:10B84000704700BF0070024008B5184B012200216C
:10B85000C3F81425C3F810250A468B0003F1804372
:10B8600003F51C33013108295A609A62F5D10F4B58
:10B870005A629A64C3F85821D3F80014D3F800240C
:10B880000A43C3F80024D3F80023C3F80823084A66
:10B89000C3F80423074B4FF492720021184684F03A
:10B8A000FDFB40220283028108BD00BF0070024000
:10B8B0000514C001B87900202DE9F04FB14BB24A10
:10B8C000D3F80013002385B01C4601201D4621FA41
:10B8D00003F6F6070BD552F8236046B100FA03F6DB
:10B8E000344342F82350BFF36F8FBFF34F8F0133C0
:10B8F000192BECD1E7070FD5FFF7A6FF00234FF474
:10B900008072012101A8CDE901330393ADF8042031
:10B910008DF80830FEF704FE14F4006F9B4D08D03C
:10B92000984BD3F8A8369BB2A5F81631012385F8B9
:10B930001C31A60204F4800736D5924ED6F8143591
:10B9400013F4807308D01FB1D6F80034D80702D49E
:10B950000820FFF7F3FC0123D6F81025D10540F1AC
:10B960005C8195F81C319BB1B5F8163100229BB271
:10B97000CDE9012285F81C2103934FF4E06288236E
:10B98000012101A8ADF80420ADF80830FEF7C8FD8C
:10B990000023CDE90133039301214FF4407301A843
:10B9A000ADF80430FEF7BCFD002F37D0754BD3F84F
:10B9B000006440F201723240C3F80024F2050DD554
:10B9C0000121C3F82C150023CDE90133039301A80D
:10B9D0004FF48063ADF80430FEF7A2FD77050FD574
:10B9E000684B0122C3F808259A65D3F8002312F4A6
:10B9F000001208BFC3F854214FF40012C3F8042307
:10BA0000B0050BD50023CDE90133039301214FF499
:10BA1000A06301A8ADF80430FEF782FD21023BD5FA
:10BA2000584BD3F880E4D3F88424D3F88814D3F89F
:10BA30008C74D3F89064D3F894045FFA81FCD3F843
:10BA40009814D3F89C341EF07F0F5FFA8EF8D2B2B0
:10BA5000FFB2F6B2C0B2C9B2DBB201D1052A1BD027
:10BA60004FF0000EADF806E08DF80D004FF4C06EFB
:10BA70008DF80E1001A80121ADF804E08DF80880C2
:10BA80008DF809208DF80AC08DF80B708DF80C60C8
:10BA90008DF80F30FEF744FD3D4B23406BB1BFF3F3
:10BAA0005B8F95F82031BFF35B8F002B40F0BD809A
:10BAB000384B1B68DA0700D500BEDFF8D080DFF80E
:10BAC000C490DFF8D8B0474600264FF0140A06F1BC
:10BAD0000C0324FA03F3DB07F1B224D50AFB069327
:10BAE0003A68D3F8083705EB461C12FA83F23A603D
:10BAF000BCF806E098B273449BB2082E4FEA461297
:10BB0000ACF8063000F099803B89834240F0958084
:10BB1000BCF80630B8889BB2984240F28E8011B9CA
:10BB20005846FFF7C9FB0136092E07F12007CED191
:10BB3000194B2340002B00F08880124BD3F86C7413
:10BB4000C3F86C74BFF36F8FBFF34F8F14F480642E
:10BB500008D0D3F88044D3F880341906C4F3C01455
:10BB600040F18C804FF00009DFF818A000264FF05C
:10BB7000140B27FA06F3DA07F0B211D456BB4CB314
:10BB80000EE000BF0070024000710240B879002052
:10BB9000FCFB1F00F0ED00E0000400014C700240CF
:10BBA0000BFB06A3D8F81020D3F8083652FA83F21C
:10BBB000C8F8102005EB4612D18A89B251FA83F3F6
:10BBC0009BB2D382D38AB8F814109BB2994258D949
:10BBD000FFF794FB0136082E08F12008C9D1002494
:10BBE000012604F1100327FA03F3DB07E0B203D4C4
:10BBF0007CB9B9F1000F0CD005EB44116301CA7A8E
:10BC0000002A53D0CA88898892B291424ED9FFF750
:10BC100095FB0134082CE4D117E0002B7FF4B8AE7B
:10BC20004FF40013C6F80833B2E60023BFF35B8F6E
:10BC300085F82031BFF35B8F3FE72A44D37A3BB9C5
:10BC40001C4B1B68D80700D500BE05B0BDE8F08FBF
:10BC5000D388BB800023D372D2884FF4E060CDE953
:10BC6000013392B2ADF804008DF8081001A801214B
:10BC700003928DF80930FEF753FC54E74FF00109A9
:10BC800072E7D28A00234FF4E06160F07F00CDE9D3
:10BC9000013392B2ADF804108DF80800012101A81B
:10BCA00003928DF80930FEF73BFC93E72B449E721C
:10BCB000AFE700BFF0ED00E001287FB5044600F0DB
:10BCC000B880022853D0002842D1764BD3F8002503
:10BCD000002A3DD14FF48002C3F808234FF40062DC
:10BCE000C3F80024BFF36F8FBFF34F8F6E4B1B68F9
:10BCF000082B10D16D4B1B68032B0CD86C4AD35CFE
:10BD00004BB16C4B6C4A1868032118BB49F2753073
:10BD1000186011601860FFF783FA48B1654B674AF5
:10BD20001868C021C0B949F27530186011601860F8
:10BD30005C4B0124C3F80045BFF36F8FBFF34F8FF7
:10BD4000FFF765FB20B9FFF783FA38B1FFF778FA00
:10BD500004B070BD1160DEE71160E9E7584B186070
:10BD60001B680193019B4FF080431C60F0E74D4C32
:10BD7000D4F804351BB1FFF74AFB0028E8D1D4F80A
:10BD800000341B05FBD54FF40063C4F80034BFF347
:10BD90006F8FBFF34F8FFFF743FA48B1454B474AC8
:10BDA000186800283FD149F2753119601060196098
:10BDB0003D4B1B68082B0FD13C4B1B68032B0BD84A
:10BDC0003B4AD35C43B13B4B3B4A186870BB49F2DA
:10BDD0007531196010601960FFF722FA48B1394BCC
:10BDE00040F2E3721A6040225A60BFF36F8FBFF3D4
:10BDF0004F8F2C4C344E80250123C4F81C55C4F8B9
:10BE00000433C6F88451FEF707FB00B17560FFF7F5
:10BE1000FEFA0028FBD00123C4F80435BFF36F8F6E
:10BE2000BFF34F8F94E700231360C1E70023136033
:10BE3000D2E71C4BD3F80025002A89D00022C3F892
:10BE40000425BFF36F8FBFF34F8F1F498020C1F8C8
:10BE50008400BFF34F8FBFF36F8FD3F80013C3F885
:10BE60000813C3F80025BFF36F8FBFF34F8FFFF7A1
:10BE7000EFF9A0B1FFF7E6F9144B5968C1F30801D7
:10BE800000230039CDE90133039318BF01214FF49A
:10BE9000007301A8ADF80430FEF742FB58E70C4BE5
:10BEA0001C60E9E70070024030010010340100100E
:10BEB000485A0B0000EC064014ED064014EC064016
:10BEC000000100400078024000E100E000ED00E0E9
:10BED00004000040F8B5047814F0010405460E464D
:10BEE0001FD103785A07C3F3800716D44FF0FF31F0
:10BEF00030466CF041FD2C7814F001040FD12B7802
:10BF00005B0704D42B7843F004032B700124002337
:10BF10001A46194630466CF0C3FB2046F8BD3C4635
:10BF2000F5E70024F9E770B504460D4628464FF0C2
:10BF3000FF316CF021FD2378C3F380065B0708D541
:10BF4000237813F0010203BF237862F38203237086
:10BF5000002600231A46194628466CF0A1FB3046FD
:10BF600070BD00008388C07800F003000228C3F38E
:10BF70000A0313D003281BD001280DD1022940F257
:10BF8000FF3208BF4FF480629A420DD20C4B186802
:10BF900010F0010008D000BE00207047022904D133
:10BFA000B3F5007FF2D101207047402BFBD9EDE7BC
:10BFB00002290CBF4FF4806240229A42F3D2E5E797
:10BFC000F0ED00E030B50A44914200D330BD4C782A
:10BFD000052C06D18C7804F07F0500EB4505E409BB
:10BFE0002B550C782144EFE710B5044600F07EF99C
:10BFF000002384F8E830204610BD38B590F8E850AA
:10C00000044655B9012380F8E83071F091F820B961
:10C010002046BDE8384000F06DB9284638BD90F89C
:10C02000E83010B504464BB1002380F8E83071F0D9
:10C03000B3F82046BDE8104000F077B910BD00000D
:10C040000148FFF7D1BF00BFDC7A00207FB50A6846
:10C0500003689A4206460C4602D0002004B070BD28
:10C060004FF453706CF0CCF905460028F5D00A481F
:10C0700000F064F904340023CDE901533268074924
:10C080000094331D70F0EEFE044628466CF0D4F99F
:10C09000B4FA84F04009E1E7DC7A002029BC090009
:10C0A0007FB506464FF45370CDE902230D466CF080
:10C0B000A7F9029A044610B9002004B070BD0090A0
:10C0C00003AB281D311D70F04BFF054620466CF078
:10C0D000B3F9002DF0D10398EFE70022026070471A
:10C0E00010B50446084670F0ADFF2060003818BF58
:10C0F000012010BD00220260704710B504460846BA
:10C1000070F0A0FF2060003818BF012010BD002390
:10C110000360704707B501920A46042101AB084449
:10C1200070F01AFE18B9019803B05DF804FB002006
:10C13000FAE730B5054685B04FF46370CDE90221CA
:10C140006CF05EF9044678B12B1D00930190DDE997
:10C1500002212868012370F03BFD054620466CF063
:10C160006BF9B5FA85F0400905B030BD0022012118
:10C17000C0E90021C0E902210321C0E906220161D2
:10C180000275704710B50446007D38B970F0D0FFD5
:10C1900008B901232375B0FA80F0400910BD0023CF
:10C1A000037570F0F9BF0F29084606D90B0705D0B3
:10C1B00001F0F0011031C8B27047102070472DE92E
:10C1C000F04F99B09A4602AF037D97F88480D7F874
:10C1D00090B0054689461646002B78D070F0A8FF2F
:10C1E000002877D118F0070477D1A8F11003102B9D
:10C1F00073D8AB69D7F88C105A4607F10C0070F071
:10C20000B9FBD7F88030E969C7E901383A1D08233E
:10C2100007F10C0070F0EEFB002861D1AB685B45C4
:10C220001AD128463146FFF7BEFF10F00F0305462E
:10C230001CD1EA1D22F00702ADEB020D0DF108083A
:10C240008DF808300DF10902AB1E0021002B11DB27
:10C2500002F8011B013BF9E7514607F10C0070F0B1
:10C26000EDFB0028DDD06FF006002CE0C3F11003D9
:10C27000DBB2DEE732464946404683F0E7FED7F8B8
:10C2800088002A46002183F009FFD7F88830AC42A5
:10C2900008EB0401234408D2102207F10C0070F0CF
:10C2A000E5FB00BB1034E4B2EFE7CDE90037002333
:10C2B0000A4607F10C00194670F016FC00280CBF66
:10C2C00028466FF005005C37BD46BDE8F08F4FF0A3
:10C2D000FF30F8E76FF00100F5E76FF00200F2E7DA
:10C2E0006FF00300EFE76FF00400ECE7002280F846
:10C2F000E420704770B590F8E44006469CB90123ED
:10C3000080F8E4304FF4BF506CF07AF8054650B135
:10C31000014630466FF074FE044628466CF08CF8F7
:10C32000B4FA84F46409204670BD90F8E42022B188
:10C33000002280F8E4206FF0C7BE7047704708B550
:10C3400013460A4619466FF06FFCB0FA80F04009B8
:10C3500008BD08B5012116206EF022FF002116202D
:10C360006EF086FF01210D206EF01AFF00210D20D6
:10C370006EF016FF01210C206EF012FF00210C2040
:10C380006EF00EFF01210B206EF00AFFBDE80840A1
:10C3900000210B206EF004BF0EB403B5014608481F
:10C3A00003AB006853F8042B019318B100F6A860A2
:10C3B00002F096FD02B05DF804EB03B0704700BFD9
:10C3C000407F0020002A29D0092824D8DFE800F087
:10C3D0001A172311140B0E20051D114B11480029AB
:10C3E00018BF18467047104B1048F8E7104B11481B
:10C3F000F5E7114B1148F2E7114B1248EFE7124BEA
:10C400001248ECE7124B1348E9E7134B1348E6E7F1
:10C41000134B1448E3E7144B1448E0E71248704705
:10C42000B05B0B00275B0B00A95B0B00325B0B00C2
:10C43000A25B0B003C5B0B009D5B0B00465B0B00A3
:10C44000985B0B00515B0B00925B0B005C5B0B007D
:10C450008C5B0B00655B0B00865B0B006E5B0B005F
:10C46000805B0B00785B0B00205B0B00B75B0B0065
:10C470000C289ABF024B53F820000248704700BFB7
:10C48000285C0B00BF5B0B0010B5044648B185F07B
:10C490001FF930B1204410F8010CA0F12E035842CE
:10C4A000584110BD4B6843608B688360CB68C360A4
:10C4B00010B50B6903610B7D03758B698361CB69D3
:10C4C000C3611F3100F1200300F1610211F8014F37
:10C4D00003F8014B9342F9D110BD00002DE9F04360
:10C4E000D3B00C4615463D490246002307A864F028
:10C4F000ECFF07A865F05EFA00285AD007A865F09F
:10C5000060FA002855D0002207A920A865F05CFA3F
:10C51000334FDFF8D890DFF8D88020A865F04AFACA
:10C52000002843D020A865F04AFA0378002B3DD0BC
:10C5300020A865F046FA00283ED020A865F03FFA12
:10C54000014604A86BF08AFC264939A86BF086FCEA
:10C5500039A904A86BF04AFE064639A86BF039FCED
:10C5600004A86BF036FC3EBBB4B120A83E6865F071
:10C5700026FA06F6A8661C4A03464146304602F0F3
:10C5800053FE20A865F01BFA611E2A46C9B2FFF7C8
:10C59000A5FF20A865F0A5F907A939A8002265F034
:10C5A00013FA39A920A8FFF77DFFB6E707A865F0C1
:10C5B00098F953B0BDE8F08320A83E6865F0FFF914
:10C5C000039020A865F05BF906F6A8660090039B2F
:10C5D0004A464146304602F027FEDAE71C80012039
:10C5E000407F002063720B005C5C0B00725C0B00F0
:10C5F0006C5C0B000146014864F0EBBF1C8001201D
:10C6000013B5124B124C196801A803F0C3FC4CF08F
:10C61000AFFB104867F036FA30B920680E4A0F4970
:10C6200000F6A86002F000FE20680D4A0D4900F6F1
:10C63000A86002F0F9FD00220A210B48FFF74EFF27
:10C6400001A803F0AFFC02B010BD00BF3C7F00208A
:10C65000407F00201C800120835C0B009B5C0B0052
:10C66000A15C0B006C5C0B009D180C002DE9F347DE
:10C67000D0E90087A7EB0804E310244C5C43244B6B
:10C680009C4289460646114602D122487BF0DCFDD9
:10C69000012C224638BF0122A418A9EB080533D289
:10C6A00054B19C4228BF1C46E820604301914CF0E5
:10C6B000CBF90199824600E0A246E8220AEB050088
:10C6C00083F0C4FC002D04DD2A464146504683F029
:10C6D000CBFCA7EB0907E835002F554404DD3A46AB
:10C6E0004946284683F0B2FC3D44B8F1000F02D021
:10C6F00040464CF0CDF9E82000FB04A4C6E900A5B3
:10C70000B46002B0BDE8F0871C46CDE735C2724F79
:10C71000CB3D8D00B35C0B002DE9F04FEFB09046A0
:10C72000789D0F461C46024678B102A85249002364
:10C7300064F0CBFE02A865F03DF930B102A865F0C7
:10C7400040F928B902A865F0CCF86FB0BDE8F08FC9
:10C75000002202A91BA865F037F907F1FF3A5FFA3A
:10C760008AFA1BA865F026F90028EBD01BA865F013
:10C7700026F90378002BE5D0D4E900239B1A3F4A21
:10C78000DB105343984506D80DB101232B701BA82D
:10C7900065F0A7F8D6E71BA865F011F906461BA8B7
:10C7A00065F00FF9814620B13046FFF76DFE8346F4
:10C7B00058B30021E82234A883F070FC1BA865F070
:10C7C0005EF86D901BA865F0FAF8014630B90DB11E
:10C7D00001232B701BA865F084F82EE0E42234A816
:10C7E00084F061FFE328F2D834A8FFF74DFE00285B
:10C7F000F0D1D4E90103984237D0E82234A983F07C
:10C8000025FC6368E8336360E4E734900146E02286
:10C8100035A883F043FCD6B90DB101222A701BA8BC
:10C8200065F05FF8E7B1BBF1000F19D00095234622
:10C830004246514634A8FFF76FFF02A934A80022F0
:10C8400065F0C2F834A91BA8FFF72CFE89E7E422A3
:10C85000314634A884F027FFE328DDD8CB46DEE755
:10C86000002DEAD001232B70E7E7014634AA2046C9
:10C87000FFF7FCFEAEE700BF1C80012035C2724FFF
:10C8800037B50446084611461A46069B0025C4E9FA
:10C890000055A56003B11D7000932346FFF73CFFD0
:10C8A000204603B030BD000060EEA07A0F4BDFEDF4
:10C8B000106AE0EE007A8CB0E1EE017A17EE902A71
:10C8C000A3EB620307EE103A67EEA67ADFED096A82
:10C8D00067EE877AE7EE676A67EE267A20EE270A28
:10C8E00060EEA70A21EE271A0CB0704712141F5FE2
:10C8F00012D3363FFF51D83F00B5012899B0B0EEB2
:10C90000406AB0EE605AF0EE415A33D0022856D059
:10C91000002840F0818022EE410A62EEC60A21EE34
:10C92000C51AE5EEA10AA6EE021AA5EE220AFFF745
:10C93000BBFFF0EE404A66EE607A25EEE47AE4EE64
:10C94000857AA1EE067A25EE410AB0EE671AA0EECE
:10C95000A50AF0EE470AFFF7A7FFF0EE400AB0EE97
:10C96000640A7CF083FFDFED2E7A20EE270A19B0EF
:10C970005DF804FB22EE410A62EEC60A21EEC51AFA
:10C98000E5EEA10AA6EE021AA5EE220AFFF78CFF39
:10C99000F0EE404A66EE607A25EEE47AE4EE857ABF
:10C9A000A1EE067A25EE410AB0EE671AA0EEA50ABE
:10C9B000F0EE470AFFF778FFF1EE640AD1E7B1EE37
:10C9C000404AF1EE604AF1EE413A21EE020A66EE8B
:10C9D000220A25EE211AE5EEE10AA6EE421AA5EE9C
:10C9E000620AFFF761FFB0EE406A60EEC47A26EE9D
:10C9F000637AE4EE867AA4EE017A21EE640AB0EE60
:10CA0000671AA3EEA00AF0EE470AFFF74DFFF0EE1B
:10CA1000400AB0EE460AA4E79FED020AA7E700BF6E
:10CA2000E02E65420000000038B504460D4640681F
:10CA300001216EF0B5FB60682946BDE838406EF014
:10CA400017BC0379994205D00171806810B1036861
:10CA50001B6818477047406803681B68184783685D
:10CA60001979022904D0003918BF0121FFF7F3BF5B
:10CA70007047000008B54260064A02608A6881601B
:10CA80002AB1054B054A06481C214CF0BFF88860C6
:10CA900008BD00BF805D0B00125D0B00275D0B0021
:10CAA000005D0B00F8B50E4D2B68DB2928BFDB219C
:10CAB00001330B4441F22F12934284BF00232B60B9
:10CAC000084B2E681F680C460A4634440146B819C4
:10CAD00083F0BCFA00233B5501342C60B0B2F8BDA2
:10CAE000CC7B0020C87B002070B5104C2368254605
:10CAF0008BB941F230106BF083FC206058B90C4BBD
:10CB00000C4A18680C49BDE8704041F2301300F639
:10CB1000A86002F089BB094B28680021BDE870407D
:10CB200041F23012196083F0B9BA00BFC87B00200F
:10CB3000407F0020905D0B009B5C0B00CC7B0020B5
:10CB4000012110B5044608460AF026FD18B1206000
:10CB50000023637410BD6BF01DFC4FF47A73B0FBBF
:10CB6000F3F001232060F4E710B5054B054C0122DA
:10CB70001A70236813B96BF00DFC206010BD00BF64
:10CB8000D47B0020D07B0020054A838A106828B11E
:10CB900041F22F12934201D8184470470148704760
:10CBA000C87B002060C20B00FFF77CBF036882686F
:10CBB00018339342036008D1C3681A1D5B68C260D2
:10CBC00003F5FC724360826003607047036882680B
:10CBD00018339342036008D1C3681A1D5B68C260B2
:10CBE00003F5FC724360826003607047F8B5002370
:10CBF0000446C0E90233C0E90433C0E90633C0E9A2
:10CC0000083303600823436020204BF01DFF656854
:10CC10002060013D6D0800EB850706464FF4FC706F
:10CC20004BF012FF00F5FC73C4E9070346F825003A
:10CC3000E060A060A0616761236167622046F8BD83
:10CC400070B504468CB00D46FFF7D0FF04F13003F9
:10CC5000A3620023E362696884F8303008AA06A85A
:10CC60000A31CDE906238DF820307BF058FE0A22E8
:10CC7000104906A87BF0F2FF294606A87BF0E4FFE6
:10CC80000D4906A87BF0FAFF04F128060146684624
:10CC90007BF0FDFD694630467BF019FE68467BF06F
:10CCA00007FD06A87BF004FDFFF71EFF20460CB031
:10CCB00070BD00BFCB5D0B00D65D0B00036870B587
:10CCC000044663B1436A45691E1DAE4204D955F856
:10CCD000040B4BF0DDFEF8E720684BF0D9FE204650
:10CCE00070BD02698368183A934210B5044602D0B9
:10CCF0001833A36010BDC0684BF0CAFE63691A1DEB
:10CD00005B68626103F5FC72E3602261F1E7D0E9E0
:10CD100000239A4209D1C3681A1F53F8043C4360A8
:10CD200003F5FC73C260836003600368183B036013
:10CD300070470000CA68C3689B1AD0E90020121A25
:10CD400007489B10D210424310B5013B152404FB49
:10CD500003238A680968521AD21000FB023010BD02
:10CD6000ABAAAAAA0A6802604A6842608A6882601E
:10CD7000CA68C260704770B5012188B0064608468F
:10CD80000AF00AFC044608B36BF004FB4FF47A7314
:10CD900006F10801B0FBF3F56846FFF7E3FF06F183
:10CDA000180104A8FFF7DEFF0026009A049B9A42B0
:10CDB0000CD0537C33B113689D4221BF1B195B1B00
:10CDC000136056746846FFF701FFEEE708B070BDC8
:10CDD00010B588B0044600F108016846FFF7C2FFAD
:10CDE00004F1180104A8FFF7BDFF2046FFF766FF16
:10CDF000204608B010BD10B5044628307BF058FC22
:10CE00002046FFF7E5FF204610BD0A6802604A6829
:10CE100042608A688260CA68C26070477FB56E46A9
:10CE20000C46054601463046FFF79CFF94E80F008C
:10CE300085E80F0096E80F0084E80F0004B070BD8D
:10CE400010B5A2B0044603A8FFF7D0FE04F1080114
:10CE500005A8FFF7E3FF04F1180109A8FFF7DEFFBB
:10CE6000039B22682360049B039203A862686360AB
:10CE70000492FFF7ADFFFFF737FE134B02A81968C6
:10CE800003F088F8A16A002203A802F089FA0024BE
:10CE900001220DF1070103A88DF8074002F0EBFA1B
:10CEA00003A802F0BDFA094B1C706BF073FA084B33
:10CEB0001860084B039305A86AF08BFF02A803F0E3
:10CEC00071F822B010BD00BF3C7F0020D47B002051
:10CED000D07B002074640B002DE9F843426A43685C
:10CEE000074600684C1C8846111AA3EBA1018C422E
:10CEF00022D97969561A08EBA6056C1CB3EB440FCE
:10CF000022D91C1B640800EB8404131DA142A3EB6F
:10CF1000010213D9994202D0204683F0A5F8236874
:10CF2000FB6003F5FC733B61A3197B62A359FB61B2
:10CF300003F5FC737C613B62BDE8F8839942EED057
:10CF4000301D801A2044E8E7991C43452CBF01EBB3
:10CF500003088844B8F1005F01D37BF06FF94FEA12
:10CF600088004BF071FD7A6A7969A8EB04040432F9
:10CF700064089142814600EB840403D0521A204693
:10CF800083F072F838684BF083FDC7E90098C6E774
:10CF90002DE9F04100F1180886B006460C4600F174
:10CFA000080140460191FFF7C5FE1328019903D9F6
:10CFB0003046FFF796FE0199336AB769183B9F42E6
:10CFC00012D00FCC3D460FC594E80300183785E812
:10CFD0000300B761414602A8FFF7C4FE02A8FFF7AD
:10CFE00096FE06B0BDE8F0814046FFF7A3FE104B69
:10CFF000984202D10F487BF027F901213046FFF714
:10D000006BFF4FF4FC70756A4BF01EFD68600FCC2F
:10D01000B5690FC5736A94E803001A1D5B6885E85B
:10D020000300726203F5FC72F3613262B361D1E70F
:10D0300055555505DC5D0B00F8B5036A8769183B4B
:10D040009F4206460C4609D00FCC3D460FC594E8DA
:10D050000300183785E80300B761F8BD00F1080147
:10D060001830FFF767FE104B984202D10F487BF053
:10D07000EBF801213046FFF72FFF4FF4FC70756A83
:10D080004BF0E2FC68600FCCB5690FC5736A94E899
:10D0900003001A1D5B6885E80300726203F5FC72E9
:10D0A000F3613262B361D8E755555505DC5D0B007D
:10D0B00038B504460D4600F108011830FFF73AFE76
:10D0C000132802D92046FFF70CFE29462046FFF719
:10D0D000B3FF38BDF0B50C468BB000234FF0FF32E4
:10D0E00004F11007054604A80792CDE904338DF832
:10D0F0001830ADF820308DF822300993FFF720FD6D
:10D10000237A8DF81830DB21384684F021FB014664
:10D1100006463846FFF7C6FC164B22681B68ADF87A
:10D1200024001B68ADF82660002A18BF134605933B
:10D1300063680793013BD91C8CBF002301238DF842
:10D14000203092B98DF8222004A92846FFF7B0FFBD
:10D15000FFF70AFD05F118016846FFF703FE684670
:10D16000FFF7D5FD00980BB0F0BD01238DF82230FC
:10D17000EAE700BF7CF10B00F0B5DFB0044622A85F
:10D18000FFF734FD04F1080124A8FFF747FE04F17E
:10D19000180128A8FFF742FE229B22682360239BE8
:10D1A000229222A8626863602392FFF711FEFFF7C4
:10D1B0009BFC444B02A8196802F0ECFEA16A4248AD
:10D1C00064F08DF9002878D009A8A26A3E490023AE
:10D1D00064F07BF909A864F0EDFB00286DD0002312
:10D1E00001220DF1070109A88DF807306AF0D5F882
:10D1F0009DF80730142B88BF14234FF0000688BF1A
:10D200008DF8073035464FF0FF379DF80720F3B211
:10D210009A4248D9EE22002122A8CDE903558DF883
:10D2200014500697ADF81C508DF81E50089582F0EA
:10D2300035FFEE2222A909A86AF0AFF8EE2806F120
:10D24000010630D1229B0393239B04939DF89030D9
:10D250008DF81430DDF8913006939DF89530003B41
:10D2600018BF01238DF81D309DF896308DF81E30C3
:10D270009DF897308DF81C30DB21BDF89830ADF863
:10D2800022300DF19A0084F063FAADF8220081B2E9
:10D290000DF19A00FFF706FC03A9ADF82000204627
:10D2A000FFF7CAFEB1E709A864F01BFB074B002299
:10D2B0001A706BF06FF8064B186002A802F072FE4D
:10D2C0005FB0F0BD3C7F00201C800120D47B00209B
:10D2D000D07B002070B50D4688B016460446FFF797
:10D2E00085FC05F108016846FFF78FFD05F118017F
:10D2F00004A8FFF78AFD0099049B99420BD00B7C90
:10D300002BB90B7AB34202D12046FFF795FE68464F
:10D31000FFF74CFCEFE7204608B070BD30B50D4676
:10D3200089B00446FFF762FC05F108016846FFF783
:10D330006CFD05F1180104A8FFF767FD0099049B37
:10D34000994209D00B7C012B02D12046FFF774FED5
:10D350006846FFF72BFCF1E7204609B030BD00001E
:10D3600010B5D0E90043144AE31ADB1002FB0312A4
:10D37000002A1BDB142A04DC182303FB0141016093
:10D3800010BD152392FBF3F3C16801EB830451F840
:10D390002310C46001F5FC748460152404FB13237E
:10D3A000182202FB031341600360E9E7D343152110
:10D3B000B3FBF1F3DB43E7E7ABAAAAAA2DE9F043FD
:10D3C000464DDFF83091DFF83081E1B0044628683F
:10D3D00002F0CBFD4249434864F097F8286802F018
:10D3E000CEFD0022A16A05A801F0DAFF04F10806CB
:10D3F000286802F0BAFD314604F11800FFF79AFCE4
:10D40000C0B2142894BF8DF8030014234FF001021A
:10D410000DF1030105A888BF8DF8033002F02BF849
:10D4200000279DF80330FCB2A34241D9314624A81D
:10D43000FFF798FC214624A8FFF792FF014601A8B8
:10D44000FFF790FC019C0021DE2228A882F026FE36
:10D450002368249363682593237A8DF89830E368D2
:10D46000CDF89930637C8DF89D30A37C8DF89E308B
:10D47000237C8DF89F30E38AD9F80010ADF8A030F6
:10D48000A38A99B141F22F1293420FD81944DB229B
:10D490000DF1A20084F049F90023EE2224A905A889
:10D4A0008DF87D31013701F0E6FFBAE74146EEE73E
:10D4B000286802F064FD05A801F0B2FF0A4B0022C3
:10D4C0001A706AF067FF094B1860094B059307A8AB
:10D4D0006AF07FFC61B0BDE8F08300BF3C7F0020B4
:10D4E0009D180C001C800120D47B0020D07B0020E4
:10D4F00074640B00C87B002060C20B0038B5104D6F
:10D500006AF048FF2A6804460AB92C6038BD0D4B02
:10D510009B1AC342FAD40C4B18680C4B1B7800F6CC
:10D52000A86043B10A4A0B4901F07EFEBDE83840CD
:10D530000948FFF743BF094A064901F075FEE4E7D1
:10D54000D07B0020002392FF407F0020D47B00206E
:10D550000C5E0B002D5E0B00D87B0020335E0B00B1
:10D56000CA68C3689B1AD0E90020121A07489B10AA
:10D57000D210424310B5013B152404FB03238A68F3
:10D580000968521AD21000FB023010BDABAAAAAA39
:10D5900010B5D0E90043144AE31ADB1002FB031272
:10D5A000002A1BDB142A04DC182303FB0141016061
:10D5B00010BD152392FBF3F3C16801EB830451F80E
:10D5C0002310C46001F5FC748460152404FB13234C
:10D5D000182202FB031341600360E9E7D3431521DE
:10D5E000B3FBF1F3DB43E7E7ABAAAAAA2DE9F04FBF
:10D5F000A3B00D460746114602A8144605F10806D9
:10D60000FFF7B0FB02A8FFF7E1FA31461EA8FFF7CB
:10D61000A9FB1EA92046FFF78DFB05F118098046DE
:10D6200031464846FFF786FBB8EB500F80F0848008
:10D6300031461EA8FFF796FB23681E9A9A4264D0D3
:10D64000314606A8FFF78EFB21460AA8FFF78AFBA2
:10D6500002A90EA8FFF786FB06A91EA8FFF7D5FBB7
:10D660000AA91AA8FFF7D1FB0EA916A8FFF77AFBA3
:10D670001EA91AA8FFF774FFDFF8889183464FF0C0
:10D68000180ABBF1000F3CDDDDE91AC4A44508BF50
:10D690001D9ADDE9160317BFACEB040452F8042C05
:10D6A000E41009FB04F404BF152402F5FC7C984245
:10D6B0000BBF199BC31A53F8040CDB1012BF09FBF4
:10D6C00003F3152300F5FC705C45A8BF5C469C4243
:10D6D000A8BF1C460AFB04F2ACEB02018C45C2F168
:10D6E000000302D0184482F0BFFC61421AA80191E5
:10D6F000FFF74EFF019916A8FFF732FEABEB040BC4
:10D70000BFE716A912A8FFF72DFB2846FFF7E9FA95
:10D7100031461AA8FFF726FB1AA91EA8FFF722FB1D
:10D7200041461EA8FFF71CFE01463846FFF71AFBCC
:10D73000384623B0BDE8F08F49461EA8FFF712FB1C
:10D74000029A1E9B9A4246D002A90AA8FFF70AFB3A
:10D75000494606A8FFF706FB21460EA8FFF702FB85
:10D760000AA91EA8FFF751FB06A91AA8FFF74DFB4F
:10D770000EA916A8FFF7F6FA1EA91AA8FFF7F0FEE1
:10D78000DFF8809083464FF0180ABBF1000F1EDDD2
:10D790001E99209B1698189C5B1A241AA342CCBF92
:10D7A000E410DC1009FB04F45C45A8BF5C4652465B
:10D7B000624301D082F058FC21461EA8FFF7E8FE24
:10D7C000214616A8FFF7CCFDABEB040BDDE716A94D
:10D7D00012A8FFF7C7FAD5E90603984202D0183815
:10D7E000A86195E74BF054F96B6A1A1F53F8043C93
:10D7F0006A62EB6103F5FC7203F5F0732A62AB61B8
:10D8000086E700BFABAAAAAA30B5D568136885B071
:10D810006A4600932B68019303F5FC730446CDE937
:10D820000235FFF7E3FE204605B030BD2DE9F04399
:10D830008DB06C4605460F4600F108012046FFF703
:10D8400091FADFF8609005F11808414608A8FFF743
:10D8500089FA009B089A93421ED01A7C012A17D19C
:10D86000D9F800105A6809688A4208BFDA689742F6
:10D870000ED1214604AE08A8FFF7C7FA08AA294628
:10D880003046FFF7C1FF96E80F0084E80F00DCE7A1
:10D890002046FFF79BF9D8E72846FFF78FFD0DB02C
:10D8A000BDE8F0837CF10B002DE9F0431C4B8DB0FB
:10D8B0001B686C4605460F4600F108012046D3F868
:10D8C0000080FFF74FFA05F1180904AE494608A891
:10D8D000FFF748FA009B089A93421AD01A7C012A53
:10D8E00013D15A68904508BFDA68BA420DD1214673
:10D8F00008A8FFF78AFA08AA29463046FFF784FFEE
:10D9000096E80F0084E80F00E0E72046FFF75EF995
:10D91000DCE72846FFF752FD0DB0BDE8F08300BFFD
:10D920007CF10B002DE9F0418CB06C4605460F46AA
:10D9300000F108012046FFF715FA05F1180804AEBA
:10D94000414608A8FFF70EFA009B089A934216D0AA
:10D950001A7C82B91B7ABB420DD1214608A8FFF779
:10D9600054FA08AA29463046FFF74EFF96E80F0002
:10D9700084E80F00E4E72046FFF728F9E0E72846AF
:10D98000FFF71CFD0CB0BDE8F0812DE9F0418CB033
:10D990006C4605460F4600F108012046FFF7E2F904
:10D9A00005F1180804AE414608A8FFF7DBF9009B13
:10D9B000089A934216D01A7C82B91B7ABB420DD1C9
:10D9C000214608A8FFF721FA08AA29463046FFF7A2
:10D9D0001BFF96E80F0084E80F00E4E72046FFF7FE
:10D9E000F5F8E0E72846FFF7E9FC0CB0BDE8F08168
:10D9F000F0B58DB06D46044600F108012846FFF7EA
:10DA0000B1F904F1180708AE39463046FFF7AAF914
:10DA1000009A089B9A420DD0294604A8FFF7F5F911
:10DA200004AA21463046FFF7EFFE96E80F0085E88E
:10DA30000F00E9E72046FFF7C1FC0DB0F0BD000084
:10DA400010B50D4A0D4C86B002A8D11F00907AF097
:10DA5000A2FE07230193009B0022DA71694620464B
:10DA6000FFF7EEF868467AF023FE054A054920469E
:10DA70007AF03DFA06B010BD5F5E0B00D87B002047
:10DA800000600020F7CD020000207047F8B5036861
:10DA90005B680446984707EE900A94ED087AF8EE22
:10DAA000677AB4EEE77AF1EE10FA47DC231D002521
:10DAB00033F8022B904238D3002D3CD004EB4504C0
:10DAC00007EE102A6388B8EEC77A9B1A37EEC77A3A
:10DAD00007EE903AF8EEE77AC7EE277A17EE900A4B
:10DAE00080F0C0FF064628460F4680F0A9FF024698
:10DAF0000B460020134980F055FE02460B46304687
:10DB0000394680F051FE0F4B002281F003F881F07E
:10DB1000F9FA07EE900AFDEEE77A17EE900A64280C
:10DB2000A8BF642020EAE070F8BD01350B2DBFD1FD
:10DB3000DFED057AEFE7DFED057AECE74FF0FF3038
:10DB4000F2E700BF00002440000000000000C842CF
:10DB500008B503681B689847013018BF012008BD4D
:10DB6000036810B55B680446984707EE900A94ED89
:10DB7000077AF8EEE77AF4EEC77AF1EE10FACCBF46
:10DB80000120002010BD704770477047704730B4C7
:10DB9000826904695510034604EB6200D20748BF4E
:10DBA00062595B6930BC48BFD358184730B48269AA
:10DBB00004695510034604EB6200D20748BF62595E
:10DBC0005B6930BC48BFD358184708B517206DF0C3
:10DBD0006BFBB0FA80F0400908BD406842F02EB9F6
:10DBE000406842F049B9406842F040BA08B5406820
:10DBF00042F0E8F808BD406842F09CB870B50546B0
:10DC0000084B0360044655F8300FA84204D006685C
:10DC10004AF03EFF3046F8E7204602F0C1FA2046BF
:10DC200070BD00BF40600B0010B50446FFF7E6FF73
:10DC3000204660216CF098F9204610BD10B5064BC7
:10DC4000036003F14C0258330446426183611C3087
:10DC500058F0C1FD204610BD7C950C0008B5044B62
:10DC60000021186802F0B2FA024B01221A7008BDB6
:10DC7000007D00202AA1002070B591F8505091F845
:10DC80005920044605F1FF3CDCF1000694F85030C1
:10DC9000486D46EB0C069E422ED1531E5E425E41FD
:10DCA00094F859309E4227D1636D1B1A18BF012387
:10DCB00084F85050606591F850000126B04284F815
:10DCC000206008BF91F8580084F8592018BF002040
:10DCD00084F8580091F85A2084F85A2073B12646E7
:10DCE00056F8285FB54209D0A868036821469B68AA
:10DCF000984718B92D68F5E70123D9E7002070BDD2
:10DD000008B501210E206DF04BFA0E2000216DF0B8
:10DD1000AFFABDE808400A206AF047BB08B51C4BC3
:10DD200093F8B40068B11B4B93F82820824209D1C4
:10DD30001948037B23BB41F015FA0028D4BF00200B
:10DD4000012008BD93F81021824205D11348037BBE
:10DD5000B3B941F0F1FAF0E793F82020824205D1FF
:10DD60000F48037B63B941F06FFBE6E793F870302F
:10DD700083420AD10B48037B13B941F0EBFBDCE78C
:10DD80008068003818BF0120DBE70020D9E700BF1A
:10DD900040CC0020609F00201C7C00204C7C002098
:10DDA0008C7C0020B47C0020F0B52DED028B83B07C
:10DDB0000446FFF7B3FF514B28B3514A93F8B430F0
:10DDC00092F82810994206D14E4841F0ADF903B0BF
:10DDD000BDEC028BF0BD92F81011994203D14A4874
:10DDE00041F03EFAF3E792F82010994203D14748F8
:10DDF00041F08AFBEBE792F870209A427CD14448CC
:10DE000041F0ECFBE3E793ED288A94F82430B5EE7B
:10DE1000C08AF1EE10FAD8BFB0EE088A002B42D1CA
:10DE20006AF0B8FAE062FFF76BFF3A4B01A8196895
:10DE300002F0B0F80F26002520206DF07FF9013E9A
:10DE40000544F9D10F20B5FBF0F080F0E9FD06465E
:10DE500018EE100A0F4680F005FE2F4B002280F0CE
:10DE600059FE0B4602463946304680F053FE81F09B
:10DE700049F9012108EE100A0E206DF0F9F994F825
:10DE80002430D4ED0A8AEBB9F4EEC88AF1EE10FA28
:10DE90004FF0010348BF84ED0A8A84F8243001A8BA
:10DEA00002F080F806E0E06A41F288312DF085FD4D
:10DEB0000028B5D0D4ED0A7AFCEEE77A17EE903A56
:10DEC00098B284E778EE687A17EE900A80F0CAFD7F
:10DED000124B002280F01EFE064618EE900A0F46F6
:10DEE00080F0C0FD02460B463046394680F05CFCAF
:10DEF00081F008F9A062D2E7002068E740CC00205A
:10DF0000609F00201C7C00204C7C00208C7C00202A
:10DF1000B47C00206468002000200C400000E03F3A
:10DF200070B5134B13490446002202F06DF92346E5
:10DF3000114A43F8302BC4E90C330023A3630F4B81
:10DF400004F13C0203F1100618685968154603C530
:10DF50000833B3422A46F7D118689B88AB80002368
:10DF60002860E365636584F85830204670BD00BFC3
:10DF7000907F0020ED430C0040600B0020600B0000
:10DF800008B5002117206DF00BF90A4B0A4A1868F2
:10DF90000A49202300F6A86001F046F9002120205C
:10DFA0006DF0FEF80A206DF09DF8054B054A1A60E9
:10DFB000012008BD407F0020605E0B006C5C0B0000
:10DFC000187C00201861002008B50C4D2C68AC426C
:10DFD00007D0A068036800219B68984708B92468A7
:10DFE000F5E7BFF34F8F0649064BCA6802F4E062BB
:10DFF0001343CB60BFF34F8F00BFFDE7C44C01203C
:10E0000000ED00E00400FA0508B5124B186818B1DD
:10E01000114900220BF0D8FC01F0EAFE0F4B1F2142
:10E02000186826F099F90E48FFF7C8F900210D206D
:10E030006DF0B6F800210C206DF0B2F800210B2035
:10E040006DF0AEF80122BDE8084011464FF0FF30F8
:10E050004BF0A6B82CA10020865E0B0020D8002033
:10E06000D87B002038B5124D2B6804467BB16AF08E
:10E0700091F92B6898420AD90E4B0F4A18680F493C
:10E0800000F6A86001F0D0F82046FFF79DFF0C4D88
:10E090002B685BB16AF07EF92B68984206D90023A1
:10E0A0002B602046BDE83840FFF7AEBF38BD00BF4B
:10E0B0001CA10020407F002039780C002D5E0B0051
:10E0C00038A1002002490222172069F061BD00BF7B
:10E0D0005DDC020070B5144D6B6813B941F0C0FDF2
:10E0E0006860124B124E93F8E0406CB93668114BE1
:10E0F00006F6A866104A1149304601F095F80CB1B1
:10E100000F4B1D60204670BD6868D3F8E4100268AC
:10E11000126890473668074A0A4B041E06F6A8663E
:10E1200008BF1346E6E700BF4C610020609F002057
:10E13000407F0020975E0B00A55E0B006C5C0B001F
:10E14000187C00208FA90C0038B50546FFF7C2FFE8
:10E15000044618B92846FFF713FF04462846FFF780
:10E16000B1FF00232C7585F85830204638BD38B5EE
:10E1700004460068844204D005684AF089FC2846B9
:10E18000F8E738BD2DE9F8438046154B58F8045F91
:10E1900003600446454515D0AF683E68B7420FD0CE
:10E1A000B368D6F800909C4208D1BB68013B30466A
:10E1B000BB6079F0A8FE30464AF06AFC4E46EDE7B7
:10E1C0002D68E7E72846FFF7D2FF00232846C4E979
:10E1D0000155E360FFF7CBFF2046BDE8F88300BFA1
:10E1E000805F0B0010B50446FFF7CCFF20461021DE
:10E1F0006BF0BAFE204610BD10B5034B0360044619
:10E20000FFF7C0FF204610BD945F0B0070B50546B8
:10E21000084B0360044655F8280FA84204D006684E
:10E220004AF036FC3046F8E7201DFFF7E5FF2046B0
:10E2300070BD00BFA85F0B0010B50446FFF7E6FFF6
:10E24000204634216BF090FE204610BD10B50446E8
:10E25000FFF7D2FF20461C216BF086FE204610BD42
:10E2600038B504460068844204D005684AF010FCC2
:10E270002846F8E738BD00002DE9F8438046154BE5
:10E2800058F8045F03600446454515D0AF683E6802
:10E29000B7420FD0B368D6F800909C4208D1BB6853
:10E2A000013B3046BB6079F02EFE30464AF0F0FB71
:10E2B0004E46EDE72D68E7E72846FFF7D1FF00233C
:10E2C0002846C4E90155E360FFF7CAFF2046BDE8D0
:10E2D000F88300BFB85F0B0010B50446FFF7CCFF12
:10E2E000204610216BF040FE204610BD10B5034BB8
:10E2F00003600446FFF7C0FF204610BDCC5F0B0053
:10E3000010B5054B044640F8343BFFF7EFFF2046BD
:10E31000FFF77CFF204610BDE05F0B002DE9F04FBA
:10E320007B4E054630689DB0002800F0B180036840
:10E330009B689847044630680368DB6898478346C3
:10E34000306803681B6998478246002C00F0A4805F
:10E35000306803685B6898470746306803681B6845
:10E360009847002877DB306803681B68984740B2FD
:10E370000124684A069205AA07AB0A92664A8DF8FC
:10E380006440CDE907330023CDE90B230FAACDE983
:10E390000F22624A059213AACDE91322604A129213
:10E3A00005AA16925F4A0993022CCDE917238DF82E
:10E3B00034300E93119315938DF86DB08DF86EA0D7
:10E3C0001A978DF86C0039D0574F3B78A3420DD087
:10E3D000564B574A1868574B5749012C08BF1346EC
:10E3E00000F6A860554A00F01FFF3C70012C25D1B3
:10E3F000E86D4CF250312DF0E0FA0246F0B94B4B8B
:10E400009DF8647018689DF86D30591E4B424B4161
:10E410009DF86E104C1E61426141012F08BF9DF8AE
:10E420006C201A9C0091CDE901424549454A00F60D
:10E43000A86000F0F9FE69F0ADFFE8652F4657F8D7
:10E44000304FBC422CD0A068036805A99B68984750
:10E4500030BB2468F5E7B5F85040381B80F0F0FA7F
:10E46000394B002280F056FB8046A88F001B89465E
:10E4700080F0E6FA02460B464046494680F074FCBE
:10E4800080F0F8FD6428A8BF642020EAE0706EE701
:10E490004FF0020A5446D3464FF0FF30074668E774
:10E4A000306858B39DF86430012B27D19DF86D304A
:10E4B000012B23D003685B689847B5F8503083423E
:10E4C00022D995F85830194C204A20681C4901334C
:10E4D000DBB285F8583000F6A86000F0A5FE95F88C
:10E4E00058300A2B0AD920681349194A00F6A86047
:10E4F00000F09AFE17480A214DF06DFB05A8FFF7C2
:10E50000FFFE1DB0BDE8F08F002385F85830F5E719
:10E51000187C0020945F0B0089DA0200E05F0B009A
:10E52000CC5F0B0079DC020048610020407F0020B6
:10E5300032BB0C00CB5E0B002D5E0B00DD5E0B00D2
:10E540006C5C0B00F85E0B0000005940315F0B0063
:10E550004C5F0B00047D002010B50446FFF7DEFE83
:10E56000636D43B193F82030002B44F6206008BF60
:10E570004FF0FF3010BD4FF0FF30FBE710B5044601
:10E58000FFF7BEFE20465C216BF0EEFC204610BD7E
:10E5900010B50446FFF7AAFE20461C216BF0E4FCF0
:10E5A000204610BD10B50446FFF748FB2046302139
:10E5B0006BF0DAFC204610BD10B5402104466BF02C
:10E5C000D3FC204610BD10B5282104466BF0CCFCCE
:10E5D000204610BD10B5302104466BF0C5FC204626
:10E5E00010BD10B51C2104466BF0BEFC204610BDCA
:10E5F00010B5174C204640F015FE2046154C164A23
:10E60000164979F074FC204640F04EFE2046144C2A
:10E61000114A144979F06BFC204640F081FF2046F6
:10E62000114C0D4A114979F062FC204640F0F8FF88
:10E6300020460F4C084A0F4979F059FC204641F01A
:10E6400061FC2046044A0C49BDE8104079F04FBCFB
:10E650001C7C00204C7C0020006000203DDC02007F
:10E660008C7C002087DB0200B47C002089DB020068
:10E67000E47C00208BDB02008DDB02007047012070
:10E680004AF0FCBAFFF7FBBF08B5054BD3F8A8006A
:10E6900021F0E2FABDE80840012200214AF080BDE5
:10E6A00040CC002008B5054BD3F8A80021F0D4FADF
:10E6B0000022BDE8084011464AF072BD40CC00205F
:10E6C00008B569F067FE014B186008BD38A100204D
:10E6D0000F4A1379022B14D0A3F10B014B424B418B
:10E6E00092F8980078B98BB90A4B1B6873B193F80C
:10E6F0005020012A09D193F85900431E584258412D
:10E7000070470123ECE7002070470120704700BFED
:10E7100040CC002018A1002008B5074B0749186815
:10E72000074A00F6A86000F07FFDBDE808400548F4
:10E730000E214DF050BA00BF407F00202D5E0B002F
:10E7400064600B00047D002008B5FFF7C1FF18B915
:10E75000BDE80840FFF7E0BF08BD000008B5FFF7BF
:10E76000B7FF28B1BDE8084002480D214DF033BA8B
:10E7700008BD00BF047D002070477047836810B556
:10E78000044613B1032201469847204610BD0000FD
:10E790001FB5FFF79DFF20B9FFF7BEFF05B05DF87D
:10E7A00004FB084B186840B100236A46012102931C
:10E7B0000AF09AF96846FFF7E1FF01204AF05EFA95
:10E7C000ECE700BF2CA100201FB5094B186840B131
:10E7D00000236A46012102930AF086F96846FFF792
:10E7E000CDFF01204AF04AFA05B05DF804FB00BFF6
:10E7F0002CA100201FB500204AF040FA074B1868F2
:10E8000040B100236A46012102930AF06DF968467F
:10E81000FFF7B4FF05B05DF804FB00BF2CA100209A
:10E820001FB501204AF02AFA064B186838B10021BA
:10E830006A4602910AF058F96846FFF79FFF05B053
:10E840005DF804FB2CA100201FB5074B186838B1F8
:10E8500000216A4602910AF047F96846FFF78EFFE9
:10E8600005B05DF804FB00BF2CA100201FB5074BCD
:10E87000186838B100216A4602910AF035F96846F5
:10E88000FFF77CFF05B05DF804FB00BF2CA1002062
:10E890002DE9F74FC34F3E79022E00F02982A6F1F1
:10E8A0000B035E425E41FFF713FFBF4BBF4DDFF826
:10E8B00048B3BF4ABF49DFF81093DFF840A3804652
:10E8C0001868434600F6A860002400F0ADFCBA4B7F
:10E8D000BA490193A04514BF5A462A4640F6B833B8
:10E8E000B74800944DF028F9B64BB74AB749B44839
:10E8F000DFF8FC82CDE9004302234DF0FCF8B44B75
:10E90000B249AF48A64214BF42464A46CDE9004349
:10E9100004234DF0F0F8AF4BA948CDE9004342463F
:10E92000042341464DF0E7F8CDE9004AA749A44841
:10E9300001232A464DF0DFF801232A464146CDE95E
:10E94000004A9F484DF0D7F8FFF7C2FECDE9004AD4
:10E95000A04214BF5A462A460123994849464DF021
:10E96000CAF8CDE9004A964801235A4659464DF067
:10E97000C2F8CDE9004A924801232A4629464DF0C3
:10E98000BAF8954A8E48CDE9004ADFF874A21146DC
:10E9900001234DF0B0F8CDE9004A904A87498848F4
:10E9A0000A234DF0A8F8CDE9004A8C4A87498448EB
:10E9B0000A234DF0A0F8CDE9004A884A80480A238E
:10E9C00041464DF098F8CDE9004A844A7C480A2334
:10E9D00049464DF090F8CDE9004A804A78480A232C
:10E9E00029464DF088F8CDE9004ADFF818A27B4AA5
:10E9F000794973480A234DF07EF8CDE9004A784AF8
:10EA00006E496F4810234DF076F8CDE9004A744AFC
:10EA10006E496B4810234DF06EF8CDE9004A704AFC
:10EA20006748102341464DF066F8CDE9004A6C4A2C
:10EA30006348102349464DF05EF8CDE9004A684A24
:10EA40005F48102329464DF056F8CDE9004ADFF81B
:10EA5000B8A1634A60495A4810234DF04CF8CDE9FB
:10EA6000004A5A49564811232A464DF044F8CDE948
:10EA7000004A534811232A4641464DF03CF8CDE95F
:10EA8000004A4F4811232A4649464DF034F8CDE953
:10EA9000004A4B4811232A4629464DF02CF8CDE96F
:10EAA000004ADFF868A1464811235A4659464DF0FE
:10EAB00022F8434807232A464946CDE9004A4DF04B
:10EAC0001AF8CDE9004A3E4807232A4629464DF068
:10EAD00012F84EBB434B444C3948CDE900634A46DB
:10EAE000042341464DF007F83849354805232A46A6
:10EAF000CDE900644CF0FFFF314805232A4641462A
:10EB0000CDE900644CF0F7FF2D4805232A4649461D
:10EB1000CDE900644CF0EFFFCDE9006428480523FF
:10EB20002A4629464CF0E7FF0024304D2A4A27495F
:10EB3000234801950B2300944CF0DDFFCDE90045FF
:10EB4000254A2B491E480B234CF0D5FFCDE9004543
:10EB5000214A1D491A480B234CF0CDFFCDE9004551
:10EB60001D4A124916480B234CF0C5FFCDE900455C
:10EB7000204D194A204912480B234CF0BCFF1E4A75
:10EB800012490F480D23CDE900454CF0B4FF1A4A55
:10EB900017490B480D23CDE900454CF0ACFF164A50
:10EBA00036E000BF40CC0020407F0020487E00209F
:10EBB0007D600B002D5E0B0099600B00F87D00203E
:10EBC000047D0020A6600B00087E0020187E002037
:10EBD000B1600B00D6600B00787E0020287E0020FC
:10EBE000887E002026610B0037610B0045610B0019
:10EBF000387E002050610B00587E0020FA600B0028
:10EC000000610B007F960B0007610B0014610B0085
:10EC10003B493C480D23CDE900454CF06CFF3A4A96
:10EC20003A4938480D23CDE900454CF064FF384B94
:10EC3000364A35493348CDE900430E234CF05BFF9B
:10EC4000344B324A34492F48CDE900430C234CF071
:10EC500052FF324B2A4A2B48CDE900431146092383
:10EC60004CF049FF3B79D7F88C01022B42D00B2B9B
:10EC70000CBF01214FF4167120F0E0FF284C23490E
:10EC800001940022034600921E481D4A4CF054FF96
:10EC90003B79D7F88C01022B2ED00B2B0CBF012116
:10ECA0004FF4167120F0CAFF002203460092164965
:10ECB000134A144801944CF03FFF3B79D7F88C017C
:10ECC000022B1BD00B2B0CBF01214FF4167120F02F
:10ECD000B5FF002200920A4A0194034611460948F2
:10ECE0004CF02AFF074803B0BDE8F04F4CF0B3BF2B
:10ECF0000126D8E50121BFE70121D3E70121E6E79D
:10ED0000087E0020047D0020587E0020487E0020E0
:10ED10005E610B0071610B00787E002083610B0047
:10ED200096610B0037B52E4B009300231A462D49F0
:10ED30002D482E4C2E4D4CF0C7FE002300941A4651
:10ED40002C492D484CF0C0FE002300941A462B4954
:10ED50002B482C4C4CF0B8FE2B4B00932B4A2C4BE1
:10ED60002C492D484CF0B0FE2C4B009300231A4642
:10ED70002B492C484CF0A8FE2B4B009300231A463D
:10ED80002A492B484CF0A0FE2A4B00932A492B4BD2
:10ED90002B4800224CF098FE2A4B009300231A4681
:10EDA000294928464CF090FE284B0093284A2949CF
:10EDB000294800234CF088FE284B294A0093294912
:10EDC000294B2A484CF080FE294620464CF083FE11
:10EDD000274A2849204603B0BDE8304079F087B87B
:10EDE000A8610B00C1E60200887E0020B1610B0023
:10EDF000F87D0020A5E60200687E002089E602007A
:10EE0000287E0020047D0020CD6C0B007DE60200F2
:10EE10007BE702006DE80200187E0020B5610B0060
:10EE200049E80200387E0020B8610B0021E80200AA
:10EE3000087E0020BD610B00F5E702007FE60200BE
:10EE4000787E002026590B0079E70200C4610B0090
:10EE50005DE70200C9E70200487E0020C7610B00A1
:10EE600049E7020091E7020085E60200587E002093
:10EE700000600020E9BA07007047704708B510200D
:10EE800049F0E2FD00230022C0E9002300230372C1
:10EE9000014B186008BD00BF987E002008B5094BE3
:10EEA00093F8F0215AB193F89F2293F8A43103B15B
:10EEB0001AB1806803681B689847012008BD5A7919
:10EEC000F3E700BF40CC002003685B68184710B52B
:10EED00000F110010446012069F066FCE06010BDFD
:10EEE0002DE9F3472F4F019304460D463846A021E4
:10EEF00083F0F8FE9F2884BF0A2387F89E30294FAD
:10EF000006464FF0000888BF9F264FF0230A46456B
:10EF10000ED097F80090484680F0ACFF20B9B9F1C8
:10EF20000A0F18BF87F800A008F101080137EEE7C3
:10EF30003DB31D49284682F075FB20B91B490522C7
:10EF40002046FFF7C1FF1A49284682F06BFB20B923
:10EF5000184905222046FFF7B7FF1749284682F0D7
:10EF600061FB20B9154905222046FFF7ADFF144982
:10EF7000284682F057FB20B9124905222046FFF7A8
:10EF8000A3FF324607492046FFF79EFF064625B1FC
:10EF90000D4904222046FFF797FF304602B0BDE836
:10EFA000F08700BF9C7E00206C5C0B00CD610B00E5
:10EFB0002D5E0B00D3610B00D9610B00DF610B00EC
:10EFC0009B5C0B00E5610B00EB610B002DE9F74347
:10EFD0000D4604464A4928461746984682F022FBC9
:10EFE00020B9484905222046FFF76EFF46492846CA
:10EFF00082F018FB20B9454905222046FFF764FF3F
:10F000004349284682F00EFB20B94249052220469A
:10F01000FFF75AFF4049284682F004FB20B93F49D8
:10F0200005222046FFF750FF3D49284682F0FAFAB4
:10F0300020B93C4905222046FFF746FF012108463A
:10F0400008F0AAFA002846D0374BB0FBF3F103FBD7
:10F05000110000F5A83000F5C070B0FBF3F603FB1B
:10F0600016004FF461662A46B0FBF6F92F4906FBFD
:10F070001906204668F086F82D49204668F082F887
:10F0800069F088F93C22B6FBF2F302FB13664FF4F9
:10F090007A710096B0FBF1F04A460190254920466E
:10F0A00068F070F8244B1E6866B12449204668F069
:10F0B00046F806F11C01204668F03BF8204920463E
:10F0C00068F03DF843463A462946204603B0BDE87D
:10F0D000F043FFF705BF2A461449204668F052F86E
:10F0E0001349204668F04EF869F054F915494FF479
:10F0F0007A72B0FBF2F2204668F044F8D2E700BF23
:10F100006C5C0B00CD610B002D5E0B00D3610B001E
:10F11000D9610B00DF610B009B5C0B00E5610B000C
:10F12000F0610B00F6610B0080510100ACBF0B00D9
:10F13000EB610B00FC610B00348100208C550C004E
:10F1400020620B0011620B000B78433BDBB2142BE7
:10F150009ABF024AD05C0020704700BFF8630B00E2
:10F160002DE9F0431E46264B93F8A032EBB007463C
:10F1700088461446002B3FD0224B1B78002B3BD1F6
:10F18000214D2868002837D00368DB68984798B37A
:10F190001E4B1F49D3F800904FF4D472684680F09C
:10F1A00055FF41463846FFF7CFFF32468DF8A401A0
:10F1B0002146684683F0BAFDB9F1000F04D0D9F8B2
:10F1C0001C1061A882F038FA0121084608F0E4F921
:10F1D00060904FF4D57049F049FC0E4A6B464FF4ED
:10F1E000D57104462FF0C2F821460246286848F03F
:10F1F00005FE204649F04EFC6BB0BDE8F08300BF31
:10F2000040CC002015A1002010A100203481002056
:10F2100050620B000C310C0010B50446006808B1B8
:10F2200049F038FC204610BD0CB42DE9FF41DDF853
:10F230002880044640460E4682F04AFA07460230CD
:10F2400049F014FC41460546019082F0F5F90A2385
:10F25000EB553D4400236B70174B93F8F13023B10D
:10F260001649304682F0DEF9E8B1E068D8B14FF0D7
:10F27000FF3169F081FB012815D122680BABCDE984
:10F280000233D568019A31462046A847029B019A6D
:10F29000039331462046FFF763FF0023E0681A46D8
:10F2A000194669F0FDF901A8FFF7B6FF04B0BDE803
:10F2B000F04102B0704700BF68D500206C5C0B00C5
:10F2C0000CB4F0B585B00AAE002356F8047B019368
:10F2D0007D6804466D00284649F0C8FB019B0190FB
:10F2E00013B1184649F0D6FB3968019882F0A4F9A9
:10F2F00033463A6801980296294683F0F3FC031ED0
:10F3000001DB9D4205DC5B1B54BF0133DB431D4425
:10F31000E1E7019D04F10803236015B3284682F05C
:10F32000D7F90F2805EB0006039007D9002203A99F
:10F33000204679F09BF9039B2060A3602068324649
:10F34000294679F028FA039B226863600021D15492
:10F3500001A8FFF761FF204605B0BDE8F04002B00C
:10F360007047014878F06DFF23620B0038B5084DF7
:10F370002B682BB1074B084A08480A2149F046FC84
:10F38000042049F061FB044600F0C8FD2C6038BD44
:10F390003C7F002028640B0031640B0040640B00AC
:10F3A0002DE9FF41184BDFF87480002704464760C1
:10F3B00040F8083B0D46164668F050FD134B03A875
:10F3C000196800F0E7FD124B124A186812490096BE
:10F3D0002B4600F6A860FFF727FF2946404662F05B
:10F3E000E4F801232A46414604F1140062F06DF866
:10F3F00003A800F0D7FD204684F8786084F879707F
:10F4000004B0BDE8F08100BF74640B003C7F0020B5
:10F41000407F002050640B006C5C0B001C800120BE
:10F4200070B500F11405284662F0C4FA044648B1EC
:10F43000054E306800F099FD284662F052FA3068B7
:10F4400000F09DFD204670BD3C7F002070B500F1AE
:10F450001406044630460D4662F0ACFA50B194F8FA
:10F4600079306B4084F8793029463046BDE87040E9
:10F4700062F0B1B870BDF8B500F114070546384622
:10F480000C46164662F096FA90B122463019824236
:10F4900007D012F8013B95F879104B4085F8793088
:10F4A000F5E7324621463846BDE8F84062F0A8B894
:10F4B000F8BD704770470368DB6A1847A0F608700C
:10F4C000FFF7F9BF0249D0F880062CF076BA00BFEA
:10F4D000A0BB0D000A2938B50D4600F6A86403D17B
:10F4E0000D212046FFF7DAFC29462046BDE83840CA
:10F4F000FFF7D4BCA0F6A860ECE7002100F6087086
:10F5000000F064BE7FB504461D4694F8353F0E46B4
:10F5100000F6A860B3B10F4B93F8A03293B10392F9
:10F52000FFF712FE0C4B039A1B68014643B1D869E2
:10F5300000951346024620462CF0C2F904B070BD77
:10F540000648F5E72B46314604B0BDE87040FFF7AA
:10F550003DBD00BF40CC00203481002060C20B00C4
:10F56000A0F6A860FFF7CEBF30B4094D95F8A441CE
:10F5700054B195F89F423CB1012480F8354F80F892
:10F58000984830BC28F0BABB002030BC704700BFA0
:10F5900040CC00200D4B03F1080210B5026003F1CE
:10F5A000500268330446C0F8A82EC0F8083F00F6A1
:10F5B000087000F0F5FD064B236004F6A46000F02F
:10F5C000CDFC204628F0DAF9204610BDCC640B00B3
:10F5D000BC150C00A0F60870DCE700BF10B50446AF
:10F5E000FFF7D8FF204640F638716AF0BDFC204690
:10F5F00010BDA0F60870F1E770B50446394E26F04C
:10F60000FFFE394B23604FF401720021C4F8886675
:10F6100004F28C60002580F041FD012384F89838C5
:10F620004FF401722946C4F89058C4F8945804F66F
:10F63000990080F033FD4FF40072294604F52A60EA
:10F6400080F02CFD4FF40172294604F54A6080F0E9
:10F6500025FD04F6A46000F061FC244BC4F8A83E2C
:10F660002A46234B2349C4F8AC5EC4F8B06EC4F8F4
:10F67000B45E04F6087000F0C7FD1F4B236003F171
:10F680004802C4F8A82E60331C4AC4F8083F03237C
:10F6900084F88436136884F8355F2BB1184B194A07
:10F6A0001948382149F0B2FA84F898384FF4E1311A
:10F6B00030461460F7F73AFF68F06CFE05463046B6
:10F6C000F7F764FF48B941F2883128462CF075F904
:10F6D00018B1642068F069FEF1E720462CF0D0F8FC
:10F6E000204670BD746C0020BC150C0018640B0023
:10F6F000907F002080640B00D4640B00407F0020CA
:10F700008E640B0097640B00B6640B0008B540F6DE
:10F71000387049F099F9FFF76FFF044B1868BDE89E
:10F72000084000F6A860FFF7D2BB00BF407F002072
:10F730000148F7F7BFBE00BF746C002010B5034B43
:10F740000360044600F02CFD204610BDFC650B0054
:10F7500010B50446FFF7F2FF20464FF4D4716AF06B
:10F7600003FC204610BD000038B50446154679BBA1
:10F770002A4B2B491868134600F6A860294AFFF760
:10F7800053FDD4F84431284A2B44C4F8443113685B
:10F790003C212B441360D4F83C31B3FBF1F2B2FBB3
:10F7A000F1F301FB132304EB83039A6C2A449A645C
:10F7B000D4F83C310A22B3FBF2F30622B3FBF2F099
:10F7C00002FB103304EB8304226B2A44226338BD0E
:10F7D000012912D1114B12491868134600F6A8608E
:10F7E000124AFFF721FDD4F86431114A2B44C4F8C2
:10F7F000643113682B441360DAE70229D8D1074B30
:10F8000007491868134600F6A8600A4AFFF70CFD7E
:10F81000D4F884312B44C4F88431C9E7407F0020F8
:10F820006C5C0B0054650B00687F002064650B0066
:10F83000487F002074650B0070B54FF46162D0F80A
:10F840003C31B3FBF2F390F8A42103F007039A4292
:10F8500004462CD0164A17491068174A00F6A860CB
:10F86000FFF7E2FC1548164904F5AE72072352F87B
:10F8700004599560566A9662566C966440F8235017
:10F88000556A41F82350013BF1D1C4F84431C4F822
:10F890006431C4F8843103600B604FF46162D4F8C2
:10F8A0003C31B3FBF2F303F0070384F8A43170BDDD
:10F8B000407F00206C5C0B008E650B00687F002091
:10F8C000487F00202DE9F041D0F83C5190F8388174
:10F8D000062201350A26B5FBF6F3B3FBF2F602FB6E
:10F8E00016360446C0F83C51F7B2B8F1000F1DD1EE
:10F8F000FFF7A2FF94F83931BB421EBF0C3684F8E3
:10F90000397144F826803C22B5FBF2F5B5FBF2F3E1
:10F9100002FB135594F83A21EBB29A421FBF1235FD
:10F9200084F83A31002344F825301DE000F1480204
:10F9300000F59C71002342F8043B8A42FBD1C4E9E4
:10F940000C33C4E90E33C4E9103304F5B27104F585
:10F95000A273002243F8042B8B42DA61DA63F9D1F7
:10F9600084F8382184F839714FF47A70BDE8F08159
:10F9700000F130020023483052F8041B82420B444D
:10F98000FAD107EE903A9FED057AF8EE677A87EEA6
:10F99000870ADFED037A20EE270A704700606A4786
:10F9A0000000C84200F14802002300F59C7052F8A4
:10F9B000041B82420B44FAD107EE903A9FED057A80
:10F9C000F8EE677A87EE870ADFED037A20EE270AE2
:10F9D000704700BF00BA5B4A0000C84210B5B9B119
:10F9E00090F84141FFF7C4FF07EE904AF8EEE77A3E
:10F9F000B4EEE70AF1EE10FA0DD4084B084A186885
:10FA0000084900F6A8602346FFF70EFC002010BD51
:10FA100090F84041E6E70120F9E700BF407F002071
:10FA2000B3650B00D9610B001A4B37B593F8C4418D
:10FA3000054654BB184BDFED196A1B6893ED036A4A
:10FA4000B4EEE66AF1EE10FA22D5FFF7ABFF95F8B7
:10FA5000423107EE903AF8EEE77A67EE867A87EE63
:10FA6000A67AB4EEC70AF1EE10FA11D40C4B17EED9
:10FA7000100A1D687EF0F6FF05F6A865CDE90001C5
:10FA8000084A09492846FFF7CFFB204603B030BD9E
:10FA90000124FAE740CC002048D900200000C842E9
:10FAA000407F0020CD650B00D9610B009FED0E7AE1
:10FAB00000F59A723B231146D1ED007AF8EE677A91
:10FAC000043AC7EE876AD8B230EE660AB4EEE00AAE
:10FAD000F1EE10FA03D5C0F13B00C0B27047013B14
:10FAE000E9D23C20704700BF00A00C4710B5154B71
:10FAF00015490446002200F087FB2046134B40F8CE
:10FB0000303B1822002180F0C9FAF022002104F1D4
:10FB1000480080F0C3FA0123A4F8383141F62813D5
:10FB20000021A4F84031322384F83A11C4F83C1182
:10FB300084F84231642204F5A27080F0AFFA2046C6
:10FB400010BD00BF907F0020EB650B00FC650B0033
:10FB500030B4826904695510034604EB6200D20791
:10FB600048BF62595B6930BC48BFD3581847000092
:10FB700008B5164B93F85D305A1E012A17D9042B8D
:10FB800015D00B791D2B10D8092B10D90A3B132B3C
:10FB90000DD8DFE803F00E0E11110C0C0C11111131
:10FBA000110C0C0C140C0C140E0EAF2B0AD00020F0
:10FBB00008BD00F0C7F8FAE700F02CF9F7E700F00D
:10FBC00039F9F4E700F046F9F1E700BF40CC002036
:10FBD000124A70B50260124A00610023C0E9052391
:10FBE000C360104B1D68061DC0E9016604469DB147
:10FBF0000C2048F029FF3146856078F07DF9E368F4
:10FC00000133E3600C2048F01FFF2946846078F040
:10FC100073F9AB680133AB60204670BD38660B00EA
:10FC200071FB0200089F002038B50446006884423A
:10FC300004D0056848F02CFF2846F8E738BD0000DE
:10FC40002DE9F8438046154B58F8045F03600446DD
:10FC5000454515D0AF683E68B7420FD0B368D6F8B7
:10FC600000909C4208D1BB68013B3046BB6078F0F5
:10FC70004AF9304648F00CFF4E46EDE72D68E7E7BD
:10FC80002846FFF7D1FF00232846C4E90155E36069
:10FC9000FFF7CAFF2046BDE8F88300BF24660B00CB
:10FCA00010B50446FFF7CCFF204610216AF05CF93E
:10FCB000204610BD10B5034B03600446FFF7C0FF9C
:10FCC000204610BD38660B0010B50446FFF7F2FF62
:10FCD00020461C216AF048F9204610BD00000000B3
:10FCE0002DE9F843164D95F85D30013B012B0F4689
:10FCF0001ED9EB68E3B10FF24009D9E90089044647
:10FD00000026B74204F1080412DD54E90212287BF0
:10FD100067F08EFC54F8040C7EF092FE42464B468F
:10FD20007EF0F8FE7FF0CEF968F03FFB0136E8E7A1
:10FD3000BDE8F883AFF30080CDCCCCCCCCCCF43F85
:10FD400040CC002007B5064A92E803006B4683E8E2
:10FD5000030001211846FFF7C3FF03B05DF804FB61
:10FD600044660B0007B5064A92E803006B4683E839
:10FD7000030001211846FFF7B3FF03B05DF804FB51
:10FD80004C660B0030B5074D0FCD87B06C460FC4E5
:10FD900095E8030084E8030003216846FFF7A0FF0D
:10FDA00007B030BD54660B0030B5074D0FCD87B09E
:10FDB0006C460FC495E8030084E8030003216846FD
:10FDC000FFF78EFF07B030BD6C660B0030B5074DF6
:10FDD0000FCD87B06C460FC495E8030084E803009C
:10FDE00003216846FFF77CFF07B030BD84660B0037
:10FDF00030B5074D0FCD87B06C460FC495E80300B2
:10FE000084E8030003216846FFF76AFF07B030BDAE
:10FE10009C660B0007B5064A92E803006B4683E830
:10FE2000030001211846FFF75BFF03B05DF804FBF8
:10FE3000B4660B0007B5064A92E803006B4683E8F8
:10FE4000030001211846FFF74BFF03B05DF804FBE8
:10FE5000C4660B0030B5084D0FCD8DB06C460FC495
:10FE60000FCD0FC495E80F0084E80F000621684607
:10FE7000FFF736FF0DB030BDEC660B0010B5032266
:10FE800004460021012068F0E5FB206028B9044BFE
:10FE9000044A05480C2148F0B9FE204610BD00BFB9
:10FEA00084670B008E670B00CE670B0010B504460D
:10FEB000006868F031FE204610BD10B54FF47A722C
:10FEC000044600238802890D7FF0CAFA01462068A3
:10FED00068F052FD003818BF012010BD00230068F3
:10FEE0001A46194668F0DCBB006868F0A1BC10B582
:10FEF0000446FFF7C3FF204610BD10B50446FFF7C8
:10FF0000D5FF204610BD08B5FFF7D7FF80F00100F0
:10FF1000C0B208BDFFF7E2BFFFF7E6BF10B503228E
:10FF200004460021012068F095FB206028B9084BA9
:10FF3000084A09480B2148F069FE00231A46194671
:10FF400068F0AEFB08B97FF051FC204610BD00BF41
:10FF5000FA670B0001680B001B680B0010B5044624
:10FF6000006868F0D9FD204610BD08B500684FF064
:10FF7000FF3168F001FD08B97FF038FC08BD08B515
:10FF8000002300681A46194668F08AFB08B97FF01A
:10FF90002DFC08BD10B5044608462160FFF7E5FFBB
:10FFA000204610BD10B504460068FFF7E8FF204664
:10FFB00010BD000070B505460E4610467AB12B689C
:10FFC00001241B682C75284600219847084B1C709B
:10FFD000BFF35B8F20462E63BFF35B8F70BDBFF313
:10FFE0005B8F2B6BBFF35B8F002BE8D0F6E700BF76
:10FFF0002AA1002010B5FFF7DDFF044610B102482A
:020000023000CC
:10000000FFF788FF204610BD3C81002038B50D4623
:1000100011461A46FFF7CEFF044618B1024829469A
:10002000FFF77AFF204638BD3C81002070B50E46B0
:1000300011461A460546FFF7DDFF044618B1314662
:10004000284600F0C3F8204670BD10B4034600F106
:1000500030020024BFF35B8F52E8001F42E8004CDF
:10006000BCF1000FF8D1BFF35B8F21B11B685DF8C5
:10007000044B1B6A18475DF8044B704708B5002213
:100080000275FFF7E2FF4FF0FF3008BD08B50368C7
:10009000002202751B686FF0004198476FF0004026
:1000A00008BD000037B504464CF04DFA174B1B78DD
:1000B00005464BB140B1164B164A18681649E3691C
:1000C00000F6A860FFF7B0F8144B1B786BB1237DE6
:1000D0005BB155B90E4B124A1868636800930E491C
:1000E000E36900F6A860FFF79FF80E4B1B7853B149
:1000F000237D43B9064B0C4A18680749E36900F6AB
:10010000A860FFF791F8284603B030BD3881002081
:10011000407F002060680B006C5C0B003081002089
:100120006F680B003181002083680B0070B5036895
:100130000A4DDB69286004469847064668F02AF9AC
:10014000014620464CF0FAF9002E04DB23683146C4
:100150001B682046984700232B6070BD3481002027
:1001600010B5044B044640F81C3B67F032FE2046B5
:1001700010BD00BFF0100D0008B50549054867F037
:10018000E5FEBDE808400449044867F0DFBE00BF53
:1001900097680B00AC7F0020A6680B007C800020D5
:1001A000084B10B504460360806A10B121464CF03C
:1001B00072FA2046044B40F81C3B67F00AFE2046CA
:1001C00010BD00BF5C690B00F0100D0010B50446B7
:1001D000416068F0DFF863681844E06010BD00001B
:1001E00008B5054B1B782BB9044B054A05488D21F2
:1001F00048F00CFD08BD00BF8C7F0020B6680B00E6
:10020000C3680B00E5680B0070B504460D4600217D
:100210001E464CF059F90D4B2360002384F82C3016
:10022000A662FFF7DDFF294604F11C0067F08EFE91
:10023000A06A48B121464CF0F4F928B9044B054AAC
:100240000548262148F0E2FC204670BD5C690B00A1
:1002500002690B0008690B00E5680B0038B5104C0B
:10026000104D002120464CF025FA20460E4C0F4A36
:10027000294677F03CFE002120464CF01BFA204630
:100280000B4C0A4A294677F032FE2046FFF72FFE34
:100290002046064A0749BDE8384077F028BE00BF2F
:1002A000907F00206101030060800020006000203A
:1002B0003C810020FBFE020070477047094B82B072
:1002C0001A88ADF804209DF804209B78002062F382
:1002D00007009DF8052062F30F2063F3174002B07A
:1002E000704700BF4081002000207047094B82B05A
:1002F0001A88ADF804209DF804209B78002062F352
:1003000007009DF8052062F30F2063F3174002B049
:10031000704700BF4081002000207047024A026001
:1003200000220271704700BF90690B0007B5027987
:10033000B2B1144B1A889B78ADF800208DF80230CA
:100340009DF80030002063F307009DF8013063F34F
:100350000F209DF8023063F3174003B05DF804FBF3
:100360000368094A5B690192042101AA9847C0F316
:1003700007238DF80000C0F307408DF801308DF899
:100380000200DDE7408100200102040307B50B4BAA
:100390000193036801AA5B69042198470022C3B254
:1003A00063F30702C0F3072363F30F22C0F307438D
:1003B00063F31742104603B05DF804FB0506070817
:1003C0001FB50D4B029344F23F73ADF80C30036838
:1003D00002AA5B69062198470022C3B263F30702B1
:1003E000C0F3072363F30F22C0F3074363F31742FD
:1003F000104605B05DF804FB090A0B0C1FB50F4A47
:1004000004465168106801AB03C31189927A1980C0
:100410009A70236801AA5B690B2120469847002245
:10042000C3B263F30702C0F3072363F30F22C0F3E1
:10043000074363F31742104604B010BD7C690B00FC
:1004400007B522238DF8003003686A465B690121F5
:1004500098470022C3B263F30702C0F3072363F394
:100460000F22C0F3074363F31742104603B05DF851
:1004700004FB000007B50B4B0193036801AA5B69FD
:10048000042198470022C3B263F30702C0F3072395
:1004900063F30F22C0F3074363F31742104603B020
:1004A0005DF804FB23573C580170427070470022EE
:1004B00002704270704702780B781AB9181E18BF84
:1004C0000120704733B140784B7898422CBF002010
:1004D000012070471846704782B00170ADF80420C3
:1004E000BDF80420A0F8012002B07047044A0023A0
:1004F00013705370034A137053709370704700BFAA
:10050000438100204081002038B50446006820B1B6
:10051000056848F0BDFA2846F9E7204638BD0000D6
:1005200010B5064B03600446082048F08DFA044BD2
:1005300044601A6802601860204610BDB0690B0064
:100540004881002038B5064B1C68054634B1606808
:10055000036829461B6898472468F7E738BD00BF41
:10056000488100200348044A04490023036077F0CF
:10057000BEBC00BF488100200060002009050300C8
:10058000036810B45C680023A4461A465DF8044B67
:100590006047C069704710B5836A2430024633B1A2
:1005A0001C7C8C422ABF1A46DB689B68F7E79042A6
:1005B00003D0137C8B4288BF0246801A18BF0120EB
:1005C00010BD0368C9B21B68184710B500238B42E1
:1005D00004DAC45C944203D00133F8E7002010BD74
:1005E0000120FCE72DE9F041174696B02C220C467D
:1005F00041F2D043002106460DEB0200ADF8003079
:100600000A917FF04BFD3946204649F022FA2368D3
:1006100002225B68694620469847204649F081FAE5
:10062000054638B11E49304667F018FC304616B012
:10063000BDE8F081142067F0B8FE3022394620462C
:1006400049F004FA3028EDD10AAFB84623682046B5
:10065000DB68984740B1236820461B6998470135FD
:10066000302D08F8010BF1D1002421461D2202A8EB
:1006700001947FF013FD01AB19463A78A2F12000F6
:100680005E28D0D81A707A78A2F120005E28CAD8E5
:100690000234202C5A70C6D003370233EDE700BF76
:1006A00060C20B00014882B002B07047604E01206A
:1006B00007B5064A034610680091054A054900F649
:1006C000A860FEF7B1FD03B05DF804FB407F002099
:1006D000B4690B002D5E0B0038B504304368024648
:1006E0003BB11D7C0C78A5422ABF1A46DB689B688B
:1006F000F6E7904203D00978137C994202D203486E
:1007000077F0A5FD02F1110038BD00BFCD690B00E7
:1007100030B585B004468DF8071000F1380103A804
:10072000FFF738FC9DF8075023682946DB68204610
:100730009847F8B10DF1070104F12000FFF7CCFF55
:1007400003784278294643EA022202A8FFF7C4FE52
:1007500003A8FFF727FC9DF80830002063F307008B
:100760009DF8093063F30F209DF80A3063F31740BA
:1007700005B030BD034B1A889B78ADF808208DF882
:100780000A30E5E740810020F0B585B00E46054609
:1007900000F1380103A81446FFF7FCFB2644B442DD
:1007A00030D014F8017B2B688DF80370DB68394674
:1007B000284698470028F2D00DF1030105F12000EA
:1007C000FFF78AFF03784278394643EA022201A8FC
:1007D000FFF782FE019BADF808301B0C03A88DF8D3
:1007E0000A30FFF7DFFB9DF80830002063F30700B5
:1007F0009DF8093063F30F209DF80A3063F317402A
:1008000005B0F0BD024B1A88ADF808209B78E5E7EB
:10081000408100208B6870B5164604460D1D0122EC
:100820005BB130781A7C904234BF9868D8681D4616
:1008300034BF012200220346F2E792B1CA68AA42FD
:1008400003D1C4E90035204670BD284677F0B4FBDB
:100850003378027C9A424FF00003F2D3C4E90003DC
:10086000F1E72846F4E72DE9F0418D6804460F468C
:1008700090460E1D01205DB105F110014046FFF7C5
:100880001AFE18B1AB682E461D46F4E7EB68FAE78E
:10089000A0B1FB68B34204D1256066602046BDE884
:1008A000F081304677F088FB0546414605F110009F
:1008B000FFF701FE20B100232360EEE73546F4E7A1
:1008C000C4E90050EAE700002DE9F3410F462A4849
:1008D00049781C46154649F0BCF8B978264848F0D6
:1008E00096FF3CB100212448FFF76BFE224800210F
:1008F000FFF767FE204849F014F9142067F055FD12
:1009000079781D482A4649F0A1F81B4848F07CFF39
:100910000128194818DD48F08FFF0446164848F0B2
:100920008BFF40EA042084B2DFF84C800026013DB2
:10093000F3B2AB4211DA404648F066FF10B14046D0
:1009400048F07AFF0136F3E748F05EFF18B10A4835
:1009500048F072FFE7E70446E6E7084B084A1868E4
:1009600008497B78009400F6A860FEF75DFC2046FD
:1009700002B0BDE8F08100BF604E0120407F002042
:10098000D5690B006C5C0B0073B5C1F30726ADF89D
:1009900004101546154831461C4649F05AF8FF2DFB
:1009A00003D91248290A48F032FF1048E9B248F04A
:1009B0002EFF0E4849F0B5F898B9142067F0F5FC01
:1009C00022460A48094D314649F040F8231A5C4254
:1009D0005C41284648F018FF20B1284648F02CFF1B
:1009E000F7E70024204602B070BD00BF604E012032
:1009F0002DE9F04F85B000242C4DDFF8C880DFF8DA
:100A0000C890ADF80C10C1F3072A032627465146BB
:100A1000284649F01EF80021284648F0F8FE2846EE
:100A200049F07FF801225146284649F00FF8284640
:100A300048F0EAFEA8B1284648F0FEFEC0B2802881
:100A400010D11B4B1B4A18681B49534600F6A8607F
:100A5000FEF7EAFB1E26304605B0BDE8F08F5F4684
:100A6000D5E73846430700F00F0B15D151464846ED
:100A7000FFF71EFE022601345F45E4B201D0042CCC
:100A8000EDD10B4B0D4A18680D4900945B4600F6FA
:100A9000A860FEF7C9FBDEE7ABF10303042BEAD83D
:100AA00051464046FFF704FE0126E4E7604E012070
:100AB000407F0020F4690B002D5E0B00246A0B00C0
:100AC0006C5C0B001C6A0B00156A0B002DE9F04FE3
:100AD0002DED028B984EDFF8908297B00C460546BC
:100AE00000F1380109A808EE902A0393FFF752FAA3
:100AF0003068924A9249234600F6A860FEF794FBBC
:100B00000022214607A8FFF7CFFC08238DF81D30EF
:100B1000B1469DF81D20772A01F20C80039B83B11A
:100B200018EE900A1946FFF750FD002800F03186B4
:100B3000D9F800008249134600F6A860814AFEF702
:100B400073FB9DF81D10404648F083FF404648F077
:100B5000E8FF9DF81D30002840F08386A3F10D02C8
:100B60006A2A00F27586DFE812F032037306730614
:100B70009B0373063E030B05730673067306730629
:100B8000F6015E0317047306A302FF033803BE00D9
:100B90007E037E037E03780473067306A103730647
:100BA000A804CF03F3037306730673067104730678
:100BB0004403730673067306CA007306F9030B0435
:100BC0005F017306ED0373066B006B007306C400D0
:100BD00065016501AE0165012C022C0273067306E6
:100BE0001B06730673067306730673067306730695
:100BF00073067306730605047306A10073065D028F
:100C00007306730612057306A1027B027306830046
:100C100073061104EB04730673067306EF0573067F
:100C20005A055A059903A9027306730673067306DB
:100C300057027306730673067306730601010101FA
:100C400007992846FFF7D4FE0446002800F0A18546
:100C500005F1240BAF6A5E46002F00F045863B7C11
:100C6000A34236BFFB68BB6837463E461F46F3E7E4
:100C70009DF81C308DF84C305F238DF84D300423E7
:100C80008DF84E3013A9002301222846FFF71CFEE1
:100C900002289DF81D1004D12B48FFF709FD0C24F4
:100CA000D6E72A48FFF704FD0924D1E79DF81C3058
:100CB0008DF84C3055238DF84D3004238DF84E308F
:100CC00013A9002301222846FFF7FEFD9DF81D1001
:100CD00020B11F48FFF7ECFC4B24B9E71D48FFF794
:100CE000E7FC0A24B4E71C481F21FFF7E1FC0B24B2
:100CF000AEE71A483F21FFF7DBFC0424A8E79DF884
:100D00001C308DF84C3034238DF84D3090238DF805
:100D10004E3013A9002301222846FFF7D5FD9DF888
:100D20001D1020B90E48FFF7C3FC472490E70D487B
:100D3000FFF7BEFC0D248BE7407F0020456A0B00C7
:100D40006C5C0B00656A0B00776A0B00806A0B0015
:100D50008A6A0B00926A0B009A6A0B00A16A0B0068
:100D6000A86A0B00B06A0B00604E0120BDF81C3071
:100D7000ADF84C30D0238DF84E300122002313A95A
:100D80002846FFF7A1FD602823D019D878B355284D
:100D900026D0BDF81C30ADF84C3013A90023012239
:100DA00028468DF84E30FFF78FFD50289DF81D1016
:100DB00033D0602836D0CE48FFF77AFC102447E7BE
:100DC0006128E6D19DF81D10CA48FFF771FC0E247A
:100DD0003EE79DF81D10C848FFF76AFC0F2437E76F
:100DE0009DF81D10C548FFF763FC112430E7BDF8DE
:100DF0001C30ADF84C300D238DF84E3001220346E7
:100E000013A92846FFF760FD1028C2D19DF81D10D8
:100E1000BB48FFF74DFC44241AE7BA48FFF748FCEB
:100E2000122415E7B848F9E7B8483821FFF740FC25
:100E300034240DE7BDF81C30ADF84C30FE238DF89E
:100E40004E300222002313A92846FFF73DFD044639
:100E5000D9F80000AE4AAF49234600F6A860FEF775
:100E6000E3F945F249439C4226D1BDF81C30ADF868
:100E70004C30FF238DF84E300222002313A9284660
:100E8000FFF722FD0446D9F80000A249A24A2346F2
:100E900000F6A860FEF7C8F942F260239C429DF874
:100EA0001D1004D19D48FFF703FC4124D0E69C4867
:100EB000FFF7FEFB1324CBE69DF81D109948FFF7C2
:100EC000F7FB1424C4E69DF81C308DF84C30422307
:100ED0008DF84D30FE238DF84E300222002313A9E9
:100EE0002846FFF7F1FC0446D9F800008E4A8949EC
:100EF000234600F6A860FEF797F945F249439C4265
:100F000006D19DF81D108948FFF7D2FB15249FE6F6
:100F1000BDF81C30ADF84C3005238DF84E3006225C
:100F2000012313A92846FFF7CFFC0446D9F8000097
:100F30007F4A7849234600F6A860FEF775F945F226
:100F400005339C4240F025849DF81D107948FFF739
:100F5000AFFB36247CE69DF81C308DF84C3018230E
:100F60008DF84D3007238DF84E300222002313A94F
:100F70002846FFF7A9FCB0F5806F06D19DF81D103B
:100F80006D48FFF795FB172462E6BDF81C30ADF8FD
:100F90004C300F238DF84E300222002313A928462F
:100FA000FFF792FCB0F54C5F04D043F23333984224
:100FB00040F0EF839DF81D106048FFF779FB262471
:100FC00046E6BDF81C30ADF84C307E238DF84E302F
:100FD0000222002313A92846FFF776FC45F2494375
:100FE000984206D19DF81D105548FFF761FB31244A
:100FF0002EE60799062389222846FFF7C5FC9DF8AF
:101000001D1020B14F48FFF753FB192420E64E482E
:10101000FFF74EFB18241BE64C487021FFF748FBF6
:101020001A2415E69DF81C308DF84C3057238DF8A6
:101030004D30FF238DF84E3013A90023012228469E
:10104000FFF742FC15289DF81D1004D14048FFF71A
:101050002FFB3D24FCE53F48FFF72AFB2D24F7E555
:10106000079930234DF260022846FFF78DFC30B11E
:101070009DF81D103848FFF71BFB5824E8E5BDF824
:101080001C30ADF84C300F238DF84E300122034652
:1010900013A92846FFF718FCB12840F07A839DF881
:1010A0001D102E48FFF704FB1C24D1E55C21F8E756
:1010B0002B481C21FFF7FCFA1D24C9E59DF81C30C4
:1010C0008DF84C306B238DF84D300A238DF84E305F
:1010D0000122002313A92846FFF7F6FBC02843D1BD
:1010E0009DF81D101F48FFF7E3FA2824B0E500BF64
:1010F000F26A0B00BF6A0B00C66A0B00CD6A0B00D8
:10110000DB6A0B00E26A0B00EA6A0B00FA6A0B006A
:10111000006B0B006C5C0B00176B0B002E6B0B0055
:10112000356B0B003C6B0B00436B0B005D6B0B00D6
:10113000656B0B007F6B0B008C6B0B00946B0B00D3
:101140009B6B0B00A36B0B00A96B0B00AF6B0B0031
:10115000B56B0B00BE6B0B00C76B0B00CD6B0B00B0
:10116000D56B0B00DE6B0B00BDF81C30ADF84C30BE
:1011700014238DF84E300122002313A92846FFF7CF
:10118000A3FB00F00300022806D19DF81D10CE48F5
:10119000FFF78EFA4A245BE5BDF81C30ADF84C3001
:1011A0000F238DF84E3013A9002301222846FFF7A4
:1011B0008BFB6A289DF81D1004D1C448FFF778FA0C
:1011C000292445E5C248FFF773FA1F2440E5C148CA
:1011D0000D21FFF76DFA20243AE5BF481E21FFF7E5
:1011E00067FA212434E5BD481221FFF761FA232470
:1011F0002EE59DF81C308DF84C3030238DF84D30A5
:101200002F238DF84E300122002313A92846FFF723
:101210005BFB302840F0BD829DF81D10B048FFF701
:1012200047FA222414E59DF81C308DF84C30192320
:101230008DF84D300F238DF84E3013A90023022274
:101240002846FFF741FBB0F54C5F9DF81D103FF4B9
:10125000B3AE43F2333398423FF4AEAEA148FFF74A
:1012600027FA2724F4E4BDF81C30ADF84C300223F3
:101270008DF84E3013A9002301222846FFF724FBE6
:101280009DF81D10814204D19748FFF711FA4624BA
:10129000DEE49648FFF70CFA2A24D9E46A218CE7A9
:1012A00093481021FFF704FA2C24D1E49DF81C3058
:1012B0008DF84C30012426238DF84D302246002332
:1012C00013A928468DF84E40FFF7FEFA132814D1D3
:1012D000BDF81C30ADF84C3013A900232246284637
:1012E0008DF84E30FFF7F0FA81289DF81D1006D1D9
:1012F0008048FFF7DDF95224AAE49DF81D107E48CE
:10130000FFF7D6F92B24A3E49DF81C308DF84C3060
:1013100029238DF84D30B2238DF84E3013A90023C8
:1013200001222846FFF7D0FA50289DF81D1004D15D
:101330007248FFF7BDF930248AE47148FFF7B8F925
:101340004F2485E46F483A21FFF7B2F932247FE455
:101350006D482A21FFF7ACF9372479E46B48362130
:10136000FFF7A6F9162473E469481D21FFF7A0F9D9
:1013700043246DE467485321FFF79AF9452467E455
:1013800065483721FFF794F9482461E463486121F7
:10139000FFF78EF95A245BE4614E06244FF474770C
:1013A000013C9DF81D1024D040460A9748F051FB9F
:1013B00004220AA9404648F015FA404648F0B1FB1D
:1013C00068BB9DF81D100722404648F03FFB0722EE
:1013D00013A9404665F0E1FF9DF84E30CA2B1ED19F
:1013E0009DF84F30CA2B1AD19DF81D104D48FFF7BC
:1013F0005FF9BDF81C30ADF84C30AB238DF84E30A2
:1014000013A9002301222846FFF75EFAA9289DF8B8
:101410001D1016D14448FFF74BF9542418E49DF8E9
:101420001D101096404648F014FB042210A94046B7
:1014300048F0D8F9404648F074FB322066F0B5FF1A
:10144000AEE73A48FFF734F9492401E438482E2141
:10145000FFF72EF95324FFF7FBBB9DF81C308DF8E6
:101460004C3023238DF84D3086238DF84E3013A950
:10147000002301222846FFF727FA92289DF81D1025
:1014800005D12C48FFF714F94C24FFF7E1BB404687
:1014900048F0DFFA01214046FFF793F8404648F054
:1014A00040FB9DF81D30002840F0D28122481946AB
:1014B000FFF7FEF85124FFF7CBBB20482821FFF7A8
:1014C000F7F84D24FFF7C4BBE66B0B00EE6B0B0087
:1014D000F66B0B00FE6B0B00076C0B00106C0B0027
:1014E000196C0B00236C0B002A6C0B00336C0B0087
:1014F0003B6C0B00446C0B004A6C0B00526C0B00F5
:101500005B6C0B00636C0B006C6C0B00746C0B0061
:101510007D6C0B00906C0B00996C0B00A16C0B00A8
:10152000D0000400A76C0B00AF6C0B00B86C0B0074
:10153000BF6C0B00C66C0B00D06C0B00126D0B0067
:101540009DF81C308DF84C3062238DF84D30082307
:101550008DF84E3013A9002301222846FFF7B4F975
:1015600018289DF81D1005D1C148FFF7A1F859248E
:10157000FFF76EBBBF48FFF79BF83C24FFF768BB43
:10158000BD481321FFF794F84E24FFF761BB9DF887
:101590001C308DF84C305A238DF84D3006238DF8D1
:1015A0004E300122002313A92846FFF78DF9AB28FE
:1015B00002D19DF81D102DE7BDF81C30ADF84C3060
:1015C0000E238DF84E300122002313A92846FFF781
:1015D0007BF95A2807D19DF81D10A848FFF768F835
:1015E0003324FFF735BBBDF81C30ADF84C3013A9E0
:1015F0000023012228468DF84E30FFF765F9E028D8
:101600009DF81D1005D19E48FFF752F85024FFF7B2
:101610001FBB9C48FFF74CF83F24FFF719BBBDF8F0
:101620001C30ADF84C30002413A923460122284673
:101630008DF84E40FFF748F9EA289DF81D1005D1B6
:101640009148FFF735F83A24FFF702BB242805D16B
:101650008E48FFF72DF85624FFF7FABAD82805D19F
:101660008B48FFF725F83524FFF7F2BABDF81C3098
:10167000ADF84C3075238DF84E300122234613A966
:101680002846FFF721F9602807D19DF81D108148F1
:10169000FFF70EF83B24FFF7DBBA7F4910A866F08E
:1016A000DDFB9DF81D20414613A8FEF79BFF13A903
:1016B00010A866F043FC13A866F08BFB774913A8CB
:1016C00066F0CCFB13A910A866F087FD044613A8AA
:1016D00066F07FFB54B19DF81D107148FEF7E8FFDE
:1016E000572410A866F075FBFFF7B2BA6D4913A82E
:1016F00066F0B4FB13A910A866F06FFD044613A8AA
:1017000066F067FB1CB19DF81D106748E6E7674966
:1017100013A866F0A3FB13A910A866F05EFD0446AB
:1017200013A866F056FB9DF81D100CB16048D5E774
:10173000692904D15648FEF7BBFF3524D1E75D483F
:10174000FEF7B6FF2524CCE79DF81C308DF84C3011
:1017500066240023012213A928468DF84D408DF8F8
:101760004E30FFF7B1F87D2801D07A2807D19DF8D7
:101770001D105148FEF79CFF4024FFF769BAD9F8C5
:1017800000604E4A00904E49234606F6A860FDF7D9
:101790004BFD9DF81D3001338DF81D30FFF7B9B9B1
:1017A0004821404648F055F9464B18681B798DF89A
:1017B0002C30454B0A90186810901B798DF84430F6
:1017C00005220AA9404648F00DF8404648F0A9F91C
:1017D000052213A9404665F0E0FD052802460FD119
:1017E00013A910A87EF024FC50B9D9F80000374A9C
:1017F000374900F6A860FDF717FD4224FFF728BA25
:10180000BDF81C30ADF8203001238DF822300222C3
:10181000002308A92846FFF757F848F28353984257
:1018200003D048F28053984207D19DF81D102948F3
:10183000FEF73EFF5B24FFF70BBAD9F80000264AFB
:10184000234900F6A860FDF7EFFC3824FFF700BA43
:10185000D9F80000214A1E4900F6A860FDF7E4FC13
:1018600097E7042895D1D9F800001D4A1D49F3E7F0
:101870001B6D0B00226D0B00286D0B002F6D0B00F4
:10188000386D0B00406D0B00496D0B00526D0B0065
:10189000596D0B00606D0B0060C20B00FDA00C00C9
:1018A0006C6D0B00DDA00C007C6D0B00BDA00C006E
:1018B0008C6D0B009C6D0B00A46D0B00B96D0B00C3
:1018C0006C5C0B004E6E0B00536E0B00EE6D0B004C
:1018D0002D5E0B000A6E0B00166E0B00D76C0B0012
:1018E000306E0B009B5C0B00B34502D0337CA342EF
:1018F00035D905F120011420049147F0A5F800F135
:1019000010020474824611300292FEF7D0FDB345F6
:10191000029A049939D16B6B2BB1286B9AF810306D
:10192000067C9E4208D30CA8FEF774FFDDE90C602C
:10193000002869D0002E65D1834563D09AF81060E5
:10194000037C9E422CBF002601265B460246514680
:10195000304676F033FB6B6B01336B635646BDF854
:101960001C30A6F811302F6905F10C0302931E46B6
:10197000002F51D007A907F11000FEF79CFD0028A9
:1019800047D1BB683E461F46F2E79AF81030307CDC
:1019900002918342CDE9043219D2EF6ABE420BD0E4
:1019A000304676F009FB049B077C0299059A9F421A
:1019B00005D2C7684FB9064630463E46B8E70CA880
:1019C000FEF728FFDDE90C76F6E73746F4E71BD98A
:1019D000286B8642F1D0304676F0DBFA049B029900
:1019E000059A0746007C984204D9F36843B930460B
:1019F0001F46E2E70CA8FEF70DFFDDE90C70DCE7FF
:101A00003846DAE70126A0E7504647F041F8B246EB
:101A1000A4E7FB683746B5E7029BB34220D105F146
:101A20000803142008EE103A47F00EF8BDF81C30F9
:101A3000038200238374029BB342824600F1100BA1
:101A400017D1EB6983B3A86959461030FEF733FD0F
:101A500050B3AE699EBB504647F01AF8B2463EE01E
:101A600006F1100107A8FEF726FD0028D7D1B474AF
:101A70008FE606F11003194658460493FEF71BFD46
:101A8000049B80B36F69BE4216D0304676F094FA5C
:101A90005946034610300493FEF70DFD20B1049B18
:101AA000DF68F7B91E4607E018EE101A5A460EA86E
:101AB000FEF7D9FEDDE90E76002E39D0B7BB029BCA
:101AC000B34233D006F110015846FEF7F4FC029BF6
:101AD0003246514676F072FAEB690133EB615646B5
:101AE000C5E73746E8E759461846FEF7E4FC002804
:101AF000B1D0AB699E42D5D0304676F04AFA07465F
:101B000000F110015846FEF7D6FC20B1F16859B932
:101B100033460F46C6E718EE101A5A460EA8FEF7CF
:101B2000A2FEDDE90E73BDE73B46BBE70120CEE731
:101B30003E4690E709A8FEF735FA17B0BDEC028BD8
:101B4000BDE8F08F002370B502221D468E1E96421E
:101B500007D9845C2C4453FA84F3E5B2DBB201323A
:101B6000F5E70144855501F8013C70BD90F8E001AE
:101B7000013804288CBF002001207047D0F8DC0118
:101B8000003818BF0120704730B4826904695510CD
:101B9000034604EB6200D20748BF62595B6930BC60
:101BA00048BFD358184730B48269046955100346BA
:101BB00004EB6200D20748BF62595B6930BC48BF82
:101BC000D3581847074B084A084910B50446186807
:101BD00000F6A860FDF728FB236820469B6998471C
:101BE000002010BD407F0020786E0B002D5E0B00A2
:101BF00008B5034A034B0448592147F007F800BFD2
:101C0000886E0B00CD5C0B00BA6E0B00000000006C
:101C10000B6DF0B523F07F42036D23F07F439A42B2
:101C20008FB004460D4629D18A6D836D9A4225D125
:101C30000A6E036E9A4221D18A6E836E9A421DD13A
:101C4000D1F88020D0F880309A4217D1D1F88C207A
:101C5000D0F88C309A4211D1D1F8A820D0F8A83011
:101C60009A420BD1D1F8A020D0F8A0309A4205D1E9
:101C7000D1F8B420D0F8B4309A420ED0636F53B18B
:101C80006A6F934207D1464B464A1868464900F6A8
:101C9000A860FDF7C9FA012600E00026012395F8A7
:101CA000507084F8203095F8513084F8507084F8E2
:101CB0005130742205F1540104F154007EF0C6F94C
:101CC000002E5ED0364D002F53D066F063FBD4F863
:101CD000B430C4F8C800D4F8A0002D680C937CF090
:101CE0009FFE29A3D3E900237CF014FFCDE90A016C
:101CF000D4F8A8007CF094FE25A3D3E900237CF05F
:101D000009FFCDE90801D4F88C007CF089FE1EA300
:101D1000D3E900237CF0FEFEA36E0493CDE9060117
:101D2000206E7CF08DFE1CA3D3E900237CF0F2FE34
:101D3000CDE90201A06D7CF083FE17A3D3E9002357
:101D40007CF0E8FE05F6A865CDE90001636F174A4F
:101D500017492846FDF768FA264656F8285FB54227
:101D60000FD0A868036821469B68984748B92D683A
:101D7000F5E728680F4A0E4900F6A860FDF754FA07
:101D8000EAE700200FB0F0BD7B14AE47E17A843F54
:101D9000F168E388B5F8E43E48AFBC9AF2D77A3EE2
:101DA000407F0020CA6E0B009B5C0B00016F0B0094
:101DB0006C5C0B004F6F0B0010B50446006810B14F
:101DC00003681B699847204610BD000038B5074DD1
:101DD00028680368DB6898470446013C04D32868F8
:101DE00003681B699847F8E738BD00BF846100208D
:101DF0002DE9F84F90F80732054633B1FFF7E6FFBB
:101E00004FF0000A5046BDE8F88F274E306803684F
:101E1000DB68984740F6FE7398420FDD234B30682D
:101E20001C680368DB68984704F6A8640346204AE8
:101E300020492046FDF7F8F9FFF7C8FF4FF0000AE8
:101E4000DFF87490544605F1B80705F50A78306854
:101E50000368DB6898470028D4DD306803681B6995
:101E600098472B19C1B2834683F8281238464AF0A6
:101E7000ADFAF02C4AEA00005FFA80FA02D8BBF112
:101E80000D0F0ED12246494640461CF035FF044650
:101E90000028DCD0D5F824330133C5F824330024DE
:101EA000D5E70134D3E700BF84610020407F0020E4
:101EB0005B6F0B00D9610B009C6F0B0013B50446E0
:101EC000084659B101917FF003FC236801995B68D2
:101ED0000246204602B0BDE81040184702B010BDCF
:101EE00038B580F82A12C11880F82B2246F2B524A2
:101EF0000022049DA0F8284280F82C3280F82D2280
:101F000081F82E2281F82F2200F22E21934204DD47
:101F1000AC5C01F8014B0132F8E703F108042146FB
:101F200000F50A70FFF70EFEE0B238BDF0B5C51837
:101F30004CF6BA64A0F82842059E80F82A320024A4
:101F400080F82B4280F82C1280F82D2285F82E4242
:101F500085F82F4285F8304285F8314200F22E256F
:101F6000A34204DD375D05F8017B0134F8E703EB9C
:101F7000014101EB026203F0FC0100F50A74014427
:101F8000814204D0D0F82E5204302A44F8E7E118F8
:101F9000100A8A71C871100C120E08720A334A7244
:101FA000D8B2F0BD2DE9F0410024ADF5407D1646D4
:101FB0000D464FF43F72214601A800947EF06EF862
:101FC00066F0E8F9144F064440F2FF2866F0E2F9A3
:101FD000B0421ED238680368DB6898470028F5D005
:101FE000386803681B699847C3B20DF804300134A0
:101FF000444501D00D2BE9D12246294668461CF004
:102000007BFE20B103200DF5407DBDE8F081044644
:10201000DCE70020F7E700BF846100202DE9F043F2
:1020200085B000240D461646984666F0B3F9CDE912
:102030000044DFF8A49002940746ADF80C404146F6
:10204000384629F0BAFCB0B3D9F800000368DB6861
:102050009847E0B1D9F8000003681B699847631CF2
:1020600004AADBB21444022B04F8100C10D19DF822
:1020700000109DF80120BA2901D1CE2A05D00023F5
:102080008DF801308DF8002001231C46D7E7234648
:102090000D2BFAD19DF80430052B14D19DF80510B5
:1020A0009DF806209DF80730012907D1AA420AD1E0
:1020B000B34208D1032005B0BDE8F08319B9AA42A4
:1020C00001D1B34206D00E22002168467DF0E6FF22
:1020D0000023DAE70120EEE7846100202DE9F047D4
:1020E0009846424B8CB018689B88ADF80C300023A2
:1020F0001646CDF80E300D46029066F04BF93C4B7B
:102100000DF10809074605AA03F1180C186859686B
:10211000144603C4083363452246F7D119889B78D7
:10212000A3700023218002221C4619F802100132FC
:10213000214453FA81F3062ACCB2DBB2F5D12C4408
:1021400056FA84F2D2B253FA84F414444FF0000ADF
:10215000DFF8AC908DF811408DF80E508DF80F60BF
:102160008DF8102054464146384629F026FC0028B8
:1021700037D0092C38D8D9F800000368DB689847B5
:102180000028F0D0D9F8000003681B6998470CAB11
:102190005344C0B213F81C3C834208D10AF1010A2F
:1021A000BAF11A0F05D102201BE00024DBE74FF043
:1021B000000A0CAB234413F8283C834202D10134BB
:1021C000E4B2D0E7032CF0D10028EED1094B0A4A43
:1021D00018680A49009600F6A8602B46FDF724F817
:1021E00001200CB0BDE8F0870320FAE7447E0B0025
:1021F000EE6F0B00407F0020CA6F0B00D9610B000F
:10220000846100202DE9F74F0E469DF830A0019221
:10221000994666F0BFF84FF00008284D0746C346C0
:102220000D99384629F0C9FB002844D02868036876
:10223000DB6898470028F3D0286803681B69984733
:10224000BBF1050FECD8DFE80BF0060D141B2227BD
:102250004FF0000BE4E7A0F1B503D3F1000B4BEB1B
:10226000030BDDE7622814BF4FF0000B4FF0020BA9
:10227000D6E781450CBF4FF0030B4FF0000BCFE7C3
:1022800082450CBF4FF0040B4FF0000BC8E71FFA5C
:1022900080F84FF0050BC3E7019B48EA00201FFAC6
:1022A00080F89845D4D228684246314665F075F8E2
:1022B0008045CDD1404603B0BDE8F08F8461002059
:1022C000D0F8A40003681B681847000038B504461E
:1022D0000D460020012168F063FF85F00101002018
:1022E00068F0C6FF94F8B4000A2201211CF078FDC2
:1022F00020B1034B03491868FFF7E0FD38BD00BF6C
:102300008461002009700B00F0B5062385B00F46EC
:102310000521CDE90113042300930646144690F8E5
:10232000B400032302221CF05BFD002843D0234DA0
:102330004FB128680368FF211B68984705B0BDE8C6
:10234000F040FFF743BD44B9304622460121FFF774
:10235000DBFF4FF4FA7066F028F896F8B460184B7B
:10236000062EE7B2C4F30721C4F3074218684FEA08
:1023700014641E4617D1134B1F7159719A71DC7189
:102380000093102341220221FFF7AAFD2B68316838
:102390001A68546801F50A7102461846234605B0CA
:1023A000BDE8F0401847084B1F7059709A70DC70F8
:1023B00000930823E6E705B0F0BD00BF846100206C
:1023C000A4820020746100206C6100203C4BF7B5B2
:1023D00090F8077280F8071204461868042F0D461B
:1023E000164600F6A86004D8364A042952F8273069
:1023F00001D9FFF7FDFB52F8212000923249334A00
:10240000FCF712FF032D35D0042D3CD0022D1FD038
:10241000002F52D00025012F84F8F0514DD0FFF746
:10242000D5FC2B4B2B4A18684FF40061FCF724FDB8
:1024300001212046FFF744FF29462046FFF746FFCB
:102440002A460121204603B0BDE8F040FFF75CBFFB
:102450001F4B204A18684FF40061FCF70EFD012164
:102460002046FFF72DFF01212046FFF72FFF3246C0
:102470000021E7E7164B174A18684FF40061FCF794
:10248000FCFC0021ECE736B1134B144A144840F22F
:10249000653146F0BBFB0E4B0E4A18684FF40061E5
:1024A000FCF7EBFC31462046FFF70AFF01212046EE
:1024B000FFF70CFF32463146C4E703B0F0BD00BF62
:1024C000407F0020607E0B002D5E0B0019700B001A
:1024D000987E002060C20B003C700B004B700B001C
:1024E000BA6E0B0038B5036800251B6805750446F5
:1024F0006FF00041984720462A460421FFF766FF07
:102500006FF0004038BD90F8043223B9012380F801
:10251000043280F80332704710B50446044802F0D4
:102520003DFD002220461146BDE81040FFF74EBF9A
:1025300054610020000000002DE9F04390F80232C1
:10254000044685B038484BB302F012FE3648DFF837
:10255000EC9002F02DFE0646334802F04DFD334B61
:102560000546D86E1DF078FB0746D9F80000304AC2
:1025700030494FF47A7800F6A860B5FBF8F3FCF721
:1025800053FE42F210739F4200D955B90022012137
:10259000204605B0BDE8F043FFF718BF02F004FD88
:1025A000D4E705210623CDE9011304230222009379
:1025B00094F8B40003231CF013FCB6FBF8F07CF095
:1025C0002FFA9FED151B41EC100B77F009FB14A3BC
:1025D000D3E9002351EC100B7CF09CFA7CF072FDE7
:1025E0000646D9F80000144A1249B6FBF8F300F683
:1025F000A860FCF719FEB7422A4601D20221C7E7BC
:1026000003212046FFF7E2FE002384F8E03105B005
:10261000BDE8F083AFF3008085EB51B81E85F33F32
:1026200000000000007CA5405461002040CC002048
:102630007C700B006C5C0B0092700B00407F0020E4
:1026400010B504460C3065F0C4FB204665F0C1FBB4
:10265000204610BD1B02B3F5961F2DE9F74F8846A3
:1026600017465EDB4FF4165593FBF5F5B5F5006F95
:10267000A8BF4FF40065284646F0F8F9064665F015
:1026800089FEDFF8D0A081460024013D65F082FE7E
:10269000A0EB0900404554D2DAF800000368DB687B
:1026A00098470028F2D0DAF8000003681B699847C1
:1026B000AC42C0B205DA631C9BB200223055F25422
:1026C0001C462C280AD0012CE0D9331913F8022C0F
:1026D0000D2A2AD113F8013C0A2B26D1D7E9003262
:1026E00093429B4601921ED0D968009330467FF0FA
:1026F00060F8009B019A1C330028F1D0124B134A5A
:1027000018681349DBF8003000F6A860FCF78CFD70
:102710009BF81840304646F0BDF9204603B0BDE8AE
:10272000F08F8025A7E7012CB0D9331913F8022CBC
:102730000D2AABD113F8013C0A2BA7D10024347029
:10274000A4E70824E6E700BF407F0020C9700B0023
:102750002D5E0B00846100202DE9F84F564B574F3A
:1027600093F978A093F97C603A68BAF1000F08BF3A
:102770004FF0070A002E804608BF06261AB90260ED
:102780004046BDE8F88F4FF44B7093F9889046F0BF
:102790005BF94B4B4B4904460022FDF735FD2046C3
:1027A000494B40F8303B7422002100257DF076FC37
:1027B0004FF0080B04F1A80304F1B800C4E92A3370
:1027C000C4F8A450C4F8B05084F8B4B049F061FA29
:1027D0004FF4FA63C4F8EC314FF08063C4F804326C
:1027E00004F50473C4E98433384BC4F80C32384B15
:1027F00084F8E051FA22294604F50A70C4E98835C4
:10280000C4F8E45184F8E85184F8F051C4F8F45164
:10281000C4F8005284F80852C4F81852C4F81C4294
:102820007DF03CFC0C20C4E97EA6C4F8245384F857
:10283000285346F009F9274B0360022306468560BA
:102840000371C4F8A400B9F1000F0DD0584646F04A
:10285000FBF8214B0546C0E900390C2046F0F4F89E
:102860002A463146FAF706F92046FFF755FE3B683F
:10287000FBB11A4DD4F8F8312868194A194900F605
:10288000A860FCF7D1FC2868D4F8FC31164A154939
:1028900000F6A860FCF7C8FC94F8F811386894F8C2
:1028A000FC2165F0F3F8386803684FF41651DB69D2
:1028B0009847C8F8004063E740CC002084610020BE
:1028C000907F0020BAA30B00E4800B00387E0B0041
:1028D000C51B0300745D0B008C5D0B00407F002066
:1028E000D5700B006C5C0B00EB700B0038B50B4D1A
:1028F0000446284602F078FB012323752368322121
:102900001B6820469847284602F048FB00222046D4
:102910001146BDE83840FFF759BD00BF54610020A3
:10292000164B93F88C20012A10B5044612D10022D0
:1029300083F88C20124B134A1868134900F6A860DC
:10294000FCF772FCFDF730FA236820469B69BDE86E
:10295000104018478AB9012283F88C20084B0B4A93
:102960001868094900F6A860FCF75EFCFDF70AFA52
:102970002046BDE81040FFF7B9BF10BD40CC002095
:10298000407F002001710B002D5E0B0024710B00B5
:102990002DE9F74302AB03E906000023C0E9003349
:1029A0008360019B1D4CDDF800901C265E430546AC
:1029B0001B4BB01044439C4209EB060702D919484F
:1029C00075F042FC1CB1304646F03EF80446264401
:1029D000AE602C60A0464E46B74210D0314640460D
:1029E00065F0A2FA06F10C0108F10C0065F09CFA02
:1029F000337E88F818301C3608F11C08ECE7A7EB8A
:102A000009070948BF08784320F040401C2303FB16
:102A1000004428466C6003B0BDE8F083B76DDBB6B8
:102A20002449920446710B00B76DDB3670B5D0E9CE
:102A300000560446AE4204D02846FFF701FE1C357E
:102A4000F8E7206808B146F023F8204670BD000082
:102A50002DE9F04F0546ADF2044D0E464FF43F729E
:102A6000002141A840917DF019FB95F8E841062C22
:102A700000F24984DFE814F0070043009B00E00007
:102A80004101E6016D02B14C206803685B6A98471A
:102A9000206803683146DB6998474FF4AB72002128
:102AA000AB487DF0FBFA642065F07FFCA949206803
:102AB000FFF704FA142065F078FCA7492068FFF7B7
:102AC000FDF9A6492068FFF7F9F9A5492068FFF745
:102AD000F5F9142065F069FCA2492068FFF7EEF9CA
:102AE000A1492068FFF7EAF9A0492068FFF7E6F955
:102AF0001423C5F8EC31012385F8E83155E20FAC19
:102B00009B49204665F0AAF90727994912A865F064
:102B1000A5F99849277616A865F0A0F9954919A84E
:102B200065F09CF9944984F834701DA865F096F915
:102B3000914920A865F092F90F2384F850300323BF
:102B40000494059304AA06CA0AAB0CA8FFF720FF59
:102B50001DA8FFF775FD16A8FFF772FD2046FFF7C9
:102B60006FFD864B864A1868864B8749009300F6AE
:102B7000A860864BFCF758FBFFF728F9734B844994
:102B80001868FFF79BF933460CAA4FF4FA712846F0
:102B9000FFF760FD0828044605D11423C5F8EC3181
:102BA000022385F8E8310CA8FFF740FFC8E00FAC1E
:102BB0007849204665F052F90027774912A865F058
:102BC0004DF97649277616A865F048F9744919A891
:102BD00065F044F902230694079306AA06CA0AABD5
:102BE00084F834700CA8FFF7D3FE16A8FFF728FD71
:102BF0002046FFF725FD614B614A1868694B624921
:102C0000009300F6A860684BFCF70EFBFFF7DEF8B8
:102C10004E4B66491868FFF751F933460CAA4FF43A
:102C2000FA712846FFF716FD08280446BBD1142385
:102C3000C5F8EC310323B4E7444F5D493868FFF72A
:102C40003DF95C4938680FACFFF738F95A493868E4
:102C5000FFF734F95949204665F000F9584912A8A0
:102C600065F0FCF80C232376564916A865F0F6F8B3
:102C70004FF00D08544919A865F0F0F8534984F84D
:102C800034801DA865F0EAF8514920A865F0E6F8FF
:102C900003230894099308AA06CA0AAB84F8508053
:102CA0000CA8FFF775FE1DA8FFF7CAFC16A8FFF7D2
:102CB000C7FC2046FFF7C4FC304B314A1868454B2F
:102CC0003149009300F6A860434BFCF7ADFAFFF7DB
:102CD0007DF842493868FFF7F1F833460CAA4FF403
:102CE0007A712846FFF7B6FC082804467FF45BAFEC
:102CF0001423C5F8EC31042353E7204C384E2068E8
:102D0000124F384B1E4A2049009600F6A860FCF787
:102D10008BFAFFF75BF834493868FFF7CFF833498F
:102D20004FF4FA722846FFF73DF90328206863D173
:102D30002F4A3049334600F6A860FCF775FA0D2497
:102D400020460DF2044DBDE8F08F00BF84610020E5
:102D50004C81002077710B009E710B00BC710B0041
:102D6000DA710B00F8710B000D720B0022720B0070
:102D700037720B003E720B0044720B00407F002044
:102D800053720B0065720B006C5C0B004A720B00F7
:102D900074720B0092720B007F720B00AE720B000C
:102DA0009B720B00C4720B00B7720B00D4720B0045
:102DB000E3720B00F5720B0007730B001E730B0020
:102DC00015730B002E730B0025730B0035730B006E
:102DD0003D730B0063730B0057730B0071730B0093
:102DE000A8730B007F730B008D730B009D730B009A
:102DF000C9700B002D5E0B00BA4EBB4BBB4ABC49E1
:102E0000009600F6A860FCF70FFAFEF7DFFFB9495D
:102E10003868FFF753F8B8494FF4FA722846FFF7BD
:102E2000C1F8032809D12068B44AB549334600F6F1
:102E3000A860FCF7F9F9012482E71423C5F8EC3106
:102E4000052359E6DFF83883AE49D8F800000FAC07
:102E5000FFF734F8142065F0A8FAAB49204609279B
:102E600064F0FCFFA94912A864F0F8FFA84927768E
:102E700016A864F0F3FFA74919A864F0EFFF0A232E
:102E800084F83430A4491DA864F0E8FFA34920A8C1
:102E900064F0E4FF0B2384F85030A14924A864F0C7
:102EA000DDFFA04927A864F0D9FF9F4984F86C7022
:102EB0002BA864F0D3FF9D492EA864F0CFFF9C4956
:102EC00084F8887032A864F0C9FF9A4935A864F084
:102ED000C5FF994984F8A47039A864F0BFFF9749E9
:102EE0003CA864F0BBFF07230B930A940AAA84F85A
:102EF000C07006CA08AB0CA8FFF74AFD06274FF0C2
:102F00001C0909FB0740FFF79BFB013FF9D28C4BE3
:102F1000764A18688B4B7649009300F6A8608A4B76
:102F2000FCF782F9FEF752FF8849D8F80000FEF757
:102F3000C5FF33460CAA4FF4FA712846FFF78AFB07
:102F4000082804467FF42FAE1423C5F8EC3106237D
:102F500027E67F4ADFF82882106851680CAB03C36C
:102F600008210CA8FEF7EEFDFEF730FFD8F80000B0
:102F7000036808225B680CA9984740F2EE230822F8
:102F800006212846FFF7AAF8074680B96C4B714A1C
:102F900018687149334600F6A860FCF745F94FF40C
:102FA000FA63C5F8EC3185F8E8710824C8E6022810
:102FB00008D1634B694A18685149334600F6A86046
:102FC000FCF732F94FF44072002140A87DF066F81A
:102FD000634B18681B790F9008210FA88DF84030BB
:102FE0000023ADF841308DF84330FEF7ABFDFEF71E
:102FF000EDFED8F80000036808225B680FA9984727
:1030000004234FF49662CDE9003240A90A234FF41D
:1030100040722846FFF7F6F883B2002B00F0738168
:10302000DFF8448140A942461E23474611F801CBF0
:1030300002F801CB013BF9D11E2340AAD25CFA541D
:103040000133282BF9D197F828304522002180B28E
:103050004FF0290BA2F11D0982421FFA89F9C0F233
:10306000918009B187F82830DFF8D4903D4AD9F82B
:1030700000001F4900F6A860FCF7D6F8D9F8000058
:10308000394B3A4A1A4900F6A860FCF7CDF8D9F84E
:103090000000374B374A164900F6A860FCF7C4F821
:1030A000D9F8000097F82830334A114900F6A86093
:1030B000FCF7BAF82C4B314A0D494FF0000A97F84B
:1030C00028C0D9F80000D44500F6A86003F11E0B13
:1030D00074DD2933FCF7A8F80AF1010A0449274AEC
:1030E0005B46ECE7BA730B00AD730B0053720B0039
:1030F0006C5C0B00BF730B00CE730B00C9700B0030
:103100002D5E0B00E2730B001E740B0016740B0097
:1031100023740B0025740B002B740B002D740B0013
:1031200033740B003B740B004B740B0043740B00A7
:103130004F740B0055740B005C740B0060740B0033
:10314000407F002073740B0067740B007E740B00CB
:103150004E7E0B008C740B00D9610B00A9740B0020
:10316000567E0B00CA740B004C810020D9740B00F2
:103170006A810020EA740B00FB740B0009750B00D8
:10318000846100201E2111FB03BCBC44002109EB1B
:10319000010E1FFA8EFE0DF5807A01311AF80EE04D
:1031A0000CF801EB1E29F2D10133DBB2092B02F13D
:1031B0001E024FF001017FF64DAF53E74FF440720E
:1031C000002140A87CF06AFFDFF8B8B1DFF8C0A1A9
:1031D0004FF000099AF82830DBF800704B4507F6ED
:1031E000A86741DD08F1290318464F4903930422DB
:1031F0007EF089FA039B58B94FF4407208F12D0113
:1032000040A87EF092FA09F1010908F11E08E1E7F1
:103210004649072218467EF076FA0028F3D10A9034
:103220004FF4407208F1310140A87EF07EFA40ABC5
:103230003F4A40493846FBF7F7FF9DF8003183B11C
:103240000AA90A2240A87FF0C1FADBF800708AF8C8
:103250005501C3B2384A374907F6A860FBF7E4FFC7
:10326000D1E78AF85531CEE73449354808227EF057
:103270004AFA48B9334B0093334A344B3449384601
:10328000FBF7D2FF02245BE532492D4808227EF08D
:103290003AFA48B9304B00932B4A304B2C49384608
:1032A000FBF7C2FF03244BE52D49254808227EF099
:1032B0002AFA48B92B4B0093234A2B4B2449384612
:1032C000FBF7B2FF04243BE528491D4808227EF0A5
:1032D0001AFA48B9264B00931B4A264B1C4938461C
:1032E000FBF7A2FF05242BE52349154808227EF0B1
:1032F0000AFA40B9214B0093134A214B144938462E
:10330000FBF792FF1CE51F4B1F4A18681F49334605
:1033100000F6A860FBF788FF4FF4FA63C5F8EC31BC
:103320000023FFF7E9BB00BF0E750B0013750B0000
:103330001B750B006C5C0B002F750B003A750B00B6
:103340006A8100204A750B00C9700B0043750B00A1
:103350002D5E0B004C750B005C750B0055750B005A
:103360005E750B006E750B0067750B0070750B00BA
:1033700080750B0079750B0082750B0092750B0040
:103380008B750B00407F00208C740B00D9610B0003
:103390004C8100202DE9F04FB64B87B01E78039387
:1033A0000446002E40F02581D0F8FC31002B46D099
:1033B00090F8B430082B46D190F80132012B17D881
:1033C0004FF41651FFF744FB082884F8B4000FD1DE
:1033D00094F8E83163B994F800320133DBB2012B81
:1033E00009BF94F8013284F80032013384F80132C5
:1033F00094F80132022B22D14FF416512046FFF7E8
:1034000027FB082884F8B4001DD194F8E83193B95B
:1034100094F800520135EDB2012D84F800520AD122
:10342000954B964A186896494FF4165300F6A860D3
:10343000FBF7FAFE0126304607B0BDE8F08F94F89E
:10344000B430082BF7D02046FFF75DF894F8B400AD
:10345000012816D18B4D8C492868FEF72FFDFA20E4
:1034600064F0A3FF89492868FEF728FDFA2064F07C
:103470009CFF87492868FEF721FDFA2064F095FF3C
:10348000B4E009281FD17F4D82492868FEF716FD58
:103490004FF47A7064F089FF7F492868FEF70EFDCB
:1034A000FA2064F082FF7D492868FEF707FDFA20C4
:1034B00064F07BFF7A492868FEF700FDFA2064F08B
:1034C00074FF7849D6E70A2811D16E4D76492868ED
:1034D000FEF7F4FC4FF47A7064F067FF6E492868D9
:1034E000FEF7ECFCFA2064F060FF6C49C2E70B28A1
:1034F00002D1644D6D49EAE7002840F098806C4B9A
:10350000009307222C2306212046FEF70FFD5D4D78
:1035100002462868016804F50A764F683146B847C4
:10352000FA23072206212046FEF778FD032807D05C
:10353000514B604A1868524900F6A860FBF774FEC8
:103540005D4B009304231A4606212046FEF7EEFC4D
:103550000246286801684F683146B847FA230422BA
:1035600006212046FEF75AFD032807D0424B534A56
:103570001868434900F6A860FBF756FE0423DFF8FD
:10358000F8B0ADF810300DF110094FF0000800232D
:103590008DF817304E2301278DF8143005AB19F83C
:1035A00001AB00933A460423062120468DF816709D
:1035B0008DF815A0FEF7BAFC02462868036831466C
:1035C0005B689847FA233A4606212046FEF726FD17
:1035D000032808D0DBF80000394A2949534600F691
:1035E000A860FBF721FEB8F1000F1DD0039A01235C
:1035F00013700C2045F028FA324D856004F50471F3
:1036000074F07AFCD4F818320133C4F818320C2064
:1036100045F01AFA04F503768660294674F06CFCCE
:10362000AB680133AB6005E74FF00108AFE707284F
:1036300054D1144D24492868FEF740FC40F2EE2096
:1036400064F0B3FE21492868FEF738FCFA2064F0E4
:10365000ACFE1F492868FEF731FCFA2064F0A5FE95
:103660001C492868FEF72AFCFA2064F09EFE1A49DD
:1036700000E700BFA2820020407F002095750B006C
:10368000D9610B0084610020B8750B00C7750B0071
:10369000EE750B00FD750B0015760B0049760B00DF
:1036A00059760B006D760B007D760B0095760B003E
:1036B0002E800B00AD760B0020800B00CC760B002B
:1036C000F5760B00B84C01201D770B002E770B0010
:1036D0003E770B004E770B005E770B000D230C221C
:1036E00002211BF07DFB00284AD0194B194D93F89D
:1036F000B83128680A2B01D0192B26D11649FEF7BC
:10370000DDFB16492868FEF7D9FB15492868FEF746
:10371000D5FB14492868FEF7D1FB13492868FEF74A
:10372000CDFB12492868FEF7C9FB11492868FEF74E
:10373000C5FB10492868FEF7C1FBFA2064F035FE8E
:103740000D492868FEF7BAFB50E70C49D7E700BFE0
:1037500040CC0020846100206E770B00A2770B0024
:10376000B4770B00E3720B00F5720B00C6770B0009
:10377000D8770B00EA770B0007730B0088770B00F4
:1037800094F8B460022E40F01582FEF71FFBC14B87
:10379000009332460A2306212046FEF7A1FBBE4DC8
:1037A00002462868016804F50A77D1F80480394692
:1037B000C04732464FF4FA7306212046FEF78EFCCE
:1037C0000328B64E07D03068B54BB64AB64900F666
:1037D000A860FBF729FDB54B009339220823062189
:1037E0002046FEF77DFB024628680168D1F8048078
:1037F0003946C0474FF4FA73392206212046FEF7B6
:103800006DFC032807D03068A94BA64AA64900F6EC
:10381000A860FBF709FDA74B00932322282306216C
:103820002046FEF75DFB024628680168D1F8048057
:103830003946C0474FF4FA73232206212046FEF78B
:103840004DFC032807D030689B4B964A964900F6FA
:10385000A860FBF7E9FC994B009306231946082260
:103860002046FEF73DFB024628680168D1F8048037
:103870003946C0474FF4FA73082206212046FEF766
:103880002DFC032807D030688D4B864A864900F608
:10389000A860FBF7C9FC8B4B00930122082306218B
:1038A0002046FEF71DFB024628680168D1F8048017
:1038B0003946C0474FF4FA73012206212046FEF72D
:1038C0000DFC032807D030687F4B764A764900F616
:1038D000A860FBF7A9FC7D4B009301220823062179
:1038E0002046FEF7FDFA024628680168D1F80480F8
:1038F0003946C0474FF4FA73012206212046FEF7ED
:10390000EDFB032807D03068714B664A664900F624
:10391000A860FBF789FC6F4B009301220823062166
:103920002046FEF7DDFA024628680168D1F80480D7
:103930003946C0474FF4FA73012206212046FEF7AC
:10394000CDFB032807D03068634B564A564900F632
:10395000A860FBF769FC614B009301220823062154
:103960002046FEF7BDFA024628680168D1F80480B7
:103970003946C0474FF4FA73012206212046FEF76C
:10398000ADFB032807D03068554B464A464900F640
:10399000A860FBF749FC534B009301220823062142
:1039A0002046FEF79DFA024628680168D1F8048097
:1039B0003946C0474FF4FA73012206212046FEF72C
:1039C0008DFB032807D03068474B364A364900F64E
:1039D000A860FBF729FC454B009301220823062130
:1039E0002046FEF77DFA024628680168D1F8048077
:1039F0003946C0474FF4FA73012206212046FEF7EC
:103A00006DFB032807D03068394B264A264900F65B
:103A1000A860FBF709FCFEF7D9F9364B0093112299
:103A2000022306212046FEF75BFA02462868016859
:103A3000D1F804803946C0474FF4FA7311220621A9
:103A40002046FEF74BFB032807D030682A4B154A67
:103A5000154900F6A860FBF7E7FB284B00933B22D3
:103A60002C2306212046FEF73BFA0246286801680F
:103A7000D1F804803946C0474FF4FA733B2206213F
:103A80002046FEF72BFB032841D030681C4B054A2B
:103A900038E000BF24800B0084610020407F0020BC
:103AA000FC770B0019780B00D9610B00777F0B00B6
:103AB00026780B00E37E0B0047780B00747E0B002A
:103AC00062780B008A7E0B0078780B00927E0B00E8
:103AD0008B780B009A7E0B009D780B00B27E0B005A
:103AE000B0780B00AA7E0B00C3780B00827E0B001F
:103AF000D5780B00B47F0B00E7780B004B7F0B00F1
:103B00000D790B00234900F6A860FBF78DFB224BD3
:103B100000930122082306212046FEF7E1F9024620
:103B200028680168D1F804803946C0474FF4FA7319
:103B3000012206212046FEF7D1FA032807D030687B
:103B4000164B174A134900F6A860FBF76DFB154B9F
:103B5000009309220D2306212046FEF7C1F90246F3
:103B6000286801684D683946A8474FF4FA6309226E
:103B700006212046FEF7B2FA0328306806D00A4A2A
:103B8000044900F6A860FBF74FFB2FE5074A0849F8
:103B9000F7E700BFD9610B007A7E0B0030790B008C
:103BA00019780B00CE7E0B0042790B0064790B0074
:103BB0002D5E0B000523032200931146042330469B
:103BC0001BF00EF994F8B430002800F0F582032BB6
:103BD000C44DC54F04F50A7640F03D822868C34ABB
:103BE000C34900F6A860FBF71FFBC24B00931423E8
:103BF0003E2206212046FEF773F902463868016826
:103C0000D1F804803146C0474FF448733E22062164
:103C10002046FEF763FA0128286840F02082B64A61
:103C2000B34900F6A860FBF7FFFAFEF7CFF8B34BF5
:103C3000009302220A2306212046FEF751F902468C
:103C400038680168D1F804803146C0474FF4FA73F0
:103C5000022206212046FEF741FA032807D02868F1
:103C6000A74BA84AA84900F6A860FBF7DDFA94F82C
:103C7000B430042B40F00382FEF7A8F8A34B009366
:103C80003922082306212046FEF72AF90246386821
:103C90000168D1F804803146C0474FF4FA733922E5
:103CA00006212046FEF71AFA032807D02868984B09
:103CB000944A954900F6A860FBF7B6FAFEF786F835
:103CC000944B00932322282306212046FEF708F96F
:103CD000024638680168D1F804803146C0474FF485
:103CE000FA73232206212046FEF7F8F9032807D0AD
:103CF0002868894B834A844900F6A860FBF794FA48
:103D0000864B00930623194608222046FEF7E8F862
:103D1000024638680168D1F804803146C0474FF444
:103D2000FA73082206212046FEF7D8F9032807D0A7
:103D300028687B4B734A744900F6A860FBF774FA55
:103D4000784B00930122082306212046FEF7C8F88D
:103D5000024638680168D1F804803146C0474FF404
:103D6000FA73012206212046FEF7B8F9032807D08E
:103D700028686D4B634A644900F6A860FBF754FA63
:103D80006A4B00930122082306212046FEF7A8F87B
:103D9000024638680168D1F804803146C0474FF4C4
:103DA000FA73012206212046FEF798F9032807D06E
:103DB00028685F4B534A544900F6A860FBF734FA71
:103DC0005C4B00930122082306212046FEF788F869
:103DD000024638680168D1F804803146C0474FF484
:103DE000FA73012206212046FEF778F9032807D04E
:103DF0002868514B434A444900F6A860FBF714FA7F
:103E00004E4B00930122082306212046FEF768F856
:103E1000024638680168D1F804803146C0474FF443
:103E2000FA73012206212046FEF758F9032807D02D
:103E30002868434B334A344900F6A860FBF7F4F98D
:103E4000404B00930122082306212046FEF748F844
:103E5000024638680168D1F804803146C0474FF403
:103E6000FA73012206212046FEF738F9032807D00D
:103E70002868354B234A244900F6A860FBF7D4F99B
:103E8000324B00930122082306212046FEF728F832
:103E9000024638680168D1F804803146C0474FF4C3
:103EA000FA73012206212046FEF718F9032807D0ED
:103EB0002868274B134A144900F6A860FBF7B4F9A9
:103EC000244BDFF8988093F85531112B40F2138181
:103ED000FDF77CFF204B0093862208230621204615
:103EE0003EE000BF407F0020846100207E790B000F
:103EF0006C5C0B000B7F0B008B790B0024800B009C
:103F0000FC770B0019780B00D9610B00DB7E0B00EE
:103F100026780B007F7F0B00047A0B00747E0B0069
:103F200062780B008A7E0B0078780B00927E0B0083
:103F30008B780B009A7E0B009D780B00B27E0B00F5
:103F4000B0780B00AA7E0B00C3780B00827E0B00BA
:103F5000D5780B004C810020A27E0B004B7F0B001C
:103F6000FDF7BEFF024638680168D1F8049031467B
:103F7000C8474FF4FA73862206212046FEF7AEF8B2
:103F8000032807D028687A4B7A4A7B4900F6A86054
:103F9000FBF74AF92C23CDF800803B22062120466E
:103FA000FDF79EFF024638680168D1F8048031466B
:103FB000C0474FF4FA733B2206212046FEF78EF8E5
:103FC000032807D028686D4B6A4A6B4900F6A86041
:103FD000FBF72AF994F8B430042B21D1FDF7F6FE53
:103FE000674B00931722142306212046FDF778FF24
:103FF000024638680168D1F804803146C0474FF462
:10400000FA73172206212046FEF768F8032807D026
:1040100028685C4B574A584900F6A860FBF704F93A
:10402000594B009309220D2306212046FDF758FF26
:104030000246386801684F683146B8474FF4FA6362
:10404000092206212046FEF749F8032828687FF454
:1040500096AD4E4A9BE54E4B00932C23C8E594F851
:10406000B4304C49032B0CBF4B4A4C4A00F6A860B5
:10407000FBF7DAF84FF47A7064F097F9D5E5484B1E
:1040800000933922082306212046FDF729FF024626
:1040900038680168D1F804803146C0474FF4FA739C
:1040A000392206212046FEF719F8032807D0286890
:1040B0003C4B304A304900F6A860FBF7B5F83A4B64
:1040C00000932322282306212046FDF709FF0246FC
:1040D00038680168D1F804803146C0474FF4FA735C
:1040E000232206212046FDF7F9FF03283FF408AEFE
:1040F00028682E4BFEE52E4B009311220223062149
:104100002046FDF7EDFE024638680168D1F80490BC
:104110003146C8474FF4FA73112206212046FDF7B5
:10412000DDFF032807D02868224B124A124900F607
:10413000A860FBF779F82C23CDF800803B220621FC
:104140002046FDF7CDFE024638680168D1F80480AC
:104150003146C0474FF4FA733B2206212046FDF753
:10416000BDFF03283FF45CAF2868044B52E700BF53
:10417000217A0B0019780B00D9610B000D790B0027
:10418000BA7E0B003C7A0B00CE7E0B006F7A0B00E0
:104190001F7F0B002D5E0B00CC790B00E0790B002C
:1041A000777F0B0026780B00E37E0B0047780B002F
:1041B000B67F0B004F7A0B00062B40F00D824FF4B8
:1041C0007A7064F0F2F8FDF701FEC64B00938A2284
:1041D000222306212046FDF783FEC34D02462868B0
:1041E000016804F50A774E683946B0474FF4967374
:1041F0008A2206212046FDF771FF0328BB4E07D017
:104200003068BB4BBB4ABC4900F6A860FBF70CF812
:1042100040F2EE2064F0C9F8FDF7D8FDB74B0093EB
:104220008A22132306212046FDF75AFE02462868FB
:104230000168D1F804803946C0474FF496738A224A
:1042400006212046FDF74AFF032807D03068AC4B13
:10425000A84AA94900F6A860FAF7E6FF40F2EE2066
:1042600064F0A3F8FDF7B2FDA64B00938A22092360
:1042700006212046FDF734FE024628680168D1F881
:1042800004803946C0474FF496738A22062120469F
:10429000FDF724FF032807D030689B4B954A9649C9
:1042A00000F6A860FAF7C0FF40F2EE2064F07DF857
:1042B000FDF78CFD954B00938A22092306212046A9
:1042C000FDF70EFE024628680168D1F804803946E1
:1042D000C0474FF496738A2206212046FDF7FEFE62
:1042E000032807D030688A4B824A834900F6A860C9
:1042F000FAF79AFF40F2EE2064F057F8854B0093EE
:104300008A22262306212046FDF7EAFD0246286878
:104310000168D1F804803946C0474FF496738A2269
:1043200006212046FDF7DAFE032807D030687A4BD5
:10433000704A714900F6A860FAF776FF40F2EE2065
:1043400064F033F8754B00938A2226230621204619
:10435000FDF7C6FD024628680168D1F80480394699
:10436000C0474FF496738A2206212046FDF7B6FE19
:10437000032807D030686A4B5E4A5F4900F6A860A0
:10438000FAF752FF40F2EE2064F00FF8654B00930D
:104390008A220E2306212046FDF7A2FD0246286848
:1043A0000168D1F804803946C0474FF496738A22D9
:1043B00006212046FDF792FE032807D030685A4BAD
:1043C0004C4A4D4900F6A860FAF72EFF40F2EE2065
:1043D00063F0EBFF554B00938A220E230621204603
:1043E000FDF77EFD024628680168D1F80480394651
:1043F000C0474FF496738A2206212046FDF76EFED1
:10440000032807D030684A4B3A4A3B4900F6A86077
:10441000FAF70AFF40F2EE2063F0C7FF454B009326
:104420008A220E2306212046FDF75AFD02462868FF
:104430000168D1F804803946C0474FF496738A2248
:1044400006212046FDF74AFE032807D030683A4B84
:10445000284A294900F6A860FAF7E6FE40F2EE2065
:1044600063F0A3FF354B00938A220E2306212046DA
:10447000FDF736FD024628680168D1F80480394608
:10448000C0474FF496738A2206212046FDF726FE88
:10449000032807D030682A4B164A174900F6A8604F
:1044A000FAF7C2FE40F2EE2063F07FFF254B009347
:1044B0008A220E2306212046FDF712FD02462868B7
:1044C0000168D1F804803946C0474FF496738A22B8
:1044D00006212046FDF702FE03283DD030681A4B26
:1044E00034E000BF89800B0084610020407F002001
:1044F000907A0B0019780B00D9610B0076800B00C5
:10450000B37A0B00D0800B00D67A0B00C7800B006B
:10451000FE7A0B00DE7F0B00267B0B00B87F0B00C2
:10452000497B0B0012800B006C7B0B0004800B009E
:104530008F7B0B00B9800B00B27B0B00AB800B00B4
:10454000CD7B0B005A800B00E87B0B00294A2A49DF
:1045500000F6A860FAF768FE40F2EE2063F025FF4F
:10456000264B00938A220E2306212046FDF7B8FC35
:10457000024628680168D1F804803946C0474FF4E4
:10458000FA738A2206212046FDF7A8FD032807D0EA
:1045900030681B4B174A184900F6A860FAF744FE2A
:1045A00040F2EE2063F001FF164B009309220D2329
:1045B00006212046FDF794FC0246286801684D68F4
:1045C0003946A8474FF4FA63092206212046FDF731
:1045D00085FD032830683AE50F2B7FF407A80A4DC4
:1045E0000A492868FDF76AFCFA2063F0DEFE0849F4
:1045F000FEF740BF19780B00D9610B0068800B00F3
:104600000A7C0B00A77F0B00846100202C7C0B0030
:10461000417C0B0010B50378DB07044604D563F03A
:10462000B9FEE368C01A10BD4FF0FF30FBE7000091
:104630002DE9F04700F5827604460FCE9CB009AD17
:104640000FC5F03433682B600FCC0EAD0FC5236857
:104650009DF824402B6014F0010439D09DF83840B7
:1046600014F0010434D009A847F056FC054609A807
:10467000FFF7D0FF09A8FFF7CDFF4FF47A73B0FB27
:10468000F3F07AF0CDF9274B00227AF08DF87AF02A
:10469000F1FC2844139009A847F02EFC149009A8B7
:1046A00047F01EFC15900EA847F00EFC16900EA8C1
:1046B00047F0FCFB013817900EA847F0E9FB0023F8
:1046C0001B93179BA0F26C70002B189004DA002447
:1046D00020461CB0BDE8F08713A9042002F0B8FF03
:1046E0000128F4D1104B0EA81D6847F0D1FB0790AC
:1046F0000EA847F0DBFB064609A8DDE91587DDE9D2
:1047000013A9FFF787FF05F6A865CDE904A0CDE959
:104710000289CDE90067079B044A05492846FAF754
:1047200083FDD5E70000E03F407F0020567C0B0072
:104730006C5C0B00000000002DE9F04790F8CC31D4
:10474000D0F8E42180F8E031D0F8D8319A428CB02A
:1047500004460FD2042B09D9AB4908680093AB4932
:104760009B1A00F6A860AA4AFAF75EFDD4F8D83181
:10477000C4F8E431236820465B6A98470546002860
:1047800000F02D8194F8B800830705D494F83851CF
:1047900015F0020500F0238110F0010504F582797F
:1047A00004F1F0082BD063F0F5FDD4F8EC3041F2C1
:1047B0008736C01AB04222D84846FFF72BFFB042D6
:1047C0001DD84046FFF726FFB04218D894F8B830FD
:1047D000B4F8BC708F4E23F0020384F8B830642222
:1047E000D4F8C030B3FBF2F306FB073794F8C430BB
:1047F00003B17F42884B9F4221DD0025EFE0824BD1
:104800001D6894F8B830DF0705F6A86514D563F085
:10481000C1FDD4F8EC40041B4846FFF7FBFE0646FA
:104820004046FFF7F7FE7D4A7849CDE90060234610
:104830002846FAF7F9FCE0E74FF0FF34ECE7B4F86C
:10484000C820D4F8CC306421B3FBF1F306FB023668
:1048500094F8D03003B17642714B9E42CDDC0223F6
:1048600084F84C3094F88031D4F884A1C4F86CA05A
:1048700023F0020384F8803150467AF0D1F85EA329
:10488000D3E900237AF046F97AF01CFCA066BAF16D
:10489000000F09D15C4B634A18685C49534600F627
:1048A000A860FAF7C1FCA8E794F89031D4F8940115
:1048B000676323F00203E66384F890317AF0C0F86E
:1048C0000022594B7AF050FA7AF0D4FB94F8383140
:1048D000606623F00203824684F83831D4F83C0144
:1048E0007AF0AEF8504B00227AF03EFA06460F46B8
:1048F00050467AF0A5F832463B4679F055FF7AF0FB
:10490000B9FB3946E06530467AF0B4FB94F8E03103
:10491000C4F888306064484647F0FEFA0390484681
:1049200047F0EAFA0490484647F0DAFA0590404624
:1049300047F0CAFA0690404647F0B8FA01380790A7
:10494000404647F0A5FAA0F26C700023089003A837
:104950000B9302F02DFE94F8483120659E0741BF6D
:1049600023F0020384F84831D4F84C31C4F8903075
:1049700094F82831980716D5D90714D523F00203E7
:1049800084F82831D4F82C3148F69F4293422AD833
:1049900018467AF045F8254B00227AF0BBF87AF0F9
:1049A00091FBC4F8840094F818319A0717D513F0D6
:1049B000010614D023F0020384F81831D4F81C0146
:1049C0007AF02EF80EA3D3E900237AF0A3F8164B61
:1049D00000227AF0C9F97AF075FB3546E06728467F
:1049E0000CB0BDE8F087084A08491068104A00F684
:1049F000A860FAF719FCD6E78FC2F5285C8FF63F5E
:104A00006F1283C0CAA1FD3F407F0020D9610B0017
:104A10008D7C0B008096980000E9A435BD7C0B00CE
:104A200000D2496BEC7C0B000000594000408F40E5
:104A30000C7D0B0038B504460068844204D005683C
:104A400044F026F82846F8E738BD38B50446006833
:104A5000844204D0056844F01BF82846F8E738BDC6
:104A60002DE9F8438046154B58F8045F036004466F
:104A7000454515D0AF683E68B7420FD0B368D6F849
:104A800000909C4208D1BB68013B3046BB6073F08C
:104A90003AFA304643F0FCFF4E46EDE72D68E7E773
:104AA0002846FFF7D2FF00232846C4E90155E360FA
:104AB000FFF7CBFF2046BDE8F88300BF007E0B0068
:104AC00010B50446FFF7CCFF2046102165F04CFAE4
:104AD000204610BD10B5034B03600446FFF7C0FF2E
:104AE000204610BD147E0B0010B5054B044640F85F
:104AF000343BFFF7EFFF2046F9F788FB204610BD57
:104B0000287E0B002DE9F04190F80332BAB004463C
:104B1000002B65D0344B02681E68036D526A059302
:104B2000002580F8035290F80272D0F890809047E8
:104B300006F6A866CDE90180059B2C4A2C49009712
:104B40003046FAF771FB09AACDE90922294A0892F1
:104B500007AA0C92284A294E94F8020296F88C3043
:104B600094F804128DF86C00CDE90D2511AACDE959
:104B70001122234A079215AACDE91522214A14923F
:104B800007AA1892204A8DF86D10013BCDE919252E
:104B900018BF012304F1300174221CA80B958DF875
:104BA0003C5010951395179539958DF86E307BF024
:104BB0004DFA54F8A85FA54207D0A868036807A972
:104BC0009B68984708B92D68F5E796F88C30012B5B
:104BD00003D10E4B186833F041FD07A8FFF784FF9F
:104BE0003AB0BDE8F08100BF407F00202E7D0B0071
:104BF0006C5C0B00945F0B0089DA020040CC002053
:104C0000287E0B00147E0B00111C03002C3E01209B
:104C100090F805322DE9F041044633BB6C4B1B681C
:104C200023B16C4D95F88C30022B0DD16A4B6B4A39
:104C300018686B4900F6A860FAF7F6FA2368204670
:104C40009B69BDE8F041184703681B6A984718B98B
:104C5000D4F8EC01BDE8F08195F88C30012BEDD152
:104C600084F805322046FFF74DFF23682046DB6AB3
:104C7000984710B12046FDF746FC564E96F869302D
:104C80004BB994F807325BB1564800F0FCF910B10B
:104C90002046FDF741FC94F80732002B40F0878056
:104CA000F06E94F8E0511AF0D7FF94F8F031804696
:104CB0003BB9236820461B6B984710B1012384F849
:104CC000F031236820465B6B9847074638B142F2C3
:104CD0001073984541D840F20113A4F802324148BC
:104CE00000F0D8F98046A8B1A7B93B4B3E4A1868F6
:104CF0003E4900F6A860FAF797FA94F802324BB1F1
:104D00007422394604F130007BF0C8F94FF4807307
:104D1000A4F80232D4F8F4513DB163F03BFBD4F86F
:104D2000F451A84294BF0025012594F8033223B919
:104D3000B8F1000F01D1002D39D094F8F0216AB3F9
:104D400094F8022252B3012384F803320023C4F8FA
:104D5000F4312046FFF7D6FE22E094F8023293B9F0
:104D6000012384F8023263F015FBA8F51C58A8F162
:104D7000100844F62063984594BF00EB0803C3185D
:104D8000C4F8F431ABE7002DEAD0D4F8F43103F1E4
:104D9000320563F0FFFA8542E2D3A0E7002BD5D1BC
:104DA000B8F1000F00D115B12046FDF7C5FB96F80C
:104DB000693023B194F80232002B7FF43FAF94F8AE
:104DC0000732002B41F2883008BF322042E700BF93
:104DD0008461002040CC0020407F00205F7D0B00DC
:104DE0002D5E0B0054610020827D0B00D9610B0009
:104DF00010B50446FFF778FE2046CC2165F0B4F8E4
:104E0000204610BD10B50446FFF764FE20461C2165
:104E100065F0AAF8204610BD2DE9F041056804466A
:104E20000F460646AC4216D0AA683B68D5F800800B
:104E30009A420ED105F108039F4209D0A368013BB5
:104E40002846A36073F05FF8284643F021FE00E097
:104E50002E464546E6E7B4420AD0A368013B3046F9
:104E6000A36073F050F83046BDE8F04143F010BE47
:104E7000BDE8F08173B506460D4B56F8045F03603C
:104E80000446B54206D0A868019401A9FFF7C4FF03
:104E90002D68F6E72846FFF7CDFD00232846C4E934
:104EA0000155E360FFF7C6FD204602B070BD00BFAC
:104EB000EC7D0B0010B50446FFF7DCFF2046102107
:104EC00065F052F8204610BD10B5034B0360044650
:104ED000FFF7D0FF204610BD387E0B002DE9F743C9
:104EE0001B4B0360044600F5037601A9194801969F
:104EF000DFF86090FFF790FFD4F8105204F50477C4
:104F0000AF4211D0AB68D5F800804B450AD1D4F838
:104F10001832013B2846C4F8183272F0F4FF2846D4
:104F200043F0B6FD4546EBE725463046FFF7CCFF9C
:104F300055F8A80FA84204D0066843F0A9FD3046F2
:104F4000F8E72046FBF72CF9204603B0BDE8F083D4
:104F5000E4800B00B84C012010B50446FFF7BEFFFB
:104F600020464FF44B7164F0FFFF204610BD10B592
:104F70000446FFF7A9FF20461C2164F0F5FF2046F8
:104F800010BD0000024A0349034872F0B0BF00BFE1
:104F900000600020B91D0300A482002010B5044663
:104FA00063F0F8F9206010BD13B5044663F0F2F920
:104FB000236822696060C01A084B094901322261E6
:104FC0001C6800924FF47A73064AB0FBF3F304F6C0
:104FD000A860FAF729F902B010BD00BF407F002099
:104FE0006C5C0B001C810B000023C0E90033C0E99E
:104FF0000233036170470000F8B5194F044663F0AF
:10500000C9F93A79022A0546F86E23D00B2A1549C8
:1050100018BF78211AF012FE2369064693B13B7936
:10502000786E022B18D00B2B4AF6C00118BF4FF434
:1050300061611AF003FE0C4B834228BF03469E4277
:1050400038BF1E46E3686268D21A531B981920EADB
:10505000E070F8BD0349DDE74AF6C001E9E700BFAB
:1050600040CC00208051010080EE3600D0E90023C2
:105070009A4210B5044604D963F08CF92368C01A2B
:1050800010BD0020FCE708B5FFF7B6FFB0FA80F0CE
:10509000400908BD38B50546FFF7E8FF164B9842B2
:1050A000044627D82B6913B1144B984222D8144DCB
:1050B0002A79686E022A17D00B2A4AF6C00118BF57
:1050C0004FF461611AF0C4FE2B79022B0FD00B2B29
:1050D0004AF6C00118BF4FF461611AF0AFFD844277
:1050E00094BF0020012038BD4AF6C001EAE74AF625
:1050F000C001F2E70120F6E7A0BB0D00E093040039
:1051000040CC0020D0E900239B1A8268012A23EAC0
:10511000E3730FD1C360134B134901328260C2683D
:1051200018684FF47A7300F6A860B2FBF3F30F4AE5
:10513000FAF77AB8EFD907EE903A90ED056AB8EE33
:10514000E77AD0ED037AF7EE006AF8EE677A76EE4A
:10515000C66A67EEA67AE7EE067AFCEEE77AC0ED5D
:10516000037AD8E7407F00206C5C0B005E810B0067
:1051700038B5044663F00EF923686060C01A094B25
:10518000094A1D6809494FF47A73B0FBF3F305F639
:10519000A860FAF749F82046FFF7B4FF002323611F
:1051A00038BD00BF407F00207B810B006C5C0B0092
:1051B000C068704738B500250446C0E900558560D1
:1051C000142229460C307AF069FF0123C4E90855FE
:1051D000C4E90B55C4E90E55C4E91155A5626563D0
:1051E0002564E56484F85030204638BD2DE9D0436D
:1051F00059EC108B002304460022494610EE100A99
:1052000057EC116B79F0F8FE002814BF53234E239E
:105210002372002200234046494679F0EDFE10B18A
:1052200009F10043994649EC108B74F0EDF851EC0C
:10523000100B79F047FFC0B2207079F001FC0246F4
:105240000B464046494679F0ADFA334B002279F0DF
:1052500061FC8046894649EC108B74F0D5F851EC1E
:10526000100B79F02FFFC0B2607079F0E9FB0246B5
:105270000B464046494679F095FA274B002279F0D3
:1052800049FC79F01FFF0023606000223946304658
:1052900079F0B2FE002814BF57234523237400225F
:1052A00000233046394679F0A7FE10B107F10043DC
:1052B0001F4647EC106B74F0A7F851EC100B79F017
:1052C00001FFC0B2607279F0BBFB02460B4630466C
:1052D000394679F067FA104B002279F01BFC06463C
:1052E0000F4647EC106B74F08FF851EC100B79F00F
:1052F000E9FEC0B2A07279F0A3FB02460B4630462D
:10530000394679F04FFA044B002279F003FC79F02A
:10531000D9FEE060BDE8D08300004E4000000000F0
:105320002DE9F04F964B8DB057EC106B55EC114BAF
:10533000009002AA03F1080E186859689446ACE878
:105340000300083373456246F6D118689B88ACF8B1
:1053500004308C4BCCF8000006AA03F1100E18683C
:1053600059689446ACE80300083373456246F6D1A9
:1053700018681B79CCF800008CF804300022824BAE
:105380003046394679F056FE002800F0E0807F4B29
:1053900000223046394679F02FFE10B96EA7D7E9C2
:1053A0000067DFF8F0B14FF0000A52465B46204636
:1053B000294679F021FE98B9DFF8DCB14FF0000AF8
:1053C00052465B462046294679F02AFE88B120469F
:1053D00029466F4B002279F0E5F904460D46EFE7C8
:1053E000204629466A4B002279F0DEF904460D4634
:1053F000DBE75BA3D3E900233046394679F08AFB2B
:1054000059A3D3E9002379F0CFF97AF055F858A3DE
:10541000D3E9002306460F462046294679F07AFB59
:1054200055A3D3E9002379F0BFF97AF045F84FF09E
:105430000B0A04460D46052200233046394604F087
:10544000030879F0BDFF05F00049B8F1000F79F1CC
:10545000000305DA18F1FF3868F0030111F10108C3
:105460000CAB03EB82024244304612F8183C02AA0D
:10547000394602F80A300522002379F0A1FF002CFA
:105480000F4675F10001064622462B4602DAE21C61
:1054900045F100030AF1FF3A9408BAF1060F44EA15
:1054A00083744FEAA305C6D14FF000094FF00A08F4
:1054B0000DF1180B204629461422002379F080FFB5
:1054C0001BF802300CAA4244019202F8283C3046F4
:1054D00039461422002379F073FF1BF80230019A39
:1054E000304602F8293C39461422002379F068FF3F
:1054F000142206460F4620462946002379F060FF15
:10550000A8F1020A04460D46B9F1000F1DD10CABFB
:105510009A444FF02B03A8F103080AF8283C09F13C
:105520000109B9F1050FC5D1009B009902AA013B01
:105530000A3112F8010B03F8010F9942F9D1009AD0
:105540000023D3720DB0BDE8F08FD046E7E70E4FD1
:10555000002626E7AFF300802A3A92CBFF7F564021
:105560000000000084D77741000000D088C3E041EC
:105570000000000000405F410000000000F9D5413C
:1055800090810B009E810B00008056C00080564029
:1055900000807640008066C0008066400000000009
:1055A0002DE9F04F2DED068B83B0CDE90001D6A398
:1055B000D3E9002351EC100B55EC114B79F0AAFA0A
:1055C000EF4B002279F0D0FBCFA3D3E9002341ECCD
:1055D000190B2046294679F09DFAE94B002279F013
:1055E000C3FBB0EE490AF0EE690A41EC180B74F007
:1055F00033F855EC104B10EE102A10EE100A2B4623
:10560000294679F087FAC2A3D3E9002379F082FA18
:1056100002460B460020DB4979F0C4F841EC100B40
:1056200074F0B0FBBCA1D1E9000153EC102B79F070
:105630009BFBB0EE490AF0EE690A06460F4673F08E
:1056400083FC59EC108B002200233046394679F058
:10565000ABF842464B4679F05DFAB0EE480AF0EE00
:10566000680A8046894673F06FFC404653EC102B65
:10567000494679F04FFAB0EE480AF0EE680A8246E1
:105680008B4673F0E9FF404653EC102B494679F006
:1056900041FAA3A3D3E90023804689463046394620
:1056A00079F038FA0022002379F07EF822462B4662
:1056B00079F030FA9CA3D3E9002306460F46504602
:1056C000594679F027FA9AA3D3E9002379F06AF8CA
:1056D00099A3D3E9002304460D464046494679F094
:1056E00019FA02460B462046294679F05BF894A346
:1056F000D3E9002304460D463046394679F00AFACC
:1057000002460B462046294679F04EF88AA3D3E993
:10571000002341EC190B5046594679F0FBF98AA356
:10572000D3E9002379F040F87FA3D3E900230446AE
:105730000D464046494679F0EDF902460B462046B3
:10574000294679F031F882A3D3E9002304460D46B7
:105750003046394679F0DEF902460B4620462946A6
:1057600079F020F876A3D3E9002341EC1A0B5046D8
:10577000594679F0CFF902460B4677A1D1E90001ED
:1057800079F010F872A3D3E9002304460D46404691
:10579000494679F0BFF902460B462046294679F082
:1057A00003F861A3D3E9002304460D463046394689
:1057B00079F0B0F902460B462046294678F0F4FF0E
:1057C00053EC192B82468B4651EC190B79F0A2F958
:1057D00053EC1A2B04460D4651EC1A0B79F09AF94A
:1057E00002460B462046294678F0DEFF41EC100BBE
:1057F00074F0C8FA55EC104B10EE102A10EE100A97
:105800002B46294679F086F9524606460F465B46F6
:105810005046594679F07EF902460B4630463946E5
:1058200078F0C2FF41EC100B74F0ACFA4CA3D3E952
:1058300000235046594659EC108B79F06BF94AA376
:10584000D3E9002306460F462046294679F062F93F
:1058500002460B463046394679F086FA42460646FD
:105860000F464B4642A1D1E9000179F07DFA454B44
:10587000002278F099FF02460B463046394679F00F
:1058800049F902460B468046894679F043F93D4B7B
:10589000002278F089FF41EC100B74F073FA404657
:1058A00053EC102B494679F05FFA42464B460646C8
:1058B0000F4679F059FA30A3D3E900238046894690
:1058C00079F028F942464B4679F024F942464B4696
:1058D00079F020F902460B462046294678F062FF0F
:1058E00023A3D3E9002341EC180B3046394679F065
:1058F00011F932463B4679F00DF932463B4679F0D4
:1059000009F952465B463FE0182D4454FB210940FB
:10591000F094FEF1906B7B3F00000040A65458418C
:10592000D6021CDE28C9EF3FBDD8147C1500F03F1D
:10593000BA490C022BE77B405F887CF1AC1FD1BEDB
:10594000CB0969F32D17B4BE355EBA490C4A5F40E6
:1059500061F179121B6FA8BE14AE47E17AF080C0E6
:10596000560E2D3A483F5841621058D916545841A6
:10597000A457FB9A8CD7E440BD9AE555B9C5E440DD
:10598000008066400000F03F78F00EFFB0EE481A4D
:10599000F0EE681A41EC100B73F066FFB0EE491A96
:1059A000F0EE691A009B83ED000BB0EE4A0AF0EEB0
:1059B0006A0A73F059FF019B83ED000B03B0BDEC45
:1059C000068BBDE8F08F00BF2DE9F04F2DED108B59
:1059D000E74B9DB015AA019003F1180518685968A6
:1059E000144603C40833AB422246F7D11B882380F8
:1059F00012A910A8FFF7D4FD9DED108BB0EE480A58
:105A0000F0EE680A73F028FEC5A3D3E90023B0EED8
:105A100040AAF0EE60AA51EC100B79F07BF853EC41
:105A20001A2B79F077F802460B460020D14978F01E
:105A3000B9FE41EC100BDDE9124541EC190B74F095
:105A4000A1F9B9A1D1E9000153EC102B79F08CF93F
:105A5000B0EE490AF0EE690A9FEDB51B8046894613
:105A600074F0BEF8B4A1D1E9000153EC102B79F029
:105A70007BF902460B464046494679F075F90246E5
:105A80000B4643EC1E2BBB4B002278F08BFEB0EE96
:105A9000480AF0EE680A41EC1C0B73F055FA53EC1F
:105AA000102BB0EE409AF0EE609A51EC100B79F0AA
:105AB00031F853EC192B79F02DF802460B4641ECE6
:105AC0001D0B51EC190B79F025F853EC192B79F0DB
:105AD00021F8B0EE480AF0EE680A41EC1F0B73F0B3
:105AE00013FE53EC102B10EE100A194679F012F841
:105AF00002460B4643EC1B2B79F00CF89E4BCDE98C
:105B00000201002251EC1B0B79F004F88CA3D3E9BD
:105B10000023CDE904012046294678F045FE0246DF
:105B20000B4604460D4678F0F5FF944B82468B46B3
:105B3000002251EC1B0B78F0EDFF02460B460020D3
:105B40008F4978F02FFEDDE9022378F02DFE8D4B92
:105B500006460F46002251EC1C0B78F0DBFF024694
:105B60000B463046394678F01FFE53EC1C2B064698
:105B70000F46DDE9040178F0CDFF02460B463046C2
:105B8000394678F00FFE804B06460F46002240460D
:105B9000494679F0E9F853EC1F2B78F0BBFF024639
:105BA0000B463046394678F0B5FF52465B4678F0F2
:105BB000B1FF52465B4678F0ADFF22462B4678F0A7
:105BC000A9FF724B06460F4600224046494679F02F
:105BD000CBF853EC1D2B78F09DFF53EC1B2BCDE93C
:105BE000060151EC1E0B78F0DDFD02460B46DDE9A7
:105BF000060178F08FFF52465B4678F08BFF224615
:105C00002B4678F087FF424641EC1E0B4B4651EC89
:105C1000190B78F07FFF22462B4678F07BFF4AA3D2
:105C2000D3E9002378F0C0FD02460B4651EC1E0B71
:105C300078F0BAFD02460B463046394678F0B4FD9E
:105C400002460B4643EC1E2B0022002379F0D4F9C8
:105C5000002840F075813EA3D3E9002351EC1E0BD0
:105C600079F0E8F9002840F06B813BA3D3E90023E9
:105C700051EC180B78F096FD37A3D3E900230446C6
:105C80000D4651EC180B78F08FFD06460F4647EC99
:105C9000106B73F059F98DED080B45EC104B73F058
:105CA000DBFC32463B46304639468DED060B78F03C
:105CB0007BFD41EC100B73F047F922462B46204642
:105CC00029468DED0C0B78F06FFD41EC100B73F055
:105CD000C3FC2F4B0022304639468DED0A0B78F07D
:105CE00019FF41EC100B73F02FF9294B00222046CD
:105CF00029468DED0E0B78F00DFF41EC100B73F083
:105D0000ABFC17A3D3E900232046294657EC106BC0
:105D100078F000FF14A3D3E9002304463AE000BF63
:105D2000002A717791527B3FF785C81E9B515841DD
:105D3000000000000000F83F187DB0E9132858412A
:105D4000399D52A246DFA13F00000000006A1841C1
:105D500000000000C05C2541BF808E28E45DEB3F61
:105D600096FC7270DD06F03FC1E30B175098743F4C
:105D7000B3810B000000F03F00004D4000003240B6
:105D80000000144000002C4000005E40000018405D
:105D9000000008400D46DDE9060178F0BBFEDDE9B4
:105DA000082378F0B7FE02460B462046294678F0D5
:105DB000F9FCADA3D3E9002304460D46DDE90A0151
:105DC00078F0A8FEDDE90C2378F0A4FE02460B462D
:105DD0002046294678F0E8FCA5A3D3E90023044631
:105DE0000D463046394678F095FEDDE90E2378F011
:105DF00091FE02460B462046294678F0D3FC9EA32E
:105E0000D3E9002378F086FE8DA3D3E9002378F050
:105E1000C9FC8D4B04460D4600224046494678F0A9
:105E200079FE53EC1A2B78F075FE53EC192B78F0B1
:105E300071FE52465B4678F06DFE02460B462046E8
:105E4000294678F0B1FC814B04460D4600224046BD
:105E5000494678F089FF53EC1A2B78F05BFE53EC3F
:105E60001D2B78F057FE53EC1B2B06460F460020E7
:105E7000774978F097FC774B41EC180B002251ECF6
:105E80001C0B78F047FE02460B4651EC180B78F0DD
:105E90008BFC02460B463046394678F03BFE5246B4
:105EA0005B4678F037FE52465B4678F033FE02469A
:105EB0000B462046294678F077FC674B04460D4692
:105EC00000224046494678F04FFF53EC1A2B78F0F9
:105ED00021FE53EC1F2B78F01DFEDDE9042306465E
:105EE0000F4600205D4978F05DFCDDE9022378F083
:105EF0005BFC02460B463046394678F00BFE5246B4
:105F00005B4678F007FE52465B4678F003FE524649
:105F10005B4678F0FFFD02460B462046294678F0A6
:105F200043FC0022002304460D4679F065F838B999
:105F300041A3D3E900232046294679F07BF850B1EC
:105F4000474B93E80700019B83E807001DB0BDECB9
:105F5000108BBDE8F08F3AA3D3E9002351EC1E0B60
:105F600078F002FF41EC100B73F04EFA51EC100B7D
:105F700079F0A8F832A3D3E90023814629462046C8
:105F800078F0F2FE41EC100B73F03EFA51EC100B7E
:105F900079F098F84FF005088246C0F11300B0FB85
:105FA000F8F000EB800078F03BFD064609F10A00AE
:105FB000B0FBF8F00F4678F033FDB9FBF8F8024675
:105FC0000B463046394678F0EFFB79F053F81CABBE
:105FD00043FA80F0019A10F81C3C13706FF0040033
:105FE00000FB0AFA0AF15F00192308EB8808B0FBEE
:105FF000F3FAA9EB080803FB1A0AD0441CAB53FAC6
:1060000088F851EC1E0B18F81C3C537079F032F8EC
:10601000144E019A90FBF6F303FB160353602046DF
:10602000294679F027F890FBF6F303FB1606019B4F
:106030009E608BE7AFF300800000000020D6334164
:1060400000000000006AF8400000E03F0000384017
:1060500000001440000022400080864000804E4036
:1060600040820B00A086010009CFE71D4C86C73E89
:10607000BDE60CDA9D1E343EC8C6539FCE3C584147
:106080002DE9F04F2DED088B59EC108B55EC124B90
:1060900089B012EE102A10EE100A2B46494657EC32
:1060A000116B5BEC13AB78F09DFF40B152465B4641
:1060B0003046394678F096FF002840F0B9805FA35B
:1060C000D3E900234046494678F04EFE5BA3D3E96E
:1060D000002341EC190B3046394678F045FE57A3B2
:1060E000D3E9002341EC1B0B2046294678F03CFE07
:1060F00052A3D3E9002341EC180B5046594678F0DF
:1061000033FEB0EE480AF0EE680A41EC1A0B72F06A
:106110001BFF55EC104BB0EE490AF0EE690A72F025
:1061200013FF57EC106BB0EE4B0AF0EE6B0A72F0F7
:106130000BFF51EC100BB0EE4A0AF0EE6A0ACDE903
:10614000060172F001FF59EC108BB0EE4B0AF0EE35
:106150006B0A73F081FA8DED000BB0EE4A0AF0EE97
:106160006A0A73F079FA8DED020BB0EE490AF0EE8F
:10617000690A73F071FA8DED040BB0EE480AF0EE87
:10618000680A73F069FADDE9060132463B465BECCA
:1061900010AB78F0BFFC22462B4678F0BBFC4246A1
:1061A0004B4678F0B7FC3246804689463B46DDE9EF
:1061B000000178F0AFFC22462B4678F0ABFCDDE91D
:1061C000022378F0A7FC02460B464046494678F089
:1061D000EBFA524604460D465B46DDE9040178F0D1
:1061E00099FC02460B462046294678F0DDFA41EC40
:1061F000100B73F0FFFA55EC104B10EE102A10EE56
:10620000100A2B46294678F01FFF08B1002400250C
:106210000CA3D3E900232046294678F07BFC78F0D4
:1062200071FF00EE100A09B0BDEC088BBDE8F08FDD
:106230009FED010AF7E700BF00000000F8C1631AF4
:10624000DCA54C4000000000CC4858410000000094
:106250002DE9F04F2DED068B51EC100B85B04AA3C4
:10626000D3E9002359EC128B55EC134B57EC116B0F
:1062700078F050FC464B002278F076FD42A3D3E93B
:10628000002341EC190B4046494678F043FC404B53
:10629000002278F069FD324641EC1A0B3B4620465D
:1062A000294678F07FFA38A3D3E9002378F032FC4E
:1062B000374B002278F058FD41EC100B41EC180BE5
:1062C00073F0CAF98DED000BB0EE4A0AF0EE6A0ADF
:1062D00072F03AFE55EC104BB0EE490AF0EE690A46
:1062E00072F032FE57EC106BB0EE4A0AF0EE6A0A1A
:1062F00073F0B2F953EC102BB0EE490AF0EE690AD4
:10630000CDE9022373F0A8F959EC108BB0EE480ADE
:10631000F0EE680A72F018FEDDE9022330463946D5
:106320005BEC10AB78F0F6FB424606460F464B4658
:106330002046294678F0EEFB52465B4678F0EAFBB1
:1063400002460B463046394678F02CFA22462B4658
:1063500041EC180BDDE9000178F0DCFBB0EE481AE7
:10636000F0EE681A41EC100B73F07EFA51EC100B52
:1063700078F0C8FE00EE100A05B0BDEC068BBDE853
:10638000F08F00BFAFF30080182D4454FB2109406B
:106390000080664010B53E4904467BF043F9002872
:1063A00055D03C4920467BF03DF9002850D03A4971
:1063B00020467BF037F900284CD0384920467BF046
:1063C00031F9002848D0364920467BF02BF90028C7
:1063D00044D0344920467BF025F9002840D032498A
:1063E00020467BF01FF900283CD0304920467BF046
:1063F00019F9002838D02E4920467BF013F9A8B3AC
:106400002C4920467BF00EF990B32B4920467BF0B7
:1064100009F978B3294920467BF004F960B328498B
:1064200020467BF0FFF848B3264920467BF0FAF877
:1064300038B3254920467BF0F5F828B32349204698
:106440007BF0F0F8002840F2511018BF002010BD7A
:106450001620FCE72D20FAE74320F8E75A20F6E75C
:106460007020F4E78720F2E79D20F0E7B420EEE704
:10647000CA20ECE7E120EAE7F720E8E74FF487706D
:10648000E5E74FF49270E2E740F23B10DFE700BF30
:1064900017A30B00CD810B00D2810B00D1810B0023
:1064A000F4A20B00D5810B00B56C0B00D9810B0059
:1064B00031740B00DD810B00DE810B00E1810B00EC
:1064C000D9B90B00E5810B00EA810B00E9810B00D3
:1064D00008B551EC100B07A3D3E9002378F01AFBA1
:1064E000034B002278F040FC41EC100B08BD00BFCC
:1064F00000806640182D4454FB2109400000000034
:1065000008B551EC100B084B002278F003FB04A3F4
:10651000D3E9002378F028FC41EC100B08BD00BF44
:10652000182D4454FB2109400080664000F1080307
:1065300073B5044603600D46E1B108467BF0C8F828
:106540000F2805EB0006019007D9002201A920467B
:1065500072F08CF8019B2060A360206832462946C7
:1065600072F019F9019B2268636000212046D15422
:1065700002B070BD014871F064FE00BF23620B00E1
:106580002DE9F0472DED0E8B55EC114B90B0824666
:10659000DF4909AA0AA859EC108BFFF7C7FFDD4BAA
:1065A00000222046294678F0FFF8DB4B0022044603
:1065B0000D4678F0D9FBD94B002278F0F5F878F049
:1065C00059FD00228AF800004FF07F5340464946AB
:1065D00078F0A0FAD24B002278F0E6F878F04AFD85
:1065E0000A9B1B5C8AF801300022CE4B20462946CC
:1065F00078F0BAFB78F03EFD4FF4B473584378F06E
:106600001FFA02460B462046294678F0CBF8C14BCC
:10661000002278F0C7F8B0A3D3E9002304460D4662
:106620004046494678F076FABA4B002278F09CFB57
:10663000A9A3D3E9002341EC180B2046294678F0A2
:1066400069FAB44B002278F08FFBB74B06460F4631
:1066500000224046494678F0E3FCB8B1B34B002233
:106660004046494678F0C8FC80B1B14B0022204634
:10667000294678F0D5FC48B1AE4B00222046294689
:1066800078F0BAFC10B120238AF80030AA4B00221F
:106690004046494678F0C4FCD8B1A84B0022404699
:1066A000494678F0A9FCA0B10022002320462946E3
:1066B00078F0B6FC002800F05C82A14B0022204656
:1066C000294678F099FC002800F053821F238AF8AD
:1066D00000309AF80000431E06205843B13878F085
:1066E000AFF97DA3D3E9002378F014FA894B002297
:1066F00078F03AFBB0EE480AF0EE680A41EC1D0B68
:1067000072F0AAFF55EC104B10EE100A74A3D3E9F7
:106710000023294678F0FEF922462B4678F0FAF954
:1067200002460B4600207D4978F03CF841EC100B06
:1067300073F028FB6CA1D1E9000153EC102B78F029
:1067400013FBB0EE480AF0EE680A41EC1C0B72F045
:10675000DBFF53EC102BB0EE40BAF0EE60BA51EC18
:10676000100B78F0D7F9B0EE480AF0EE680A41EC69
:10677000190B72F0E9FB55EC104B10EE100A5CA3FC
:10678000D3E90023294678F0C5F922462B4678F054
:10679000C1F953EC1D2B41EC1A0B3046394678F009
:1067A00001F822462B4678F0B5F953EC182B044635
:1067B0000D4651EC180B77F0F7FF41EC100B72F01F
:1067C0004BFF604B002251EC180B8DED000B78F065
:1067D000A1F941EC100B72F03FFF4F4B002251EC3E
:1067E000180B8DED020B78F095F941EC100B72F05F
:1067F00033FF9FED411B8DED040B45EC104B73F007
:10680000EFF953EC192B51EC190B8DED060B78F0C9
:1068100081F94D4B41EC1D0B002251EC190B78F026
:1068200079F902460B460020484977F0BBFF53EC4C
:106830001D2B77F0B9FF404B06460F46002251EC66
:106840001A0B78F067F902460B463046394677F066
:10685000ABFF2BA3D3E9002377F0A4FF22462B46FE
:1068600078F058F922462B4678F054F922462B4608
:1068700078F050F922462B4678F04CF922462B4608
:1068800078F048F9324B002278F06EFA53EC192B6D
:1068900006460F460020214977F084FF53EC1A2B5F
:1068A00077F082FFDDE9062378F034F91A4B0022F5
:1068B00078F05AFA22462B4677F076FF02460B46CE
:1068C0003046394677F070FF0FA3D3E90023064620
:1068D0000F463FE0AFF30080182D4454FB210940E0
:1068E0008004ACF2906B7B3F00000040A6545841FE
:1068F000DDA447E2DF9A7B3F000000000000084073
:1069000068ED10E55A04D93F789CA223B9FCEF3F0B
:10691000ED810B0000806640000018400000F03F51
:10692000000024400080764000004C4000005040B1
:106930000000084000002840000052400000554080
:1069400000002240000010400000324000001440CF
:1069500000005E4051EC1C0B78F0DCF802460B4660
:106960003046394678F0D6F8BFA3D3E9002377F054
:106970001BFF78F0A7FB53EC192BCAF80400AE49B3
:10698000002077F00FFFAD4B06460F46002251EC7A
:106990001A0B78F0BFF802460B463046394677F0BE
:1069A00003FFA74B06460F46002251EC1A0B78F066
:1069B000B1F853EC1A2B78F0ADF802460B4630468E
:1069C000394677F0F1FE22462B4678F0A3F82246AE
:1069D0002B4678F09FF822462B4678F09BF822460B
:1069E0002B4678F097F8974B002278F0BDF92246B5
:1069F00006460F462B462046294678F08BF8924BE8
:106A0000002278F087F802460B463046394677F088
:106A1000CBFE8E4B41EC1E0B002251EC190B78F093
:106A200079F802460B460020894977F0BBFE53EC0B
:106A30001D2B77F0B9FE874B06460F46002251EC1E
:106A40001A0B78F067F802460B463046394677F065
:106A5000ABFE69A3D3E9002377F0A4FE22462B46C0
:106A600078F058F822462B4678F054F822462B4608
:106A700078F050F822462B4678F04CF822462B4608
:106A800078F048F822462B4678F044F8724B002202
:106A900078F06AF902460B4651EC1E0B77F084FE43
:106AA00053EC1C2B04460D4651EC1B0B78F032F8CE
:106AB00002460B462046294678F02CF850A3D3E92D
:106AC000002304460D4651EC180B78F023F84EA332
:106AD000D3E9002306460F46DDE9000178F01AF8F5
:106AE00002460B463046394677F05CFE48A3D3E9B0
:106AF000002306460F46DDE9020178F00BF8024656
:106B00000B463046394677F04FFE43A3D3E90023C6
:106B100006460F46DDE9040177F0FCFF02460B460E
:106B20003046394677F03EFE3DA3D3E9002377F0A7
:106B3000F1FF02460B462046294677F035FE3AA380
:106B4000D3E9002377F0E6FF78F0BCFA0022044690
:106B500000234046494678F04FFA00283DD1CAF854
:106B600008400AA871F0A4FD10B0BDEC0E8BBDE882
:106B7000F087324B00222046294678F051FA40B186
:106B8000364B00222046294678F036FA08B12123F8
:106B90009DE5324B00222046294678F041FA40B16B
:106BA0002F4B00222046294678F026FA08B12323ED
:106BB0008DE52B4B00222046294678F031FA00283B
:106BC0003FF487AD274B00222046294678F014FA7F
:106BD00000283FF47EAD252379E5204677F020FF9D
:106BE00013A3D3E9002377F0DFFD78F06BFACAF83E
:106BF0000800B6E7AFF30080422DD84CD2CA01405E
:106C000061AE94CC45F2EF3F2C024D638399643F13
:106C10004ABA6F364F23C63EFC48CCE45C5C2D3E3E
:106C200000000040A6545841789CA223B9FCEF3FD5
:106C300000000000D0126341000014400000224018
:106C400000001040000038400000E03F00004D40D0
:106C500000804E4000C082400080864000003540E9
:106C600000804040000045400000000080841E413C
:106C70002DE9F043A7B0064608AA4349DFF8208172
:106C800014A88DED020B8DED001BFFF74FFC08AA39
:106C90003E491AA8FFF74AFC08AA3D4920A8FFF779
:106CA00045FC05AA3B4908A8FFF740FC05AA3A495C
:106CB0000EA8FFF73BFC9DED001B9DED020B05A808
:106CC000FFF75EFC9DF81440BDF814303380013CA2
:106CD000032394FBF3F303EB4303069FB7FBF8F0A6
:106CE000E51A4FF0180926AB09FB053577F098FE39
:106CF00000222A4B77F056FD78F0E4F955F8483C2D
:106D0000079D1B5CB370284677F08AFE1CA3D3E96D
:106D1000002378F029F841EC100B72F075FB002C81
:106D200004F00104B8BF644251EC100B26AB09FB20
:106D3000043478F09FF9142390FBF3F202FB130361
:106D400054F8782CD35CF37097FBF8F308FB1377B7
:106D500095FBF8F308FB13550EA87760B56071F04A
:106D6000A7FC08A871F0A4FC20A871F0A1FC1AA847
:106D700071F09EFC14A871F09BFC27B0BDE8F08375
:106D800000000000006AF84003820B000C820B0038
:106D9000C4810B0015820B002A820B000000F03F1B
:106DA000A08601000000000010B504462DED048B04
:106DB000006877F045FE2AA3D3E9002377F0AAFE06
:106DC00041EC180B606877F03BFE25A3D3E9002364
:106DD00077F0A0FEB0EE480AF0EE680A41EC190B1D
:106DE00004F10C00B0EE491AF0EE691AFEF7FEF954
:106DF000B0EE491AF0EE691AB0EE480AF0EE680AF1
:106E000004F12000FFF7BCFBB0EE491AF0EE691A5E
:106E1000B0EE480AF0EE680A04F12C00FFF728FFF4
:106E2000B0EE491AF0EE691AB0EE480AF0EE680AC0
:106E300004F13800FEF7C8FDB0EE491AF0EE691A09
:106E4000B0EE480AF0EE680A04F14400FEF768FA72
:106E5000BDEC048B002384F8503010BDAFF30080EC
:106E600048AFBC9AF2D77A3E10B50446C0E900128A
:106E70008360142200210C3079F010F90023C4E95A
:106E80000833C4E90B33C4E90E33C4E91133A362F8
:106E900063632364E3640123204684F85030FFF7E2
:106EA00083FF204610BD10B490F8504044B90468E8
:106EB0008C4205D14468944202D184689C4209D036
:106EC000012480F85040C0E900125DF8044B836053
:106ED000FFF76ABF5DF8044B704700000000000038
:106EE0002DE9F04F2DED048B0F461146A1B0096836
:106EF000064698460BA8D2E90123FFF7B5FF9DF897
:106F0000B8300B989DF83890002B14BF50234E23B7
:106F10000028D8BF404209EE103A77F091FD0446B0
:106F200048460D4677F08CFD2FA3D3E9002377F078
:106F3000F1FD02460B462046294677F033FC2CA390
:106F4000D3E9002377F0E6FD41EC180B0C989DF88F
:106F500041409DF840500028D8BF404277F070FD76
:106F60009DF848300893824620468B46CDF8248011
:106F700077F066FD1CA3D3E9002377F0CBFD024632
:106F80000B465046594677F00DFC19A3D3E9002370
:106F900077F0C0FDCDE90454CDE9060119EE103AB1
:106FA0000F4ACDF800908DED028B394630467AF0CD
:106FB00067FA012204460023A24203D2B15C0132E7
:106FC0004B40F9E7074A391B30197AF059FA204447
:106FD00021B0BDEC048BBDE8F08F00BFAFF30080A3
:106FE0004C820B0075820B0000000000D012634140
:106FF00054E41071732AD93E2DE9F04F2DED048B26
:107000000F461146A1B04968064698460BA8536939
:10701000D268FFF729FF9DF8B8300B989DF838909B
:10702000002B14BF50234E230028D8BF404209EE46
:10703000103A77F005FD044648460D4677F000FD0E
:107040002FA3D3E9002377F065FD02460B462046C7
:10705000294677F0A7FB2CA3D3E9002377F05AFD4C
:1070600041EC180B0C989DF841409DF840500028C9
:10707000D8BF404277F0E4FC9DF848300893824640
:1070800020468B46CDF8248077F0DAFC1CA3D3E9A8
:10709000002377F03FFD02460B465046594677F0F5
:1070A00081FB19A3D3E9002377F034FDCDE9045423
:1070B000CDE9060119EE103A0F4ACDF800908DED9A
:1070C000028B394630467AF0DBF901220446002370
:1070D000A24203D2B15C01324B40F9E7074A391BA7
:1070E00030197AF0CDF9204421B0BDEC048BBDE815
:1070F000F08F00BFAFF300804E820B0075820B0053
:1071000000000000D012634154E41071732AD93E8C
:107110002DE9F04F2DED028B1446B3B05369D268C0
:10712000804689461DA86168FFF79EFE236A0026F7
:107130001AA8CDE91A3678F0A3FD054600F09CF8B0
:1071400048B13146012000F027FACDE91A061AA805
:1071500078F096FD0546D5E9013B1D981793002868
:107160002B681893D8BF4042636A199377F068FC84
:107170009DF880A0064650460F4677F061FC3AA382
:10718000D3E9002377F0C6FC02460B463046394669
:1071900077F008FB36A3D3E9002377F0BBFC41EC82
:1071A000180B1E989DF889609DF888700028D8BF3C
:1071B0004042002577F044FCCDE912554D23119350
:1071C000626BCDE90F321F9B0E93E36B0D93236E21
:1071D0000C93A36D0B93CDE914019DF890300A93A5
:1071E000304677F02DFC20A3D3E9002377F092FC02
:1071F00002460B46DDE9140177F0D4FA1CA3D3E96B
:10720000002377F087FC199B0293189B0193179B2F
:10721000134A0093CDE908015B46CDE906768DED72
:10722000048BCDF80CA0494640467AF029F901229A
:1072300004462B46A24204D218F8021001324B40F9
:10724000F8E7084AA9EB040108EB04007AF018F902
:10725000204433B0BDEC028BBDE8F08FAFF300806B
:107260007D820B0075820B0000000000D01263418C
:1072700054E41071732AD93E014B1878704700BF4F
:10728000AC82002010B586B0002102A87BF0A8FADD
:1072900030BB61F07FF8134A13491278029B044611
:1072A00008687AB91149124A00F6A860F7F7BCFFDE
:1072B000104BDDE902011C600F4BC3E90001012006
:1072C00006B010BD042A96BF0C490D4A51F8222081
:1072D000009206490B4A00F6A860F7F7A5FFEEE713
:1072E0000020EDE7AC820020407F00206C5C0B00AA
:1072F000D7820B00A8820020B082002064850B009A
:10730000BF5B0B00F8820B002DE9F74F88469146D2
:10731000044661F03FF8D8E900AB7DA3D3E9002330
:10732000524573EB0B03074619DB614C43F698217A
:10733000206824F042FB18B1032003B0BDE8F08FB1
:107340005C4B5D4A18685D4B00935D49534600F6FF
:10735000A860F7F769FF61F01DF82060ECE752A321
:10736000D3E90023524573EB0B0315DA504C43F677
:107370009821206824F021FB0028DDD14D4B514A93
:1073800018684E4B4E49CDE9003200F6A8604E4ACF
:107390005346F7F749FFDEE74C4D464E2B78B9F1DF
:1073A000000F43D0042B96BF494A4A4B52F8233072
:1073B00030684949042C96BF454A464A52F8242071
:1073C000009200F6A860454AF7F72EFF444B95F867
:1073D00000901F60022C88BF424B2C7088BF1F603A
:1073E000414BD8E900011F60404BC3E90001FFF7A2
:1073F00049FFB9F1000F17D12A78AAB13C4C216896
:1074000091B1042A98BF324B306894BF53F82230B0
:10741000304B009300F6A860364B374A2E49F7F7F9
:1074200003FF20682FF09AFB012086E79C420ED9CB
:10743000042C98BF264B306894BF53F82430254B5A
:107440002E4A254900F6A860F7F7EEFEBEE7042CA9
:1074500006D130682A4A53461F4900F6A860F3E770
:10746000032C09D11E4B2749186824F0A6FA18B935
:107470003068254A5346EFE72B7830681649042BCD
:1074800096BF134A134B52F82330042C96BF104A70
:10749000104A52F82420009200F6A8601B4AF7F721
:1074A000C3FE002049E700BFC070BEB50000000069
:1074B000B8820020407F002036830B00C0648E6AB3
:1074C000D9610B00C070BEB562830B00AC82002096
:1074D00064850B00BF5B0B006C5C0B00B0830B0082
:1074E000BC820020C0820020A8820020B082002040
:1074F000C83C0120A0840B00A5840B00FA830B007C
:1075000015840B0040771B0030840B0066840B0051
:10751000BF648E6A0000000038B50E4C0E4D68B195
:1075200060F038FF24682D68001B4FF47A74B0FBBC
:10753000F4F400F013F82844204438BD60F02AFF2A
:107540002368C01A4FF47A73B0FBF3F02B68184429
:10755000F3E700BFA8820020B082002037B50020EA
:10756000FFF7DAFF002300906846019378F088FB6C
:107570004FF0FF330362DDE9004578F06FFE02460D
:107580000B462046294678F051F951EC100B77F064
:1075900071FD03B030BD0000044B1B78834202D361
:1075A0000846FFF7B9BF0020704700BFAC8200203B
:1075B00070B5446904F26B73002B1946B8BF04F22E
:1075C0006E716FF0630293FBF2F202EBA1024FF4D3
:1075D000C87593FBF5F10A4440F26D1101FB0323DA
:1075E00002691849A3F52F23012A51F82210A3F6A6
:1075F0003A130FDD04F26C72A4070BD1642692FBE0
:10760000F6F406FB142424B992FBF5F405FB1422CE
:1076100002B90131C2680C4C013A19448368114423
:107620004FF461625A43D317C4FB012344680068D6
:107630003C216143521843EBE1730446101843EBBD
:10764000E47170BD78850B008051010000000000DE
:10765000F0B5074687B008460E46FFF7A9FF044677
:107660000D462EA1D1E90001A0424FF0000271EBBE
:107670000503CDE90245049218DB214E43F698211B
:10768000306824F09AF910B1032007B0F0BD1D4B0B
:107690001D4A18681D4B00931D49234600F6A8603B
:1076A000F7F7C2FD60F076FE3060EDE712A1D1E998
:1076B0000001A04271EB050315DA114E43F6982143
:1076C000306824F07AF90028DED10E4B114A186890
:1076D0000E4B0F49CDE9003200F6A8600E4A234652
:1076E000F7F7A2FDDEE77369B3F5967FCCD202A966
:1076F0003846FFF709FEC8E7C070BEB500000000BD
:10770000B8820020407F0020E2840B00C0648E6AB3
:10771000D9610B00C070BEB50E850B00BF648E6AC8
:10772000000000008B1C9A4210B509D9445CEF2C74
:1077300006D144186478B82C02D1C45C8F2C14D0C4
:10774000CC1CA24213D9425CF02A10D101444A78E1
:107750009F2A0CD1C35C8F2B09D1035D4533DBB26B
:10776000042B8CBF0020042010BD0320FCE7002068
:10777000FAE710B5042A86B04FF0000328BF0422B0
:10778000044601A801938DF8083078F05FFC01A948
:1077900003A860F063FB03A9204643F0D9FC04462C
:1077A00003A860F016FB204606B010BD00F0E00311
:1077B000C02B0AD000F0F003E02B08D000F0F80056
:1077C000F02814BF012004207047022070470320D6
:1077D00070472DE9F04F89B0002589460092049347
:1077E0001D608046002800F084808A4280F08680F8
:1077F00083180393835CE22B01D0F02B7ED1CDE97B
:107800000155139B9D4275DA129A02EB05122B016A
:107810000592129A52F803B0BBF1000F3BD09BF8CF
:107820000030002B37D0039A12789A4233D1584651
:1078300079F04EFF064670B3009B03444B4506D8D3
:1078400002465946039878F0F3FB002847D00027FA
:10785000009CBA46A14507D94A4621464046FFF753
:1078600061FF08B10444F5E7564507D93246514651
:107870005846FFF757FF80B18244F5E7A14507D985
:107880004A4621464046FFF74DFF08B10444F5E75C
:10789000009BE61A24D10135B3E7A145FBD908EBDB
:1078A000040318F8040007930BEB0A01FFF77EFFAF
:1078B00006901BF80A00FFF779FF069A8242EAD188
:1078C0001444A145E7D392445645E4D3079B184698
:1078D00078F0AEFB0028DED1069A1744BAE73746A7
:1078E000029BBB42D7D2049B02971E60059B01936B
:1078F000D1E70190019809B0BDE8F08F0195F9E753
:107900002DE9F04F85B0002499460E9B0460054692
:107910008846846043601646002A3ED0A2464FF057
:10792000010B4C4539D2109B01930F9B00932246CB
:1079300003AB49463046CDF80CA0FFF74AFF98B19B
:107940006A68C36885F808B09A42ACBF6A606B6029
:10795000B8F1000F05D0119B82681A442B681344BC
:107960002B60039B1C44DCE74A4621463046FFF768
:10797000D9FE08B10444D4E7305D3119FFF716FF92
:107980000746B8F1000F06D002464046FFF7F1FE69
:107990002B68184428603C44C3E7284605B0BDE87E
:1079A000F08F70B5054686B01E4614469AB1104653
:1079B000059179F08DFE059903460C9A03920B9A76
:1079C00002920A9A2846CDE900622246FFF798FF04
:1079D000284606B070BD1346EFE710B500F10C0362
:1079E000002002468A420BDA53F80C4C2CB1247862
:1079F0001CB11C68A042B8BF204601321033F1E729
:107A000010BD10B588B068B171B10C7874B10A9C22
:107A10000092CDE901340A460023014605A8FFF78C
:107A2000C0FF059808B010BD0846FBE72046F9E7FF
:107A30002DE9F04F2DED028B89B0DDE91447824628
:107A400088461D46164632B90024204609B0BDECD2
:107A5000028BBDE8F08F002BF6D0002313700028B6
:107A6000F2D00029F0D09C42EEDD084679F030FEDD
:107A700008EE100A97B3387898B3189B00933946EC
:107A8000DDE916235046FFF7BCFF4C4B834684428A
:107A9000B8BF1F46384679F01BFE3B78002B08BF65
:107AA0004FF0000BA4EB0B030493189B009381464B
:107AB000DDE9162341465046FFF7A3FFA04205F13A
:107AC000FF3510DC2A464146304679F02EFE002371
:107AD0007355304679F0FCFD0446B6E7BB46374F98
:107AE000D8E78346D6E70024A34618EE103A9C4216
:107AF00036D208EB0403039318F80430E22B01D0CC
:107B0000F02B18D100230793179B0193169B00932A
:107B100018EE101A07AB22464046FFF75AFE50B146
:107B2000079A80683AB1189B1844049B83449B458C
:107B300016DC1444D9E718EE102A21464046FFF718
:107B4000F1FD08B10444D0E7039B1878FFF72EFE3F
:107B50000399059002465046FFF70BFE059AE4E7AD
:107B600034B92A463946304679F0DFFD7455B0E71E
:107B7000AC4228BF2C46B9F1000F08D009EB040332
:107B8000AB4204D9A94534BFA5EB09040024224621
:107B90004146304678F05AFAB9F1000F0BD0A542B1
:107BA00009D92D1BA94528BFA94630194A4639468F
:107BB00078F04CFA4C440023335546E760C20B0082
:107BC0002DE9F04F9DB082460A929DF8A820269C90
:107BD000079288461D46002B00F0F180184679F088
:107BE00077FD299B0393289B0293279B0646CDE9AB
:107BF00000432A460346002113A8FFF781FE149B89
:107C0000A342B8BF23461C1B09930A9B04EBD47400
:107C100003EB640300270B930697B74280F0CF80F5
:107C2000079B7BB17B1CB3420CD2EA5D2A2A09D1A7
:107C3000EB5C2A2B06D1069B83F001030693BC1C48
:107C40002746EAE7324639462846FFF76BFD08B17A
:107C50003C18F5E7289B0193279B0F9000933A4629
:107C60000FAB31462846FFF7B4FD0446D0B1C168DA
:107C7000099AB0F908300A98521A02EBD27200EB56
:107C8000620209B260680190009112B20FFA88F1A5
:107C9000504642F097FFA368299A0F9C13449844DA
:107CA0003C44CDE73C46079B43B1631CB34205D23D
:107CB0002A5D2A2A02D1EB5C2A2B17D032462146B4
:107CC0002846FFF72FFD88B9289B0193279B139027
:107CD0000093224613AB31462846FFF77AFD28B9B8
:107CE000285DFFF763FD0444A642DCD8EB19A742E8
:107CF000089303D1E85DFFF759FD3C18079B002B63
:107D0000069B08BF00230C93E31B059398D0BDF995
:107D10002CB04FF000090027059A07EB09039A429F
:107D200006D9089AD05CFFF741FD3844202844D991
:107D30002FB9059BA3EB0907202F28BF2027089BFD
:107D40003A4603EB090113A878F080F91CAB3B44D9
:107D5000002203F8242C0C9B73B113A910A860F027
:107D60007DF808F1010110AB5A4609B2504643F0C4
:107D7000A5F810A860F02DF813A910A860F06EF80F
:107D800010AB5A460FFA88F1504643F097F810A806
:107D900060F01FF813A910A860F060F810A9504611
:107DA00043F0D6F90D9010A860F013F80D9B98449D
:107DB000059BB9444B45AED842E70746ACE71DB03A
:107DC000BDE8F08F806C20EAE070704700207047BB
:107DD00038B590F84C30012B04460D4605D190F88B
:107DE000403013B1406C41F05BFD94F83410606C8E
:107DF00041F02FFE606C8021F8F7E3FB606C0368B4
:107E000029461B689847606CBDE8384041F089BE40
:107E100030B404680D4611461A46029B2868B3F92F
:107E20000030B2F900200968A44630BC6047012A3E
:107E300003D0022A03D0002070470160FBE70B68E3
:107E40000360F8E7022A06D0032A02D0012A00D1F3
:107E50000160002070470B680360FAE730B4826964
:107E600004695510034604EB6200D20748BF62590B
:107E70005B6930BC48BFD358184730B48269046985
:107E80005510034604EB6200D20748BF62595B6994
:107E900030BC48BFD358184730B4826904695510C4
:107EA000034604EB6200D20748BF62595B6930BCED
:107EB00048BFD358184730B4826904695510034647
:107EC00004EB6200D20748BF62595B6930BC48BF0F
:107ED000D358184707B500680B68019383680BB93E
:107EE00070F0D7F9C36801A9984703B05DF804FBA7
:107EF00010B50446406C41F0D3FCA16C4B1C02D081
:107F0000606C41F029FD012010BD000010B5034B4D
:107F10000360044642F02AF9204610BD7C880B001D
:107F200010B50446FFF7F2FF2046502162F01CF81E
:107F3000204610BDF7B5CC681646114A24F47F04DC
:107F400024F47F44D2E90075B4F1807F0CBF8C7BB0
:107F50004C7BED1BB4EBA50F4FEAA50203D30948F8
:107F6000214670F077F957F824402268009395680D
:107F700033460A4601462046A84703B0F0BD00BF7D
:107F8000CC820020A8850B0010F0800F114B04D18B
:107F900000221A70104B1A7070471A781870C22A93
:107FA0000CD0C32A0DD03E30C0B201280FD90A4BE5
:107FB0001A7862B901221A70BF207047064B00225E
:107FC000E9E7054B00221A7040F0C000704700201E
:107FD000704700BFC5820020C482002010B4019801
:107FE0000968B0F90040064812680068B3F900302B
:107FF00000B1806901945DF8044B12F0DFBD00BF51
:1080000048D9002010B50446006808B140F040FD92
:10801000204610BD08B50248F6F7B0FB08BD00BF0A
:108020004883002090F840302DE9F74F044613B103
:10803000406C41F035FC94F84C30012B3AD1678A02
:10804000C7F180074FF0000A07EBD777FF267F10B4
:10805000D146D0463546A38A5FFA8AF1B1EBD30FF9
:108060005BDA4FF0000C638A5FFA8CF098421CDAFE
:1080700011FB03F30344A2689BB212F803E0E26829
:1080800012F803B0F3450BD08D4228BF0D4688454A
:1080900038BF8846864228BF0646814538BF81469C
:1080A00002F803E00CF1010CDDE762F0D9FB0AF104
:1080B000010AD0E70027FF26B946B8463546A38A0D
:1080C000F9B2B1EBD30F27DA4FF0000C638A5FFAF5
:1080D0008CF098421CDA11FB03F30344A2689BB2B4
:1080E00012F803E0E26812F803A0F2450BD08D42CB
:1080F00028BF0D46884538BF8846864228BF0646B9
:10810000814538BF814602F803E00CF1010CDDE740
:1081100062F0A6FB0137D2E70027FF2D00F0AA800E
:1081200094F84C30012B4FD1236821215B6A204603
:108130009847236856FA87F15B6AC9B22046984788
:108140005FFA87FA23680AEB09015B6AC9B2204625
:108150009847236822215B6A20469847236829466E
:108160005B6A20469847236841465B6A20469847E9
:108170000027A84577D3B246CA4520D847B994F816
:108180003410606C41F065FC606C4021F8F719FA1E
:10819000A268606C638A05FB0323026813F80A1067
:1081A00012680137FFB29047102F03D1606C41F085
:1081B000B8FC00270AF1010A5FFA8AFADCE7013508
:1081C00062F04EFBEDB2D4E7032B1BBFB71C07F0E8
:1081D0000F0B3709C7F3071747F0100308BF06F066
:1081E0000F0B0193A84545D32368A5F150015B6AA5
:1081F000C9B220469847236859465B6A204698478B
:10820000236801995B6A20469847B2460027CA4511
:1082100020D847B994F83410606C41F01AFC606CB7
:108220004021F8F7CEF9A268606C618A05FB012154
:10823000026811F80A10126890477B1CDFB2102FF9
:1082400003D1606C41F06DFC00270AF1010A5FFA6E
:108250008AFADCE717B1606C41F063FC013562F02B
:10826000FFFAEDB2BEE72FB1606C03B0BDE8F04F8E
:1082700041F057BC03B0BDE8F08F000037B50446AD
:1082800090F84401C8B103C96D4685E80300D4F8ED
:10829000400130B1036800211B6898470848F7F790
:1082A00039FE00231A46D4F83C01294660F0F8F95B
:1082B000431E584258410123237503B030BD00BF0F
:1082C0003C810020B5EEC00AF1EE10FA9FED3D7A38
:1082D0000AD530EE070A90F849316BB9012380F8CE
:1082E000493180ED530A7047B4EEC70AF1EE10FA37
:1082F000A8BF30EE470AEEE7D0ED537ADFED326AE1
:1083000030EE670AB4EEE60AF1EE10FA41DD30EE27
:10831000470AB5EEC00AF1EE10FAB4BFF1EE406ABA
:10832000F0EE406AB7EE006AF4EEC66AF1EE10FABB
:10833000D9D4B3EE096AF4EEC66AF1EE10FA32DC73
:10834000B2EE046AF4EEC66ADFED206A9FED206AA1
:10835000F1EE10FAD8BFF0EE466A20EE260AF2EEF1
:10836000086AB4EEE60AF1EE10FA1FDCFAEE086ACB
:10837000B4EE660AF1EE10FA48BFB0EE660A37EEC8
:10838000800AB5EEC00AF1EE10FA12D530EE070AF7
:10839000A7E7DFED106AB4EEE60AF1EE10FA48BF87
:1083A00030EE070AB5E7DFED0C6AD6E7B0EE660AF5
:1083B000E5E7B4EEC70AF1EE10FAA8BF30EE470ABF
:1083C0008FE700BF0000B443000034436666263FD9
:1083D0003333B33E000034C39A99593F0000000084
:1083E0002DE9F0432DED048BB0EE409AF0EE609A4B
:1083F000B0EE418AF0EE618A454D83B05FF0CAFF6E
:108400002A79022A0746E86E39D00B2A414918BF5B
:10841000782117F03DFC95F86830044643B1D5F853
:1084200084004FF4967117F033FC844238BF044641
:10843000394E3A4B3A4D96ED000B9C4251EC100BE5
:1084400098BF4FF4FA684FF000024FF000038DED33
:10845000000B94BF08FB04F84FF0FF3876F0C2FD24
:10846000304C9DED000B60B186ED009B85ED008BDF
:1084700094ED000A03B0BDEC048BBDE8F083254900
:10848000C7E795ED001BB0EE483AF0EE683AB0EE63
:10849000492AF0EE692AFDF7F3FDF2EE047AB4EE14
:1084A000E70AF1EE10FADFF8849009D5D9F8000058
:1084B0000028DDD0381A4045DAD31B4B2360D3E7C0
:1084C00095ED001BB0EE483AF0EE683AB0EE492A5E
:1084D000F0EE692A96ED000BFDF7BAFE10EE100AD9
:1084E00076F0C0FA08A3D3E9002376F013FB76F008
:1084F00009FE86ED009B85ED008B00EE100A2060E2
:10850000C9F80070B6E700BFF8C1631ADCA54C409B
:1085100040CC002080510100388300209BC4200003
:1085200040830020A4610020000080BF348300202D
:10853000F7B50446ADF80410174697491E460022C9
:10854000964BF7F761FE2346954A43F8342BC4E96E
:108550000D33944B944A22630025C4E91135C4E9D4
:108560001743C4E91E4304F18803C4E922338F4B47
:10857000C4F884308E4BE264C4E9263504F150011E
:1085800004F1A403C4E91411C4E9293304F16C0112
:10859000884BA266C4E91B11E5632464A565656682
:1085A0006567C4F88050C4F89050C4F89440C4F88B
:1085B000AC50C4F8A030804BC4F8B040C4E92D35AD
:1085C00004F1C003C4E930337C4BC4F8BC307C4BAD
:1085D000C4F8C850C4E93435BDF80430A4F8E83014
:1085E000FF22012384F8082184F8092184F80A2154
:1085F00084F80B2184F80C2184F80D2184F80E21D5
:1086000084F80F2184F8102184F81121C4E936552B
:10861000C4E93855C4F8CC4084F8EA7084F8EB60BB
:1086200084F8F150A4F8F250A4F8F450C4F80051C2
:10863000082184F81221202084F8132184F81421C1
:1086400084F8152184F8162184F8172184F818215C
:1086500084F8192184F81A2184F81B2184F81C213C
:1086600084F81D2184F81E5184F81F5184F820518C
:1086700084F8215184F8225184F8235184F824513C
:1086800084F8255184F8265184F8275184F828511C
:1086900084F8295184F82A31C4F834512A465FF00D
:1086A000D9FFC4E94F0528B9464B474A4748162128
:1086B00040F0ACFA9623A4F84831C4F8445104F5CC
:1086C000AA70F7F72BFC4FF4A76040F0CFF9102207
:1086D0005323C0E9002300F10802134600F5A76008
:1086E0009D6010338342FBD1394B3A4F1A603A4BAD
:1086F000D3F88450394B1868394B6A1E9A4200F6F9
:10870000A86040D82B46374A3749F6F78DFD374ADF
:10871000C5F3C40302EA25226D09134305F4FC6581
:108720001D433D80502040F08FF905469DF80570AF
:1087300041F0BAFC2E4B2B6000231A46314685F8D7
:1087400040306B64284642F0C8FD4FF0FF33C5E966
:108750000E33284B6B64284BAB64012385F83470CF
:10876000C4F8585184F8F130682040F06DF9D4F81D
:108770005811054642F00AFE2046C4F85C51C4F880
:10878000404103B0F0BD1D4A1749F6F74DFD4FF6C5
:10879000F0733B80C6E700BFEE930B00907F002094
:1087A000A4890B0085A40300B4880B00DC880B00AF
:1087B000E5A40300F0880B00218B030018890B004F
:1087C00035A5030073A10B00F2850B0038860B0062
:1087D000D88200208861002074660020407F00203D
:1087E000D6E2360F4E860B002D5E0B0000F8FFFF21
:1087F0007C880B00604E012060AE0A007E860B0074
:1088000090F8443170B504460D4633B390F84531C5
:108810008B4222D0174E09B3174B184A18681849D3
:1088200000F6A860F6F700FD164A30684FF4807134
:10883000F6F722FBD4F8580142F093FCD4F8580123
:1088400042F08FFC236801261B6826750021204614
:1088500098470D4B1E7084F8455170BD094A306829
:108860004FF48071F6F709FBD4F8580142F07DFC13
:108870002575F0E7987E0020407F0020B1860B0030
:108880002D5E0B0060C20B002AA1002090F8483139
:10889000C02B9CBF3E33DBB280F84831704790F864
:1088A0004831452B84BF3E3BDBB280F848317047EE
:1088B00010B5084B04461E21D0F85C01196042F047
:1088C000A9FD236800211B6820469847024B01221E
:1088D0001A7010BD906100202AA1002009B1FFF795
:1088E000E7BF704713B50446D0F85C01019142F030
:1088F000BCFDD4F85C010199012242F0F7FD20464D
:1089000002B0BDE81040FFF7D3BF0000124B134A7E
:10891000134910B50446186800F6A860F6F784FC01
:10892000104A1068002310F0010084F846310CD181
:108930000D4B0E4919600E49D9600E49996001230B
:1089400013600D490D4A6FF0D2FA20460649BDE882
:108950001040FFF7C7BF00BF407F0020C0860B005C
:108960006C5C0B00C8820020488300205181040009
:10897000117E03002F7E030015800300006000209D
:1089800010B50446D0F85C0142F0A1FD037B012B39
:108990000CD1D4F85C0142F0D5FD5FF0FBFC044B38
:1089A00018602046BDE81040FFF782BF10BD00BF31
:1089B0003083002038B50446D0F85C010D4642F003
:1089C00086FD037B012B10D1D4F85C0155B942F030
:1089D000B9FD5FF0DFFC054B18602046BDE838406C
:1089E000FFF766BF42F04EFDF3E738BD308300204D
:1089F0000FF0FEBB0F4B07B593F8F820AAB9082378
:108A00000C21CDE900310C4801230079042116F036
:108A1000E7F950B1094B1B6843B193F85020012A84
:108A200003D193F85830092B00D8002003B05DF82B
:108A300004FB00BF68D5002040CC002018A1002016
:108A400038B505460C200C463FF0FEFF291D84601A
:108A50006FF052FAEB680133EB600C203FF0F4FF4B
:108A6000214685606FF048FAA3680133A36038BDE2
:108A700038B5002383608B6804460D462BB1022273
:108A80009847EB68E360AB68A360204638BD38B513
:108A9000002383608B6804460D462BB10222984761
:108AA000EB68E360AB68A360204638BD38B50023AF
:108AB00083608B6804460D462BB102229847EB6811
:108AC000E360AB68A360204638BD1FB50446684626
:108AD000FFF7ECFF6A4600212046FFF791FE68464B
:108AE000F5F74CFE04B010BD07B529B91146FFF7E4
:108AF000ECFF03B05DF804FB012300226946CDE9D9
:108B00000032FFF7BBFBF4E71FB500236946029371
:108B1000FFF7DBFF6846F5F731FE05B05DF804FBB3
:108B20002DE9FF4190F8453104460D46A3B1B54B00
:108B30001B78052B14D107C9B34B83E80700B34951
:108B4000D4F85C01022242F099FC2046FFF7B0FE07
:108B5000D4F85C0142F076FF002004B0BDE8F0815B
:108B60000FF046FB0646B0B195E80700A64B83E838
:108B70000700A749D4F85C01022242F07FFC20469E
:108B8000FFF796FED4F85C0142F05CFFD4F8580180
:108B90000BF0E4F9E0E7D4F85C0142F098FC94F8BB
:108BA0001231427B9A421DD12B79112B0BD1994B5B
:108BB0009A699B689A4224D1974B324618684FF0C5
:108BC000FF3129F063FC2B79122B0BD1914B9A6961
:108BD0009B689A421BD1904B002218684FF0FF31DE
:108BE00029F054FCD4F85C0142F071FC94F8133184
:108BF000427B9A420ED12B79112B4DD10DF03EFCC8
